:020000040800F2
:10000000000001105D030408D143030825F1000836
:10001000610404086104040861040408000000008D
:10002000000000000000000000000000CD430308B5
:10003000C943030800000000C543030895070108F1
:1000400061040408610404086104040861040408EC
:100050006104040861040408F19B0008E19C0008A5
:1000600061040408A59C0008699C00081DB90008EB
:100070000DB90008FDB80008EDB80008DDB80008AB
:10008000C9B80008B5B80008610404086104040890
:100090006104040861040408610404082D9C00083C
:1000A00001F8000871F800086104040881F80008EC
:1000B00061F8000851F8000841F80008F9BE00088E
:1000C00001BF0008EDBE0008F5BE00086104040889
:1000D000610404085909010861040408BD08010805
:1000E000B59B000861040408414F0308F1F70008BC
:1000F00011F800086104040821F80008A1B80008FC
:10010000610404086104040831F80008610404086B
:10011000610404086104040861040408610404081B
:100120008DB8000879B8000865B8000851B8000813
:100130003DB800086104040861040408610404086F
:10014000610404086104040861040408893D03088B
:1001500029B8000815B8000801B8000821080108EE
:10016000E1BE0008E9BE0008610404086104040857
:1001700061040408610404086104040861040408BB
:08018000610404086104040895
:08018800F4FE03000100000079
:10019000160008009C240020A42400200000000079
:1001A000180600081D000100D42800206429002042
:1001B000000000002006000827000400F4280020AA
:1001C0006829002000000000220600080101040048
:1001D000CC29002070380020000000000000000042
:1001E000080209001C3800207438002000000000BC
:1001F000D781000806020C00253800208038002036
:100200000000000059910008070202004838002051
:100210008C3800200000000026060008FF010100C5
:100220005C380020903800200000000028060008FC
:1002300002000C0034380020943800200000000038
:1002400000000000030001005C3A0020643A002036
:10025000000000000000000003123200D23B00202A
:10026000A03B0020000000000000000025005A0014
:10027000EC3A0020463B0020000000000000000097
:10028000F6010800E43A0020DC3A002000000000FB
:100290000000000001000A00FC4100204C42002048
:1002A000000000002A0600081A000800E4410020AF
:1002B00058420020000000003406000829005000C9
:1002C0007C460020444700200000000000000000A1
:1002D000140002007846002094470020000000002F
:1002E0003C06000810000300E84500209847002065
:1002F000000000003E06000828000C00DC4500203D
:100300009C4700200000000042060008260008006C
:10031000D4450020A8470020000000004E06000839
:1003200023000E00DC440020B04700200000000045
:10033000E143020819000500CC450020C047002019
:100340000000000056060008F8010100C845002022
:10035000C8470020000000005C06000800010400FF
:10036000C4450020CC470020000000005E060008C5
:10037000010205000C4D00207C510020000000000F
:10038000E969020800020500D047002084510020DE
:1003900000000000000000001E000400184B0020B8
:1003A0008C510020000000006206000822000C00B2
:1003B000984A0020905100200000000066060008C6
:1003C0000E00DE0008520020306000200000000017
:1003D00031EA0108130004001853002010610020C6
:1003E000000000007406000802010300F75100201D
:1003F00014610020000000003581010818002C0065
:1004000078740020A474002000000000D9DA0208EB
:1004100006001A00E46F0020D074002000000000E5
:1004200051EA010834001000106F0020EC74002025
:1004300000000000A9CC0308FB010100EC6D0020C6
:10044000FC74002000000000DDE50008FC0109004C
:10045000B46C00200075002000000000A9E5000831
:10046000F7010600AC6C00200C75002000000000B5
:10047000780600080A001200186100201475002098
:10048000000000007E0600081F000E009876002085
:10049000C076002000000000900600080502010060
:1004A00084760020D0760020000000009E06000820
:1004B0000301060012760020D47600200000000020
:1004C000A00600082C0010004C7900203C79002088
:1004D0000000000075D602082B002400807900205F
:1004E0005C7900200000000045D602081B00F400E3
:1004F000AC7900202C7B002000000000F969020884
:1005000012001600107B0020207C0020000000005C
:10051000A60600080B100C00808300202885002010
:1005200000000000BC0600080C00240066850020C6
:100530001086002000000000392F02080D00340052
:1005400090990020C499002000000000B124030805
:100550000202030084990020F899002000000000A6
:100560000000000011000C00048E0020FC99002007
:100570000000000035820108FD012400A48600204F
:10058000089A00200000000059810008FE010800C0
:10059000908600202C9A002000000000E5E500086D
:1005A0000400C000F0C70020E4C9002000000000E3
:1005B00000000000F90104005CAA0020A4CA002089
:1005C00000000000C98100082A00600028D0002037
:1005D000C8CF00200000000081CC03081500700087
:1005E00068CE002088D0002000000000000000003D
:1005F0000500050078D10020B4D1002000000000E3
:10060000C8060008F501620010D10020BCD100200E
:0806100000000000ADDB03084F
:10061800C409000019012828000020030000033C39
:1006280001000A0AE8030000640001007E05EA05EB
:10063800B4053200030000010500000000010000BD
:1006480000000000000001155802D903C50300008E
:100658002801000004009001000000000100C8000B
:10066800141E010064002C01280000000801040089
:1006780024010000000000300100005A00000000C2
:1006880090012C01C8006400000000000000010077
:100698000000000500000000040101000000000047
:1006A8000001000000000000000000000000000041
:1006B800000000002B21231E0002000001000A0197
:0506C800010102000128
:1006CD000000803F0000803F0000803F01000000DF
:1006DD0050010000070000000200000000000000B3
:1006ED00000000000102030406070809FF010000D5
:1006FD000000803F74340408050804000000000069
:10070D0000540408985304086034040800000000E5
:10071D00A034040805080A00000000000054040875
:10072D009853040890510408000000000000803F19
:10073D000000803F00600240106002400000000099
:10074D00000B000000002000000000000000000071
:10075D00006002402860024000000000060C00000E
:10076D0000002000000000000000000000600240BA
:10077D004060024000000000100D0000000020004D
:10078D0000000000000000000060024058600240C0
:10079D0000000000160E0000000020000000000008
:1007AD000000000000600240706002400000000088
:1007BD00200F0000000020000000000000000000DD
:1007CD00006002408860024000000000261000001A
:1007DD00000020000000000000000000006002404A
:1007ED00A060024000000000301100000000200059
:1007FD00000000000000000000600240B8600240F0
:10080D0000000000362F0000000020000000000056
:10081D00000000000064024010640240000000006F
:10082D000038000000004000000000000000000043
:10083D0000640240286402400000000006390000F8
:10084D0000004000000000000000000000640240B5
:10085D004064024000000000103A0000000040001B
:10086D0000000000000000000064024058640240D7
:10087D0000000000163B00000000400000000000DA
:10088D00000000000064024070640240000000009F
:10089D00203C0000000040000000000000000000AF
:1008AD0000640240886402400000000026440000FD
:1008BD000000400000000000000000000064024045
:1008CD00A064024000000000304500000000400020
:1008DD00000000000000000000640240B864024007
:1008ED00000000003646000000004000000000003F
:1008FD0000000000FFFFFFFF554A02080000000046
:10090D000000000001000000E00100000000803F39
:10091D000800000020700020702D7200FA00000009
:10092D000100000001000000789604080F0000008F
:10093D00000000000000000000000000EC1400208A
:10094D00F48F0408FC8F04080490040800000000D4
:10095D00000000000000000000000000DE8F040811
:10096D0004000000F3520308000000000000000026
:10097D000C900408010000000000000000000000C1
:10098D0000000000000000000E000000000000004C
:10099D00000000000000000062C900200100C40931
:1009AD000000000060C900200100C4090000000023
:1009BD005EC900200100C409000000005CC90020D0
:1009CD000100C4090000000058C900200100C4093D
:1009DD00000000005AC900200100C40900000000F9
:1009ED0056C900200100C4090000000054C90020B0
:1009FD000100C40900000000A85100200100C8003A
:100A0D0001000000A65100203200307532000000B8
:100A1D00A5510020055A0500A051002000FF01003E
:100A2D00A45100200100000080020020A2510020EE
:100A3D0002000000445F04089F51002000FF0100E8
:100A4D00A35100200100000080020020A1510020D0
:100A5D0002000000445F0408349004080F000000F9
:100A6D0000000000000000000000000088020020CF
:100A7D00547600209CFF2C0100000000981D0020E2
:100A8D000A000000905104081C760020E0150C1798
:100A9D0000000000991D0020080000009853040874
:100AAD009A1D00200500000000540408B7810020A5
:100ABD0002000000A85104081E530020012001006F
:100ACD001D53002002000000B4510408EE52002016
:100ADD000000F40101000000EC5200200000F401C0
:100AED0001000000EA5200200000F40101000000A6
:100AFD00E85200200000F40101000000E652002041
:100B0D0000FF010002530020E803D0070A00000097
:100B1D0000530020006401000A0000000153002072
:100B2D00006401000A000000FA5200200064010078
:100B3D000A000000FF520020006401000A000000BE
:100B4D00FE520020006401000A000000FD5200204A
:100B5D00006401000A000000F952002000FF0100AE
:100B6D000A000000F852002000FF01000A000000FA
:100B7D00045200200000F401010000000252002088
:100B8D000000F40101000000005200200000F401FB
:100B9D0001000000FE5100200000F40101000000E2
:100BAD00F552002000C80100F452002000C80100D9
:100BBD00F352002000C80100F25200200064010031
:100BCD000A000000F152002000FF01000A000000A1
:100BDD000D53002000C801000C53002000C8010077
:100BED000B53002000C801000A53002000C801006B
:100BFD000953002000C801000853002000C801005F
:100C0D000753002000C801000653002000C8010052
:100C1D000553002000C801003C90040800000000AE
:100C2D000000000000000000000000004C900408CF
:100C3D0009000000000000002C030020040000004B
:100C4D00549004080900000000000000200300205B
:100C5D0004000000F89404080900000000000000E2
:100C6D0014030020040000005C900408090000003B
:100C7D00000000000803002004000000609004083C
:100C8D000900000000000000FC020020040000002C
:100C9D00689004080900000000000000F002002028
:100CAD00040000007090040809000000000000001E
:100CBD00E402002004000000789004080900000000
:100CCD0000000000D8020020040000000C90040871
:100CDD000100000000000000000000000000000006
:100CED00000000000E0000000000000000000000E9
:100CFD0000000000809004080000000000000000CB
:100D0D000000000000000000E49D04080700000042
:100D1D000000000050030020000000009090040827
:100D2D000800000000000000440300200000000047
:100D3D009C9004080800000000000000380300200B
:100D4D00000000000C9004080100000000000000ED
:100D5D000000000000000000000000000E00000078
:100D6D00000000000000000000000000A490040836
:100D7D000000000000000000000000000000000066
:100D8D00B49004080D000000000000008C0300204A
:100D9D0000000000BC9004080D00000000000000E1
:100DAD008003002000000000C4900408070000002C
:100DBD00000000007803002000000000CC90040823
:100DCD000D000000000000006C030020000000007A
:100DDD00D49004080D000000000000006003002006
:100DED0000000000DC900408070000000000000077
:100DFD0058030020000000000C90040801000000C2
:100E0D0000000000000000000000000000000000D5
:100E1D000E000000000000000000000000000000B7
:100E2D00E490040800000000000000000000000035
:100E3D0000000000E49D04080C000000000000000C
:100E4D00AA51002000000000F89004080C000000DA
:100E5D0000000000AC5100200000000008910408C3
:100E6D000C00000000000000E25100200000000016
:100E7D00189104080C00000000000000D65100205D
:100E8D00000000002C9104080C0000000000000080
:100E9D00AE51002000000000945F04080C0000001B
:100EAD0000000000B051002000000000389104083F
:100EBD000C00000000000000B251002000000000F6
:100ECD004C9104080C00000000000000AA51002005
:100EDD0000000000549104080C0000000000000008
:100EED00AC510020000000005C9104080C000000D3
:100EFD0000000000B85100200000000068910408B7
:100F0D000C00000000000000BA510020000000009D
:100F1D00709104080C00000000000000BC5100207E
:100F2D00000000007C9104080C000000000000008F
:100F3D00BE51002000000000889104080C00000044
:100F4D0000000000C0510020000000009491040832
:100F5D000C00000000000000C25100200000000045
:100F6D00A09104080C00000000000000C4510020F6
:100F7D0000000000AC9104080C000000000000000F
:100F8D00C651002000000000B89104080C000000BC
:100F9D0000000000DA51002000000000C09104089C
:100FAD000C00000000000000D851002000000000DF
:100FBD00C89104080C00000000000000E65100205C
:100FCD0000000000D49104080C0000000000000097
:100FDD00E851002000000000E09104080C00000022
:100FED0000000000EE51002000000000FC9D0408F0
:100FFD000C00000000000000C8510020000000009F
:10100D00EC9104080C00000000000000D0510020FD
:10101D0000000000F49104080C0000000000000026
:10102D00CA51002000000000009204080C000000CE
:10103D0000000000CC510020000000000C920408BC
:10104D000C00000000000000CE5100200000000048
:10105D00149204080C00000000000000D251002082
:10106D0000000000046B04080C00000000000000EC
:10107D00DC51002000000000209204080C0000004C
:10108D0000000000D4510020000000002C92040844
:10109D000C00000000000000E451002000000000E2
:1010AD00389204080C00000000000000DE51002002
:1010BD0000000000409204080C0000000000000039
:1010CD00E051002000000000489204080C000000D0
:1010DD0000000000EA5100200000000050920408BA
:1010ED000C00000000000000EC510020000000008A
:1010FD000C9004080100000000000000000000003A
:10110D0000000000000000000E00000000000000C4
:10111D0000000000000000005892040800000000CC
:10112D0000000000000000000000000068920408AC
:10113D000500000000000000FD510020000000002F
:10114D000C900408010000000000000000000000E9
:10115D0000000000000000000E0000000000000074
:10116D000000000000000000709204080000000064
:10117D00000000000000000000000000B88F04080F
:10118D000000000000000000E61700200400000031
:10119D007C9204080D000000AD520308EC03002002
:1011AD0000000000949704080D000000A1530308EF
:1011BD00E003002000000000809104080D000000F5
:1011CD0085530308D403002000000000809204081A
:1011DD000800000000000000C8030020040000000B
:1011ED00EC9104080D00000069520308BC030020B7
:1011FD0000000000889204080900000000000000B3
:10120D00B0030020040000009092040803000000C9
:10121D00A9C0030898030020000000000C900408EA
:10122D0001000000000000000000000000000000B0
:10123D00000000000E000000000000000000000093
:10124D00000000009492040800000000000000005F
:10125D000000000000000000A49204080D00000032
:10126D00000000000004002000000000AC92040803
:10127D000A000000000000001F53002000000000C5
:10128D00B89204080A000000000000002753002057
:10129D0000000000C09204080A00000000000000D9
:1012AD002F53002000000000C89204080700000022
:1012BD0000000000F8030020000000000C9004085E
:1012CD000100000000000000000000000000000010
:1012DD00000000000E0000000000000000000000F3
:1012ED0000000000D492040800000000000000007F
:1012FD000000000000000000E89204080700000054
:10130D00000000003C04002000000000F4920408DE
:10131D000800000000000000300400200000000064
:10132D0000930408080000000000000024040020C1
:10133D00000000000C9304080800000000000000ED
:10134D001804002000000000189304080800000095
:10135D00000000000C040020000000000C900408A8
:10136D00010000000000000000000000000000006F
:10137D00000000000E000000000000000000000052
:10138D00000000002493040800000000000000008D
:10139D005702002000000000309304080B000000ED
:1013AD0000000000A4040020000000003893040891
:1013BD000B00000000000000980400200000000059
:1013CD00449304080B000000000000008C04002072
:1013DD0000000000509304080B0000000000000006
:1013ED0080040020000000005C9304080B00000046
:1013FD000000000074040020000000006893040841
:10140D000B00000000000000680400200000000038
:10141D00709304080B000000000000005C04002025
:10142D00000000007C9304080B0000000000000089
:10143D0050040020000000008893040808000000FC
:10144D000000000044040020000000000C9004087F
:10145D00010000000000000000000000000000007E
:10146D00000000000E000000000000000000000061
:10147D00000000009493040800000000000000002C
:10148D000000000000000000A89304080800000000
:10149D0000000000D404002000000000B4930408F4
:1014AD000800000000000000C8040020000000003B
:1014BD00C09304080800000000000000BC040020D8
:1014CD0000000000CC93040808000000000000009C
:1014DD00B0040020000000000C9004080100000082
:1014ED0000000000000000000000000000000000EF
:1014FD000E000000000000000000000000000000D1
:10150D00D4930408000000000000000054020020E5
:10151D0000000000E49304080B0000000000000030
:10152D000405002000000000F09304080B000000EB
:10153D0000000000F804002000000000FC930408E7
:10154D000700000000000000F00400200000000073
:10155D00089404080700000000000000E8040020C3
:10156D0000000000149404080700000000000000B3
:10157D00E0040020000000000C90040801000000B1
:10158D00000000000000000000000000000000004E
:10159D000E00000000000000000000000000000030
:1015AD0020940408000000000000000054020020F8
:1015BD00000000002C94040807000000000000004B
:1015CD0050050020000000003494040807000000BE
:1015DD000000000048050020000000003C940408B5
:1015ED000700000000000000400500200000000082
:1015FD004494040807000000000000003805002096
:10160D00000000004C9404080700000000000000DA
:10161D00300500200000000054940408070000006D
:10162D000000000028050020000000005C94040864
:10163D000700000000000000200500200000000051
:10164D006494040807000000000000001805002045
:10165D00000000006C94040807000000000000006A
:10166D0010050020000000000C900408010000008F
:10167D00000000000000000000000000000000005D
:10168D000E0000000000000000000000000000003F
:10169D00749404080F00000000000000198802086F
:1016AD000000000058050020FB5100200A32010007
:1016BD00FA51002001FA0100F651002000C8010086
:1016CD00F4510020E803D007010000004F4D4E49B2
:1016DD0042555346345344009E51002000030100EF
:1016ED009D510020000301007C9404080F000000B0
:1016FD0055870208318702080000000034060020DB
:10170D00889404080F000000F9860208B9860208C3
:10171D0000000000AC060020949404080F000000A7
:10172D0091870208798702080000000060070020F9
:10173D00A09404080F0000002F880208000000008C
:10174D00C58A0208580A0020A89404080F0000005A
:10175D002D5303080000000000000000A80A00201F
:10176D00B09404080F000000F18B0208C58B02082D
:10177D006D8A0208840B0020B89404080F00000045
:10178D00E5880208B588020800000000240C00203E
:10179D00C09404080F00000061890208A5890208A1
:1017AD0000000000C40C0020F652002001030100CF
:1017BD00CC9404080F0000008188020855880208A7
:1017CD0000000000B40D0020D49404080F000000A8
:1017DD0015890208F58A020800000000400E00205D
:1017ED00E09404080F000000D5890208418B02081F
:1017FD0000000000E00E0020F05200200103010067
:10180D00E894040800000000000000000000000043
:10181D0000000000F494040808000000000000001F
:10182D000010002000000000FC94040807000000D8
:10183D0000000000F80F0020000000000C950408C7
:10184D000700000000000000F00F00200000000065
:10185D00189504080700000000000000E80F0020A4
:10186D00000000002495040803000000A9C003082F
:10187D00D00F0020000000000C90040801000000B3
:10188D00000000000000000000000000000000004B
:10189D000E0000000000000000000000000000002D
:1018AD002C9504080000000000000000000000005E
:1018BD00000000003C9504080A0000000000000034
:1018CD002061040800000000449504080A0000008F
:1018DD0000000000048C0408000000004C95040872
:1018ED000A000000000000000E5300200000000060
:1018FD00549504080A000000000000000C100020A0
:10190D00000000000C900408010000000000000021
:10191D000000000000000000000000000E000000AC
:10192D000000000000000000000000005C950408AD
:10193D00000000000000000000000000000000009A
:10194D006895040803000000A9C003085810002082
:10195D00000000008C94040803000000A9C00308D7
:10196D0040100020000000008094040803000000D7
:10197D00A9C0030828100020000000007495040879
:10198D0005000000000000009C5100200000000038
:10199D007C950408070000000000000020100020C6
:1019AD0000000000889504080700000000000000FA
:1019BD0018100020000000000C9004080100000029
:1019CD00000000000000000000000000000000000A
:1019DD000E000000000000000000000000000000EC
:1019ED0094950408000000000000000000000000B5
:1019FD00000000007460040803000000A9C0030883
:101A0D00A010002000000000A895040803000000AD
:101A1D00A9C00308BC15002000000000B095040803
:101A2D0003000000A9C0030888100020000000007A
:101A3D00B895040803000000A9C003087010002029
:101A4D00000000000C9004080100000000000000E0
:101A5D000000000000000000000000000E0000006B
:101A6D00000000000000000000000000C495040804
:101A7D000000000000000000000000000000000059
:101A8D00D0950408070000008D8B02083811002046
:101A9D00000000001092040803000000A9C0030814
:101AAD002011002000000000DC9504080300000058
:101ABD00A9C003080811002000000000E4950408E7
:101ACD0003000000A9C00308F01000200000000072
:101ADD00EC95040807000000718B0208E810002047
:101AED0000000000B097040803000000A9C003081F
:101AFD00D010002000000000F8950408030000003D
:101B0D00A9C00308B8100020000000000C900408C4
:101B1D0001000000000000000000000000000000B7
:101B2D00000000000E00000000000000000000009A
:101B3D0000000000049604080F000000E187020871
:101B4D00A987020800000000401100200C9604082F
:101B5D000F000000418A0208000000000000000094
:101B6D00E0110020189604080F0000009D86020861
:101B7D0081860208000000006C12002020960408E7
:101B8D000F00000000000000000000000000000039
:101B9D0020130020309604080F000000198A020857
:101BAD00A98B020800000000AC1300203896040831
:101BBD000000000000000000000000000000000018
:101BCD00988E040803000000A9C00308D414002057
:101BDD00000000002496040803000000A9C00308BB
:101BED00BC140020000000001C9604080300000037
:101BFD00A9C00308A41400200000000044960408A6
:101C0D0003000000A9C003088C1400200000000090
:101C1D005096040803000000A9C0030874140020A6
:101C2D000000000058960408020000003D950208CF
:101C3D000000000000000000609604080200000093
:101C4D003D95020801000000000000006C9604089C
:101C5D00020000003D950208020000000000000097
:101C6D00000000000E000000000000000000000059
:101C7D00000000000001010101000000349804087B
:101C8D000F00000049BA020800000000000000002B
:101C9D003C17002008980408000000000000000018
:101CAD000000000000000000B88F040800000000D4
:101CBD0000000000C71700200400000094970408DE
:101CCD000D00000011C30208041C002000000000DC
:101CDD00809104080D000000E9C20208F81B0020E5
:101CED0000000000809204080800000000000000C1
:101CFD00EC1B002004000000EC9104080D00000016
:101D0D0069CE0208E01B002000000000909204083C
:101D1D0003000000A9C00308C81B0020000000003C
:101D2D001898040803000000A9C00308B01B002088
:101D3D00000000000C9004080100000000000000ED
:101D4D000000000000000000000000000E00000078
:101D5D0000000000000000000000000008980408CA
:101D6D000000000000000000000000000000000066
:101D7D00B88F04080000000000000000C717002005
:101D8D000400000040970408030000002DC0020865
:101D9D00981B002008000000EC9104080D000000C5
:101DAD0069CE0208E01B002000000000909204089C
:101DBD0003000000A9C00308C81B0020000000009C
:101DCD001898040803000000A9C00308B01B0020E8
:101DDD00000000000C90040801000000000000004D
:101DED000000000000000000000000000E000000D8
:101DFD000000000000000000000000002098040812
:101E0D0000000000000000000000000000000000C5
:101E1D00B88F04080000000000000000C717002064
:101E2D00040000004897040803000000A9C003083F
:101E3D00101C0020000000000C90040801000000A0
:101E4D000000000000000000000000000000000085
:101E5D000E00000000000000000000000000000067
:101E6D0000FFFF0000000000AA5503009FAA5505C2
:101E7D00010000AA550B010000AA5507010000AA98
:101E8D00550902000000012D202D2D202D2D2D2D69
:101E9D00202D2D2D0000000000000000000000008E
:101EAD000000000000002D202D2D202D2D2D2D208A
:101EBD002D2D2D2D00000000000000000000000061
:101ECD00000000000000000001000000C012000032
:101EDD003275002088130C170100000034750020A6
:101EED0088130C17000000009896040800000000ED
:101EFD00000000000000000000000000A89604088B
:101F0D0008000000000000001C1800200400000064
:101F1D00B49604080800000000000000101800200E
:101F2D000000000090920408040000008DBD02081E
:101F3D0000000000000000000C90040801000000EB
:101F4D000000000000000000000000000000000084
:101F5D000E00000000000000000000000000000066
:101F6D003075002088130C17010000002E7500201D
:101F7D0088130C1700000000F09604080F000000F5
:101F8D0099BA020800000000000000002818002087
:101F9D005C75002001000000C05304082D75002061
:101FAD0001000000CC53040836750020020000002B
:101FBD00D4530408AAC9002000000000000000004E
:101FCD00A8C900200000000000000000A6C90020E4
:101FDD000000000000000000A4C900200000000067
:101FED0000000000A2C90020000000000000000059
:101FFD00A0C9002000000000000000000C18002007
:10200D0000000000000000002C7500200200000000
:10201D00E0530408F89604080000000000000000DA
:10202D000000000000000000A89604080800000051
:10203D0000000000AC18002004000000B496040855
:10204D000800000000000000A018002000000000A3
:10205D00909204080400000079BA02080000000004
:10206D00000000000C9004080100000000000000BA
:10207D000000000000000000000000000E00000045
:10208D000000000000000000000000000897040898
:10209D000000000000000000000000000000000033
:1020AD00189704080D000000B9BC0208E8180020BC
:1020BD0004000000249704080D000000BDBA0208BA
:1020CD00DC18002004000000309704080D0000000B
:1020DD007DBC0208D0180020000000003C970408C9
:1020ED00030000004DC00208B818002008000000D1
:1020FD004897040803000000A9C00308101C002025
:10210D00000000000C900408010000000000000019
:10211D000000000000000000000000000E000000A4
:10212D000000000000000000000000000490040802
:10213D000000000000000000000000000000000092
:10214D005097040804000000F9CD020800000000BB
:10215D00000000000C9004080100000000000000C9
:10216D000000000000000000000000000E00000054
:10217D000000000000000000000000009C97040813
:10218D000000000000000000000000000000000042
:10219D00646D04080D0000000000000048190020C7
:1021AD0004000000AC9704080800000000000000C7
:1021BD003C19002004000000B89704080800000036
:1021CD00000000003019002004000000C097040832
:1021DD000800000000000000241900200400000089
:1021ED00C89704080800000000000000181900201E
:1021FD0004000000D0970408080000000000000053
:10220D000C19002004000000D897040808000000F5
:10221D00000000000019002004000000E0970408F1
:10222D000800000000000000F41800200400000069
:10223D000C900408010000000000000000000000E8
:10224D0000000000000000000E0000000000000073
:10225D000000000000000000E89704080F000000D7
:10226D0089BA020800000000000000005419002087
:10227D00F09704080F0000000000000000000000AF
:10228D0000000000CC190020F89704080F00000092
:10229D000000000000000000000000006C1A00208B
:1022AD008076002004000000EC53040828750020FF
:1022BD00E0150C17000000002B7500200800000031
:1022CD00985304082A7500200500000000540408E6
:1022DD00009804080F00000000000000000000003E
:1022ED0000000000BC1A00200101000058980408ED
:1022FD00B88F040800000000000000006898040872
:10230D007098040800000000012000007498040873
:10231D007C9804080000000001400000809804082B
:10232D00307D040800000000012000008C98040896
:10233D009898040800000000040000009C98040810
:10234D002C9E04080000000004000000A89804085A
:10235D00C473040800000000010000000102000029
:10236D0000000101FFFF000009024300020100C04F
:10237D0032090400000102020100052400100105CC
:10238D002401000104240202052406000107058230
:10239D00030800FF09040100020A000000070501FF
:1023AD00024000000705810240000000FF00000010
:1023BD005D130308151303086512030800000000E0
:1023CD00D10F0308B91103083912030821110308AD
:1023DD000000000000000000C50F03087D3B03084E
:1023ED00793B0308753B0308693B0308653B03080C
:1023FD00713B03086D3B03088D3B0308813B0308CC
:10240D00113C0308253C0308FD3B0308E93B030889
:10241D00D53B030804030904120100020202004027
:10242D008304405700020102030100002515030833
:10243D0045140308C955030815100308F1130308C3
:10244D00251003084110030805100308F50F0308B4
:10245D00000000000000000001010100000000006C
:10246D00010203040102030406070809010000002C
:10247D00306B0408000000000000000045810108D9
:10248D00A086010004000000000000000000000014
:10249D00000000000000000000000000000000002F
:1024AD000000000010920408A0670408000000005E
:1024BD00519D01087D000000060000000000000095
:1024CD0000000000000000000000000000000000FF
:1024DD000000000000000000389A04080000000011
:1024ED0000000000B92F0108E80300000300000000
:1024FD0000000000000000000000000000000000CF
:10250D00000000000000000000000000409A0408D8
:10251D00000000000000000059EB0108102700002A
:10252D00030000000000000000000000000000009B
:10253D00000000000000000000000000000000008E
:10254D00A08E040800000000CDD40208F509010892
:10255D00204E0000050000000000000000000000FB
:10256D00000000000000000000000000000000005E
:10257D0000000000806C0408000000000000000056
:10258D006D2A010810270000010000000000000066
:10259D00000000000000000000000000000000002E
:1025AD0000000000000000004C9A0408000000002C
:1025BD000000000075E50008E803000005000000BC
:1025CD0000000000000000000000000000000000FE
:1025DD00000000000000000000000000589A0408F0
:1025ED000000000000000000A9870108204E000037
:1025FD0003000000000000000000000000000000CB
:10260D0000000000000000000000000000000000BD
:10261D00689A04080000000000000000B185010860
:10262D00204E00000300000000000000000000002C
:10263D00000000000000000000000000000000008D
:10264D0000000000789A040800000000000000005F
:10265D00C5280108400D0300030000000000000024
:10266D00000000000000000000000000000000005D
:10267D000000000000000000FC5F040800000000E6
:10268D00000000004537030810270000010000007E
:10269D00000000000000000000000000000000002D
:1026AD00000000000000000000000000886C04081D
:1026BD000000000000000000D17A02081027000081
:1026CD0003000000000000000000000000000000FA
:1026DD0000000000000000000000000000000000ED
:1026ED00889A04080000000000000000D9F30308D8
:1026FD00A0860100010000000000000000000000A5
:10270D0000000000000000000000000000000000BC
:10271D00000000009C5F04080000000000000000A5
:10272D0001F3030850C30000010000000000000089
:10273D00000000000000000000000000000000008C
:10274D000000000000000000FC9D040800000000D7
:10275D000000000071EE0308A861000001000000F8
:10276D00000000000000000000000000000000005C
:10277D00000000000000000000000000909A040816
:10278D000000000000000000F5810208A086010095
:10279D00010000000000000000000000000000002B
:1027AD00000000000000000000000000000000001C
:1027BD00406004080000000000000000E93301083B
:1027CD00A00F00000100000000000000000000004C
:1027DD0000000000000000000000000000000000EC
:1027ED00000000009C9A040800000000000000009A
:1027FD009DF30208102700000100000000000000FA
:10280D0000000000000000000000000000000000BB
:10281D000000000000000000046C0408000000002F
:10282D000000000071810108A00F000001000000F0
:10283D00000000000000000000000000000000008B
:10284D000000000000000000000000001C960408BD
:10285D0000000000000000002DDD03081A410000FB
:10286D00010000000000000000000000000000005A
:10287D00000000000000000000000000000000004B
:10288D000C680408000000000000000039BE0208BA
:10289D0010270000010000000000000000000000F3
:1028AD00000000000000000000000000000000001B
:1028BD0000000000CC99040800000000000000009A
:1028CD00DD8C02081A41000001000000000000002C
:1028DD0000000000000000000000000000000000EB
:1028ED000000000000000000A89A0408000000008D
:1028FD00000000008D240308400D030000000000BF
:10290D0000000000000000000000000000000000BA
:10291D00000000000000000000000000B09A040854
:10292D0000000000000000009D890108A086010044
:10293D000300000000000000000000000000000087
:10294D00000000000000000000000000000000007A
:10295D0001000000FFFFFFFF01000000685E0C009A
:10296D004300000000000000000000000000000017
:10297D00000000000000000000000000000000004A
:10298D0043000000000000000000000000000000F7
:10299D00000000000000000000000000000000002A
:1029AD0043000000000000000000000000000000D7
:1029BD00000000000000000000000000000000000A
:1029CD0043000000000000000000000000000000B7
:1029DD0000000000000000000000000000000000EA
:1029ED004300000000000000000000000000000097
:1029FD0000000000000000000000000000000000CA
:102A0D004300000000000000000000000000000076
:102A1D0000000000000000000000000000000000A9
:102A2D004300000000000000000000000000000056
:102A3D000000000000000000000000000000000089
:102A4D0081060408C1040408000000004C9E04081F
:102A5D00F18F0408339D0408339D0408339D040849
:102A6D00339D0408339D0408339D0408339D0408E9
:102A7D00339D0408339D0408FFFFFFFFFFFFFFFF99
:102A8D00FFFFFFFFFFFF00000100415343494900D5
:102A9D000000000000000000000000000000000029
:102AAD0000000000000000000000415343494900B0
:102ABD000000000000000000000000000000000009
:102ACD0000000000000000000000000010240020A5
:102ADD0000000000000000000000000000000000E9
:102AED0000000000000000000000000000000000D9
:102AFD0000000000000000000000000000000000C9
:102B0D0000000000000000000000000000000000B8
:102B1D0000000000000000000000000000000000A8
:102B2D000000000000000000000000000000000098
:042B3D000100000093
:10800000436B826A816930B41C68456A24F00104BC
:108010001144AA421C60D9600DD3016900248A1A58
:108020005A6084621A68002142F0010280F84C1004
:1080300030BC1A607047AA1A5A608562F2E700BF26
:10804000436A8269F0B4D154436A0469426B0133D4
:10805000A34228BF00234362FAB1116811F0010165
:1080600001D0F0BC7047856A1768866927F0010760
:108070002E449D421760D6600BD3641B546081620E
:108080001368002143F0010380F84C10F0BC13602A
:1080900070475D1B55608362F2E7826DD36843F0E1
:1080A0008003D360DDE700BF026B10B462B1836C64
:1080B000C2684469D11A013B615C5DF8044B08BF9A
:1080C00013468364C8B27047016A4369C4685B5C45
:1080D0000131A14228BF114601625DF8044BD8B2BC
:1080E000704700BF436B13B190F84C007047836A30
:1080F000406A181AB0FA80F040097047416A836AF2
:1081000099420AD3CB1A416B026961B14968501E8A
:108110000B4483420AD2C01A704702691144CB1A39
:10812000416B0029F2D1501EC01A704700207047E1
:10813000036B43B1826C5B6893422FBF981AC0688F
:108140009B1AC0187047C269036A9A422FBFD01A9F
:10815000C0688018C01A70470A4B30B503F1140488
:1081600093F900205D78072AC8BF143A81180433B8
:108170000D7313F8025C855413F8012C0A76A342A0
:10818000EED130BD7C2C040803682DE9F041DF6995
:108190001FB13B46BDE8F0411847002A164611DDE5
:1081A00004460D460E4400E023689B68204698472D
:1081B0000028F9D0236815F8011B1B682046984752
:1081C000AE42F1D1BDE8F081002325220270437058
:1081D0008370C370704710B5074B03F10C0193F91E
:1081E00000205C78845402449C78D470DC789471CC
:1081F00004338B42F3D110BD902C040830B4446892
:1082000014B12368A5885D83036840F2E93001E07A
:10821000002833D01D89013815F0020F80B2F7D045
:1082200089B2998140F2E93101E0002950D01889E2
:10823000013910F0010F89B2F7D0998940F2E93184
:1082400001E000292FD01889013910F0020F89B2FE
:10825000F7D092B29A8140F2E93201E0002A4BD085
:108260001989013A11F0010F92B2F7D09B8914B12C
:108270002368A2881A83012030BC70472C498B42A6
:1082800008D0A1F578418B424CD001F580618B423A
:10829000D4D10220274901EB00104189013189B274
:1082A00041814189CAE7224A934208D0A2F5784227
:1082B000934235D002F580629342D8D102211D4B02
:1082C00003EB01114B8901339BB24B814B89CEE704
:1082D0001748834207D018498B4227D001F58061A7
:1082E0008B42ABD10221134800EB011148890130C8
:1082F00080B248814989A1E70D498B4207D00E4AD7
:10830000934211D002F580629342B0D10222094B10
:1083100003EB0212538901339BB253815389A6E7C1
:108320000121CCE70120B5E70122F0E70121DAE7DE
:108330000030014090D2002000380040F0B4848921
:108340004FF6FF764FF47A7463B3002A3CD0177867
:10835000013201E0B4421AD00589013C15F0020552
:10836000A4B2F7D0BCB284814FF47A7402E0BCB2FC
:10837000B4420CD0058915F0010504F1FF37F6D0A1
:108380008589ADB209B10D700131013BDCE7104BBD
:1083900098420BD0A3F57843984217D003F5806339
:1083A000984202D00120F0BC70470225094B03EB34
:1083B00005156B8901339BB26B81688980B20030EF
:1083C00018BF0120F0BC7047FF27C5E70125EDE786
:1083D0000030014090D2002070B5044640681E462F
:1083E00010B103688088588341F08001206840F212
:1083F000E93300E0F3B10589013B15F0020F9BB2B0
:10840000F8D08BB2838140F2E93300E093B1058963
:10841000013B15F0010F9BB2F8D08389134631461A
:108420000022FFF78BFF636813B11A689B881383E0
:10843000012070BD0A49884207D00A4B98420DD0EE
:1084400003F580639842E9D10223074901EB031346
:108450005989013189B259815B89DFE70123F4E74A
:10846000003001400038004090D20020002870B554
:108470001EDB0928044620DD012303EB83035B0098
:10848000B0FBF3F2092AF8D87BB10E4EB4FBF3F03F
:108490000928CCBF57223022A6FB03E5024403FB88
:1084A0001044EB0801F8012BF0D100230B7070BDD4
:1084B0002D230B7040420131DBE7303001F8010B16
:1084C000F3E700BFCDCCCCCC884230B44FF00104F0
:1084D0002ED301FB04F4B0FBF4F58D42F9D284B144
:1084E000AAB901E0B0FBF4F5092DCCBF5722302228
:1084F0002A4404FB150003F8012BB4FBF1F4002C13
:10850000F0D100221A7030BC7047B0FBF4F5092D91
:10851000CCBF372230222A4404FB150003F8012B7C
:10852000B4FBF1F4002CF0D100221A7030BC70477B
:108530000546002AEBD1D7E703685A1C0260197080
:10854000704700BF2DE9F047089C2578002B804636
:1085500089460CBF4FF0200A4FF0300A661C35B335
:10856000002A29DD334601E0024698B113F8011BC9
:10857000501E0029F8D1971E60B13D46013D51467D
:108580004046C8476B1C002BF8DC257827EAE770CB
:10859000013055B1041B29464046C847301916F82A
:1085A000015B002DF7D1BDE8F087BDE8F087002A18
:1085B00004DC2846BDE8F0870020EBE7571EDCE727
:1085C0000A44914251D030B441F2210411F8013BE8
:1085D00080EA0320430010F4004F84EA03059BB2B5
:1085E000ADB208BF1D466B0015F4004F84EA0300CE
:1085F0009BB280B208BF1846430010F4004F84EAD3
:1086000003059BB2ADB208BF1D466B0015F4004FC9
:1086100084EA03009BB280B208BF1846430010F4FE
:10862000004F84EA03059BB2ADB208BF1D466B0044
:1086300015F4004F84EA03009BB280B208BF1846CD
:10864000430010F4004F84EA03059BB2ADB208BFAB
:108650001D466B0084EA030015F4004F85B298B202
:1086600018BF28468A42B1D130BC7047836842683F
:10867000D0ED037A00EB83010133934281ED040ACC
:10868000836004BF0023836000EB830393ED047ACF
:10869000036870EE277A9A42C0ED037A77EEC77AC4
:1086A000C0ED037A0CDA013307EE103AF8EEC76A30
:1086B000B7EE007A87EEA60A036030EE070A70472D
:1086C00007EE102AB8EEC77A87EE870A704700BF18
:1086D00090ED097A90ED004AD0ED0A6AD0ED014A9A
:1086E000D0ED047A90ED035AD0ED025AA4EE007A50
:1086F000B0EE406AB0EE470AB0EE667AA6EE247A93
:1087000067EEC07AA0EE457AE6EE257A80ED097A2A
:10871000C0ED0A7A704700BFD0ED057A90ED013ABE
:10872000D0ED003AD0ED064A90ED024A90ED077A7E
:1087300090ED035A90ED086AD0ED045AC0ED067A28
:10874000F0EE406A27EE830AC0ED056AA3EEA60AA2
:1087500080ED087AA4EE240AA5EE470AA5EEC60A23
:1087600080ED070A704700BFD0ED007A90ED017AE6
:1087700030EE670AE7EE007AB0EE670AC0ED007AE5
:10878000704700BF704700BF2DE9F04FDFF81CB203
:10879000DFF81CE2BBF80020DEF80060BBF9043013
:1087A000BBF90250BBF90A80C2EB261404FB04F4A7
:1087B00024135200C2EBE60203FB04F305FB02F2B2
:1087C0009B1303EBE223B3F5FA364FEAE37589B066
:1087D00045F1FF373246A6FB0645CDE9024502FBCF
:1087E00007F205EB4202CDE90467029EBBF908409F
:1087F000039208FB02FC4FEAE87906FB09CC3A46F3
:10880000A8FB0689049ECBF81830E51704FB02F29A
:1088100006FB0522A4FB0667E14417444FEA182231
:1088200042EA096200924FEA292201923D03DDE902
:108830000078340345EA16553F19BBF806600690E8
:1088400048EB05083C1C48F5004503EB8302A4FBFC
:10885000068906FB0599803213124FEA69064FEA32
:10886000E977079356EA07038A4600F09280DDE92C
:108870000489BBF90E20DEF80440BBF9100049461C
:10888000C4F5801ED317DDE9024502FB01F108FBA8
:108890000311A2FB08230B444FEA43492B46C1179F
:1088A00000FB03F304FB0133A0FB0401BBF90C4004
:1088B0001944E30001937346DC170023009349EA4F
:1088C000D2394FEA4248DDE9002310EB080041EBC2
:1088D0000901E50712184FEACE744B4145EA5E05DF
:1088E000A41A65EB0305221945EB050312196B4128
:1088F00099019001801841EA926159418B008200F0
:1089000043EA9073101943EB05018B00820043EAA0
:10891000907310460019194632463B46694137F0BC
:1089200049FBBBF916204C13450B45EAC14502FB38
:1089300004F6D31705FB0366A2FB05233344BBF9FA
:10894000146002FB04F405FB034406FB01FEA2FBDA
:108950000523F717234400FB07EE540EA6FB006720
:10896000774444EAC3144FEAD64800194FEA6365D6
:1089700048EA473869414FEAE74918EB0008BBF974
:10898000124049EB01094FEA182646EA0966200120
:108990003618069B0BB1360A1E60BAF1000F02D0E2
:1089A000079BCAF8003009B0BDE8F08F04470020EB
:1089B00074240020704700BF704700BF2DE9F04FBE
:1089C000DFF8F8C1DFF8F8E1BCF80A70DEF80860FB
:1089D000BCF80C30BCF808A03C028BB0361B4FF042
:1089E0000004CDE90034009CBCF806304FEA17655E
:1089F0004FF0000767EB0507B946B046A4FB0667D2
:108A00000024CDE90634009C002304FB09770024F0
:108A1000CDE90034AAFB0823CDE90223039AF30D24
:108A200000930AFB09230393009B43EA4723009327
:108A3000029B4FEAD31AFB150193039B4AEA436A50
:108A4000DDE9002344464D46CDE90845069C12F574
:108A5000FA62A4FB086743F1000304FB0977CDE940
:108A60000623BCF80440039BBCF802204FEAE31B3A
:108A7000230C059323040493340A44EA07643D124B
:108A8000DDE904674FEAC23816EB0A0647EB0B072D
:108A900018EB0408DDE906344FEA524949EB0509B1
:108AA000B3F5FA6F74F10004B246BB463CDADDE977
:108AB0000067BC00B20044EA9673B41847EB0305A4
:108AC00022463C462B4602FB04F406FB0344A2FB71
:108AD00006232344940844EA83749D105B104FEAF4
:108AE0003202B8EB040869EB0509BAEB020A6BEB3A
:108AF000030BDDE90623304C4FF0FF35A242AB41BA
:108B00002CDBDDE90856A5FB052305FB06F403EB8A
:108B10004403D40F44EA4304DD17DDE90623121BA6
:108B200063EB0503CDE90623DEF80C40A4FB082324
:108B300004FB0933540D44EAC3245D15B4EB0A0A5F
:108B400065EB0B0B4FEADA3343EA4B4300B10360AA
:108B500009B1069B0B600BB0BDE8F08F40F6AC523C
:108B6000B4184FF0000347EB03052246A2FB022393
:108B700004FB05F403EB4403941843EB0305A4182A
:108B80005D414FEA850CA6004CEA947CB41A6CEB6C
:108B90000305DF00D6006D104FEA340447EA527730
:108BA000921B63EB0703B8EB040869EB05091AEBAA
:108BB000020A4BEB030BA4E724FAFFFFF046002068
:108BC000742400204FF480530382704750F8043C13
:108BD000012280F83520143803B11847704700BFD0
:108BE000BFF34F8F0549064BCA6802F4E062134396
:108BF000CB60BFF34F8F00BFFDE700BF00ED00E08B
:108C00000400FA05F8B5027B466903681F2A2DD9CE
:108C1000A2F120055F682024AC402742114617D0FE
:108C20001022AA40DC60DA605A68EA40D40749D4CE
:108C3000716B756A0A68B46A22F00102A5420A6083
:108C400037D1012286F84C20027B11461F2A20D9F9
:108C50002039082258688A40024200D0DA60042293
:108C6000586802FA01F1014221D1F8BD20241D68A3
:108C70009440254211460CD0102191409C6099608F
:108C80001968D140C907D3D5012101FA02F29A60CF
:108C9000CEE7082218688A40024200D09A60042277
:108CA000186802FA01F101420BD09960F8BDD96051
:108CB000F8BD04463046FFF7A3F9227B236811462E
:108CC000C4E7F8BD012202FA05F5DD60B0E700BF98
:108CD00070B4037B04681F2B08D9203B20216268F5
:108CE00001FA03F31A421CD170BC7047202122689C
:108CF00001FA03F31A42F7D042691449582000FBE5
:108D0000021251685689CD680868296821F001016E
:108D10002960828992B222EA06028281A36070BC35
:108D2000704742690949582000FB02125168568970
:108D3000CD680868296821F001012960828992B212
:108D400022EA06028281E36070BC70471070002046
:108D500030B4094B1C786CB1084A002502EBC404FE
:108D6000116893884D628889083203439BB2A242FE
:108D70008B81F5D130BC70473074002034740020F2
:108D800010B4037B01681F2B09D9203B20224C68BB
:108D900002FA03F31C4214D15DF8044B7047202201
:108DA0000C6802FA03F31C42F6D00C4A4068002417
:108DB000147002685DF8044B22F0010202608B60BF
:108DC0007047064A40680024147002685DF8044B3E
:108DD00022F001020260CB60704700BFAF7A002032
:108DE000F0B5C40022189200AE498B585B689D8A8A
:108DF000ADB2EEB2F7070A445CD4B70732D5BFF381
:108E00005F8F167EF6B2012E00F0C780A64D1A8B3A
:108E1000BFF35F8F221801EB8202167E022E00F054
:108E2000D580221801EB8202167E032E00F0888086
:108E30009A8895F9106092B242F480629A80221862
:108E400001EB8202127E013296425BD1AA7C00269F
:108E50006E74002A40F09580204401EB80000023CE
:108E60004375F0BD77074ED416F0400600F0C98078
:108E70008D4D1E8A95F910E0176AF6B207F80E605C
:108E80005FFA8EFE0EF1010C4FFA8CFC177E85F80E
:108E900010C00CF103029742664600F01C812218B4
:108EA00001EB8202127E9445C9D10EF1020676B220
:108EB0002E74C4E71E887C4D26F400663604360CFA
:108EC0001E801E88B6B246F480661E80967E0027FD
:108ED0002F74002E48D06E7C002E42D0221801EB59
:108EE00082020126127E6E74022A00F0B9802218D6
:108EF00001EB8202927D42F001021A82204401EBD2
:108F00008000037EF0BD684D967E0127AF74002E71
:108F100073D06E7C002E7BD1221801EB8202527E30
:108F2000002A00F0A3801A882E7C92B2013642F407
:108F3000007276B21A802E741A88D205FCD47EE7AD
:108F4000927E002A3FF474AF6A7C002A3FF470AF2F
:108F50009A8895F9106022F480621204120C9A80AB
:108F60006DE7D27DFF2AB9D0221801EB8202967DEF
:108F700006F0FE061E82D37DFF2BBFD0FF232B748D
:108F8000BCE79A8822F4407212042044120C01EBD0
:108F900080009A8000234375F0BD927E424D002AE6
:108FA0003FF435AF6A7C002A3FF431AF1A8822F4CF
:108FB00080621204120C1A80BFF35F8F1A8B1A881A
:108FC000AE7492B242F400721A8031E7927E002AA7
:108FD0003FF427AF6A7C002A3FF423AF1A8895F943
:108FE000106022F480621204120C1A809A8822F413
:108FF00080621204120C9A8021E76A7C002A8BD0CE
:1090000091E715F0800F284D3AD195F9106016E7D9
:10901000167ED2F820E01F88022E95F9106045D9FF
:1090200027F480673F043F0C1F801F8AFFB20EF8B1
:1090300006701F88D2F820E0BFB247F400771F8087
:10904000F2B21F8A561C76B2FFB20EF806709F88E5
:10905000961CBAB276B242F480622E749A806BE7A4
:109060001A8892B242F400621A8040E71A8895F991
:10907000106092B242F4807201271A806F745BE72D
:1090800095F91070B7F1FF3F2CD0D669F65D1E82BE
:1090900092F818E001377AB2964516462A747FF4A2
:1090A000CEAEA3E720D2002074240020BFB247F444
:1090B00000771F801F8AFFB20EF80670F6B21F8A73
:1090C000D2F820E0721C52B20336FFB276B20EF82C
:1090D00002702E7430E79A8822F480621204120C17
:1090E0009A80DCE6D77D1F822E74957E1DB9127E94
:1090F000002A7FF403AF9A8822F480621204120CD3
:109100009A80FBE690F8493013B1002280F849209C
:109110001846704770B5044682B00830256A6B4621
:1091200006223B21A847A8B19DF804009DF80060E5
:109130009DF801109DF802509DF803209DF8053020
:1091400041EA062143EA002342EA05226182A28223
:10915000E382012002B070BD0023012243608360DE
:10916000036003714370C271837283704371027232
:10917000C3727047F8B50468C4F30D0405460E4683
:1091800004B32F682CF088FD092840F08880454CF6
:10919000236923F440732361236943F4007323613B
:1091A000236943F0010323613E602CF075FD2369C0
:1091B000092823F00103236171D12B6804332B604C
:1091C0000020F8BD384B394A93422BD902F5804232
:1091D000934226D902F5804293422AD902F5804271
:1091E000934228D902F58032934226D902F5003203
:1091F000934224D902F50032934222D902F500327B
:10920000934220D902F5003293421ED902F5802202
:1092100093421CD9B3F1016F1BD3052006F06EFDFC
:10922000FBE708242CF038FD092814D04FF0FF305C
:10923000F8BD1024F6E71824F4E72024F2E72824E8
:10924000F0E73024EEE73824ECE74024EAE748244E
:10925000E8E75824E6E7134F3B6923F440733B618A
:109260003B6943F400733B613B6923F0F8033B61C6
:109270003B6943F002031C433C613B6943F4803388
:109280003B612CF009FD3B6923F002033B613B6924
:10929000092823F0F8033B613FF473AFC6E76FF092
:1092A0000100F8BD003C024000400008FF3F0008FC
:1092B000F8B504460D468E180027B54201D1206945
:1092C000F8BDE368591CE160234415F8012B1A72BC
:1092D0000429F2D1206918B9A1682046FFF74AFF96
:1092E0002061E760E9E700BFF0B583B004466B4654
:1092F000062203211E2035F0EDFA00283CD09DF80F
:1093000000509DF801109DF802709DF803209DF813
:1093100004609DF8053041EA052142EA072243EA4C
:10932000062309B212B21BB2144D06EE901A07EED4
:10933000102A07EE903AF8EEE66A95ED005AD5ED60
:10934000025A95ED016AB8EEC77AF8EEE77A66EE52
:10935000856A27EE257A67EE867AFDEEE66ABDEE2F
:10936000C77AFDEEE77A16EE901A17EE102A17EE7E
:10937000903A2180A280638003B0F0BD00000020FD
:1093800000B583B001AB03220021772035F0A2FAAB
:109390009DF805309DF804209DF806001B0243EA65
:1093A0000243184303B05DF804FB00BF08B5FFF7A4
:1093B000E7FF014BD86008BD7424002008B5FFF713
:1093C000DFFF014B986008BD74240020682035F051
:1093D00081BA00BF2FF0A6BE70B582B004466946C0
:1093E00018302FF01DFCA8B19DF805009DF8016014
:1093F0009DF802109DF803509DF804209DF806305A
:1094000041EA062143EA002342EA0522A184E284DC
:109410002385012002B070BD03685B6A03B1184761
:10942000704700BF03681B6A03B11847704700BF4D
:1094300003682DE9F041DF691FB13B46BDE8F0410B
:109440001847002A164611DD04460D460E4400E07A
:1094500023689B68204698470028F9D0236815F8B0
:10946000011B1B6820469847AE42F1D1BDE8F08150
:1094700003689B69184700BF03685B69184700BF12
:1094800003681B69184700BF0368DB68184700BF03
:1094900003689B68184700BF03685B68184700BFF4
:1094A00003681B68184700BF014B1868F8E700BF46
:1094B000A025002038B50C46097849B1054601348D
:1094C0002B6828461B68984714F8011B0029F7D120
:1094D00038BD00BF064B53F820302BB11A689B886B
:1094E00051690B4201D1138370475383704700BF0A
:1094F0001CD4002010B50409013C032C17D80D4BD7
:1095000033F8142000F00F0042FA00F313F00103C7
:109510000DD0012303FA00F00138104036F09AFD17
:10952000054A064B125D104403EBC00010BD00203D
:1095300010BD00BF545F0408505F0408C0D2002073
:109540002DE9F04F4A484B494B4B4C4C4FF0010A28
:109550004FF002094FF004084FF0080C4FF0100EC6
:1095600020274026802530F8022B12F0010F03D06F
:109570001960A3F804A0083312F0020F03D0196099
:10958000A3F80490083312F0040F03D01960A3F875
:109590000480083312F0080F03D01960A3F804C048
:1095A000083312F0100F03D01960A3F804E0083359
:1095B00012F0200F02D019609F80083312F0400F84
:1095C00002D019609E80083312F0800F02D019601B
:1095D0009D80083312F4807F05D04FF4807B1960A2
:1095E000A3F804B0083312F4007F05D04FF4007BD9
:1095F0001960A3F804B0083312F4806F05D04FF45B
:10960000806B1960A3F804B0083312F4006F05D022
:109610004FF4006B1960A3F804B0083312F4805FB4
:1096200005D04FF4805B1960A3F804B0083312F43E
:10963000005F05D04FF4005B1960A3F804B0083355
:1096400012F4804F05D04FF4804B1960A3F804B09A
:109650000833D20B04D04FF4004219609A800833CB
:1096600001F58061A1427FF47EAFBDE8F08F00BFBD
:10967000545F040800000240C0D2002000100240E5
:1096800000286AD003682DE9F04F03F13F4404F548
:109690007E045F4EA40A0125345D04F01F066409B0
:1096A000032C05FA06F559D0042C00F0AC80022CEE
:1096B00059D08588B5FA85F0C0F11F0080B2C40882
:1096C00003EB840400F00700266A80000F27874020
:1096D00026EA07062662276A01F003068240701E0A
:1096E0003A430128C1F3810CC1F300182262C1F38F
:1096F00041113DD90024224601274FF0030E03E01B
:10970000102A04F1020426D007FA02F0A84302F15D
:109710000102F5D1D3F800C00EFA04F0C04300EA0C
:109720000C0CC3F800C0D3F8008006FA04FC4CEA25
:10973000080CC3F800C0D3F80CC000EA0C00D860D5
:10974000D3F80CC001FA04F040EA0C00102AD860EB
:1097500004F10204D8D1BDE8F08F70472D4C266C7F
:1097600035432564A5E72B4C666C35436564A0E75B
:10977000002002464FF0010E4FF0030904E00132D1
:10978000102A00F102003CD00EFA02F737EA050475
:10979000F5D1D3F800A009FA00F4E4430AEA040A78
:1097A000C3F800A0D3F800B006FA00FA4AEA0B0AA0
:1097B000C3F800A0D3F808A004EA0A0AC3F808A076
:1097C000D3F808B00CFA00FA4AEA0B0AC3F808A06A
:1097D000D3F804A02AEA07075F60D3F804A008FAC8
:1097E00002F747EA0A075F60DF683C40DC60DF6839
:1097F00001FA00F401323C43102ADC6000F102005F
:10980000C2D1BDE8F08F034C266B3543256350E78A
:10981000EC52040800380240002855D0026802F1DA
:109820003F4303F57E032DE9F04F9B0A544DEB5C5B
:1098300003F01F055B090124032B04FA05F444D04F
:10984000042B00F09780022B44D001F00306731E16
:10985000012BC1F3810CC1F300188588C1F34111BC
:109860003DD90024234601274FF0030E03E0102BBF
:1098700004F1020426D007FA03F0A84303F1010320
:10988000F5D1D2F800C00EFA04F0C04300EA0C0C87
:10989000C2F800C0D2F8008006FA04FC4CEA080CBA
:1098A000C2F800C0D2F80CC000EA0C00D060D2F8B8
:1098B0000CC001FA04F040EA0C00102BD06004F157
:1098C0000204D8D1BDE8F08F70472E4B1D6C2C439D
:1098D0001C64BAE72B4B5D6C2C435C64B5E700203D
:1098E00003464FF0010E4FF0030904E00133102B43
:1098F00000F102003CD00EFA03F737EA0504F5D177
:10990000D2F800A009FA00F4E4430AEA040AC2F813
:1099100000A0D2F800B006FA00FA4AEA0B0AC2F830
:1099200000A0D2F808A004EA0A0AC2F808A0D2F8F7
:1099300008B00CFA00FA4AEA0B0AC2F808A0D2F8FA
:1099400004A02AEA07075760D2F804A008FA03F730
:1099500047EA0A075760D7683C40D460D76801FAE5
:1099600000F401333C43102BD46000F10200C2D15B
:10997000BDE8F08F034B1D6B2C431C6365E700BFF4
:10998000EC52040800380240F0B5044690F84D004F
:1099900083B0002840F0A480674EF77C002F40D0B1
:1099A00004F11805A06935F08BF894F846201A21C7
:1099B0002846FEF723FC012006F0F4FDA06935F0EF
:1099C0006BF8284694F85C10256D6B460622A84774
:1099D000D0B19DF802609DF803309DF800509DF8CD
:1099E00001109DF804009DF8052043EA06231BB2F0
:1099F000E3845BB241EA052142EA00220133A184FB
:109A0000228506D003B0F0BDB4F926305BB2013335
:109A1000F8D194F924300133F4D1062006F06EF920
:109A2000F0E7254655F8180F35F04AF880226B21EB
:109A30002846FEF7E3FB962006F00EFE032268217F
:109A40002846FEF7DBFB962006F006FE03226B217C
:109A50002846FEF7D3FB0F2006F0A4FD10226A2152
:109A60002846FEF7CBFB0F2006F09CFD3A466C2102
:109A70002846FEF7C3FB0F2006F094FD94F848201B
:109A800019212846FEF7BAFB0F2006F08BFD18229D
:109A90001B212846FEF7B2FB0F2006F083FD1022A3
:109AA0001C212846FEF7AAFB0F2006F07BFD1022A2
:109AB00037212846FEF7A2FB0F2006F073FD012296
:109AC00038212846FEF79AFB0F2006F06BFDA069AF
:109AD00034F0E2FF012006F065FD0123F37461E735
:109AE000FFF708FD0546D8B1202300218371C1711D
:109AF000FFF792FE2146114B41F8143F28462FF004
:109B000025F8AB88B3FA83F3C3F11F03012212FADD
:109B100003F33FF441AF0A490A6813430B603BE784
:109B20000146FFF779FE2146044B41F8143F2846D1
:109B30002FF00CF830E700BF74240020CD8B000814
:109B4000003C014010B1036882885A83704700BF0F
:109B500010B1036882881A83704700BF18B1036888
:109B6000828809B95A8370471A83704710B40A4B28
:109B70000A4A1C7801238340234052F8200029B967
:109B8000B3FA83F149095DF8044BE7E7191C18BFE4
:109B900001215DF8044BE1E718D400201CD400201B
:109BA00030B1036882881B691A4214BF012000206B
:109BB000704700BF2DE9F0410B4E346873691C40BB
:109BC0000FD0DFF828800127B4FA84F3C3F11F0314
:109BD00007FA03F558F8230003689847AC4375610A
:109BE000F2D1BDE8F08100BF003C01403486002086
:109BF0002DE9F0410B4E346873691C400FD0DFF83B
:109C000028800127B4FA84F3C3F11F0307FA03F590
:109C100058F8230003689847AC437561F2D1BDE85A
:109C2000F08100BF003C0140348600202DE9F04166
:109C30000B4E346873691C400FD0DFF82880012771
:109C4000B4FA84F3C3F11F0307FA03F558F82300AD
:109C500003689847AC437561F2D1BDE8F08100BF5D
:109C6000003C0140348600202DE9F0410B4E346861
:109C700073691C400FD0DFF828800127B4FA84F301
:109C8000C3F11F0307FA03F558F823000368984748
:109C9000AC437561F2D1BDE8F08100BF003C0140EA
:109CA000348600202DE9F0410B4E346873691C4066
:109CB0000FD0DFF828800127B4FA84F3C3F11F0323
:109CC00007FA03F558F8230003689847AC43756119
:109CD000F2D1BDE8F08100BF003C01403486002095
:109CE0002DE9F0410B4E346873691C400FD0DFF84A
:109CF00028800127B4FA84F3C3F11F0307FA03F5A0
:109D000058F8230003689847AC437561F2D1BDE869
:109D1000F08100BF003C014034860020084A094819
:109D200008B5536C43F4804353640021402238F05B
:109D3000F0FE054B4FF0FF321A60C3F8032008BD58
:109D40000038024034860020748600202DE9F0415E
:109D5000044618460D461646984635F061FC2768BD
:109D6000E6722844A07229467D6943463246204661
:109D7000AC46BDE8F0416047036810B504461B6877
:109D80009847236820469B689847A37B0133A373B9
:109D900010BD00BF10B5036804469B689847FF23B9
:109DA00001226373227310BD08B5FFF7A3FB38B11E
:109DB0002C2282710022C2712021BDE808402BE5CF
:109DC00008BD00BF30B4456815B12B68AA885A8316
:109DD000026841F0800140F2E93301E0002B47D0F6
:109DE0001089013B10F0020F9BB2F7D089B291812C
:109DF00040F2E93301E0002B3AD01189013B11F028
:109E0000010F9BB2F7D09389938940F2E93300E0C8
:109E1000D3B11189013B11F0020F9BB2F8D0FF239F
:109E2000938140F2E93300E073B11189013B11F0F5
:109E3000010F9BB2F8D09489E4B215B12B68AA88BF
:109E40001A83204630BC704715498A4207D0154B0B
:109E50009A4221D003F580639A42EED10223124A3E
:109E600002EB03135A89013292B25A815B89E4E70B
:109E70000B498A4207D00B4B9A420FD003F58063FF
:109E80009A42C1D10223084901EB031359890131D8
:109E900089B259815B89B7E70123E0E70123F2E743
:109EA000003001400038004090D20020F8B5050194
:109EB000684C694B625961199A4204EB050704BF6B
:109EC00001230B730646387A34F0E6FC3B7A03F044
:109ED0001F015B090122032B02FA01F26DD0042B52
:109EE00066D0022B5CD0631901361879FFF702FBAC
:109EF000F6B2074610B11223C671837163195879FF
:109F0000FFF7F8FA10B11323C671837163199879BA
:109F1000FFF7F0FA10B11423C671837166190A2194
:109F2000F2793846FFF7ACFB7079FFF7E3FAF27984
:109F30000A21FFF7A5FBB079FFF7DCFAF2790A21D5
:109F4000FFF79EFB6359454A934247D0424A9342EA
:109F500050D0434A934259D0424A934262D0424A37
:109F600093426BD0414A93422CD02C44227BE2B9DD
:109F700001200222198801F4415141F445710A433C
:109F800002431A809A8B22F400621204120C0721F9
:109F90009A8319821A8892B242F040021A80F8BD60
:109FA000334B596A0A435A629DE700200246E1E7B3
:109FB0002F4B19690A431A6195E72D4B196A0A4319
:109FC0001A6290E702F564424FF40010536A43F4BA
:109FD000001353622BF0C0FE6359C6E702F58432CA
:109FE0004FF48050536A43F4805353622BF0B4FE15
:109FF0006359BAE702F500324FF48040136A43F424
:10A00000804313622BF0B0FE6359AEE702F5FE32D7
:10A010004FF40040136A43F4004313622BF0A4FE94
:10A020006359A2E702F582324FF40050536A43F4B9
:10A03000005353622BF090FE635996E702F5684295
:10A040004FF48010536A43F4801353622BF084FE64
:10A0500063598AE790D20020003800400030014068
:10A06000003C0040003401400050014000540140D9
:10A0700000380240427A02B9704710B504460368BE
:10A08000406804F10A0198470023637210BD00BFC5
:10A09000437A5A1C0344D2B242729972037A9342B1
:10A0A00000D802B9704710B504460368406804F14F
:10A0B0000A0198470023637210BD00BF302828D0E2
:10A0C000312828D0322828D0332828D0342828D046
:10A0D000352828D0202828D0212828D0102828D07A
:10A0E000112828D0122828D0132828D0142828D0A6
:10A0F000152828D0162805D0172808BF0F2202D00F
:10A10000002070470E22114B03EB420393F821000D
:10A1100070470022F7E70122F5E70222F3E7032266
:10A12000F1E70422EFE70522EDE70622EBE707223D
:10A13000E9E70822E7E70922E5E70A22E3E70B223D
:10A14000E1E70C22DFE70D22DDE700BF7C2C0408ED
:10A1500070B5448806460D46C4F30B042246002120
:10A16000284638F0D6FC3369094A934209D3094A94
:10A17000934206D2224628461946BDE8704036F082
:10A18000B1B923B121462846BDE87040184770BDDB
:10A1900018060008CD060008064B07498B4202D37B
:10A1A0000023184670471A88C2F30B029042F8D079
:10A1B0001433F3E79001000818060008024A1368F8
:10A1C00023EA00001060704718530020F8B51A4DBC
:10A1D0002B789F2B2ED16B78BE2B2BD105221749C4
:10A1E000A81C38F0E1FC28BB072229464FF6FF7077
:10A1F000FEF7E6F9124FEC1D22884AB1A618BE42BE
:10A2000018D2052A16D92146FEF7DAF93446F3E7C3
:10A2100021460222FEF7D4F90222A118FEF7D0F956
:10A220000634084B641B1C8041F60F53C31A584276
:10A230005841F8BD0020F8BD004000085C5F0408EC
:10A2400000800008744300202DE9F04FDFF858919A
:10A25000504F8DB00326A7EB090718220DEB020023
:10A26000002138F056FC4C4BCDF8189007971A692E
:10A27000002A04DA494A5A6002F188325A600122FF
:10A280008DF82C20F322DA60454B464C18689A88EA
:10A2900004909B79ADF8142004A9072206A88DF834
:10A2A0001630FFF705F8072204A94FF6FF70FEF7F6
:10A2B00087F9DFF8F8B080464FF0000A5C4539D3E3
:10A2C0000CAC002524F82C5D0222214606A8FEF7DE
:10A2D000EFFF022221464046FEF772F940BAC04322
:10A2E000ADF80800022202A906A8FEF7E1FF0998CE
:10A2F00078B108ABC0F104022946184438F009FCD3
:10A300000A9818B9089906A8FEF734FF00230A90A6
:10A3100009939DF82C300A9A23B11F490B6943F029
:10A3200000430B61013E2DD0002A96D1FFF74EFF6E
:10A3300050B32CE065888DF80DA0C5F30B05AA1D60
:10A34000ADF808202288C2F30B01120BADF80A10F9
:10A350008DF80C2002A9062206A8FEF7A9FF062206
:10A3600002A94046FEF72CF9616880462A4606A8F5
:10A37000FEF79EFF616840462A46FEF721F9143435
:10A3800080469BE7002AD1D0052005F0B7FC0DB030
:10A39000BDE8F08F00800008003C024023016745C3
:10A3A000BC2C0408900100080040000818060008B2
:10A3B0000378202B024600F10100F9D0092BF7D0D9
:10A3C0002D2B2CD02B2B03BF5378B7EE000A02465F
:10A3D000B7EE000AA3F13001C8B209289FED467A12
:10A3E00010D8F2EE046A07EE901AF8EEE77A12F847
:10A3F000013FE7EE267AA3F13001C8B20928B0EE9A
:10A40000677AF0D92E2B4CD003F0DF03452B0BD00D
:10A41000F7EE007A67EE276A20EE260A7047537837
:10A42000BFEE000A0246D5E710B451782D2959D065
:10A430002B290ABF9178501C901C0024A1F13003F5
:10A44000092B53D8002303EB830301EB430310F8DC
:10A45000011FA1F13002092AA3F13003F3D9B3F5AA
:10A460009A7F28BF4FF49A73072B42D9DFED236AF6
:10A470001A46F7EE007A083A072A67EEA67AFAD863
:10A4800003F007032BB1F2EE046A013B67EEA67AF4
:10A49000FBD124B3C7EE276A5DF8044B20EE260AF1
:10A4A00070475378A3F13001C8B2092802F10102C4
:10A4B000AAD8F2EE046AF0EE665A07EE901AF8EEA9
:10A4C000E77A12F8013F87EEA66AA3F13001C8B21D
:10A4D000092866EEA56A37EE067AEED994E767EEAC
:10A4E000276AD9E7901C91780124A7E7F7EE007A54
:10A4F000CFE7F7EE007AC5E70000000020BCBE4CB5
:10A50000B5EEC00ADFED317AF1EE10FACCBF30EED5
:10A51000270A30EE670ADFED2E7A20EE270A30B5E3
:10A52000FDEEC07A87B017EE904A054684EAE470E3
:10A53000002303A9A0EBE4700193009302932FF092
:10A5400031FE002CACBF20232D2303A88DF8003052
:10A5500035F066F8012803A924D002282DD003285D
:10A5600005BF3023684668468DF8013038F0F7FAA9
:10A57000684635F055F80338C4B222466946284685
:10A5800038F04BFB00232B55284635F049F82E2296
:10A59000431C2A540DEB0401E81838F0FDFA284654
:10A5A00007B030BD302368468DF801308DF8023099
:10A5B0008DF8033038F0D3FADAE7302368468DF8A7
:10A5C00001308DF8023038F0CAFAD1E76F12033A41
:10A5D00000007A442DE9F041064615460846B6FBD0
:10A5E000F2F43CB905FB1464124B1B5D00F8013B0F
:10A5F000BDE8F081B4FBF2F767B90E4B05FB1747D6
:10A6000005FB1464DA5D00F8012B1B5D00F8013BCB
:10A61000BDE8F081B7FBF2F8B8F1000F02D0404678
:10A62000FFF7D8FF05FB1878024B13F8082000F855
:10A63000012BE3E7645F040830B402681146531C41
:10A64000036011F8024B0160D31C517803609378CA
:10A65000151D05601B0443EA0123D078234343EA18
:10A66000006030BC704700BF0368591C1A46016087
:10A6700012F8021B0260587841EA0020704700BFC0
:10A6800038B504460068154635F02CFF22682A4488
:10A69000226038BD036810B40A0E5C1C04601A7096
:10A6A00003680A0C5C1C04601A7003680A0A5C1CCC
:10A6B00004601A7003685A1C026019705DF8044B3C
:10A6C000704700BF036810B40A0A5C1C04601A706B
:10A6D00003685A1C026019705DF8044B704700BF94
:10A6E00003685A1C026010B4197003680A0A5C1CE3
:10A6F00004601A7003680A0C5C1C04601A7003681A
:10A70000090E5A1C026019705DF8044B704700BFB7
:10A7100003685A1C026019700368090A5A1C026017
:10A72000197070472DE9F047002488B080460F4625
:10A730001E46A14605AD531C0393117839B3252954
:10A7400033D1931CCDF810900393507830284ED01D
:10A750004FF0000AA0F13003DBB2092B42D96C287C
:10A7600019D0642800F0938024D825281CD063D900
:10A77000582876D063281BD131784046B847039AD1
:10A78000531C03931178043601340029D7D1204695
:10A7900008B0BDE8F087039B5A1C03921B78642B1A
:10A7A0007CD02AD8252B54D1252140460134B847E6
:10A7B000039AC0E7732833D044D975284FD106F1E6
:10A7C000040E30682B4600220A217646FDF77CFEF7
:10A7D000049A0095534639464046FDF7B3FE039A66
:10A7E0000444A8E704AA03A92FF02CF9B7E7D31C67
:10A7F000039390784FF0010AACE7732B10D05BD92C
:10A80000752B3AD0782B96D1A3F15802B2FA82F286
:10A81000306852092B4610210436FDF755FED7E764
:10A820003368049A0093394600234046FDF78AFEB8
:10A8300004360444039A7EE70028B9D1204608B0C4
:10A84000BDE8F0876E28B3D1039A336804361C60E4
:10A8500071E72AD9582BD7D0632B8DD06BE7782896
:10A86000A6D1A0F15802B2FA82F2306852092B4602
:10A870001021FDF729FE0436AAE706F1040E306820
:10A880002B4600220A217646FDF71EFEA0E7331D67
:10A89000306829461E46FDF7E9FD99E7331D30680B
:10A8A00029461E46FDF7E2FD92E7002B7FF443AFF9
:10A8B000204608B0BDE8F0876E2BC6D03BE700BF4E
:10A8C0000EB400B584B005AB019053F8042B0649D3
:10A8D000039301A8FFF726FF019B00221A7004B022
:10A8E0005DF804EB03B07047398500080FB430B54C
:10A8F00083B006AB0A490B4853F8042B096800687B
:10A900000193FFF70FFF084C05462068FEF7B4FDE2
:10A910000028FAD0284603B0BDE8304004B07047A4
:10A92000F8370020FC370020A0250020DFED2B7A2F
:10A93000B4EEE70AF1EE10FA4ADDDFED296A9FED89
:10A94000297A01E0B0EE670AB4EEC70AF1EE10FA18
:10A9500070EE667AF6DC9FED247AF4EEC77AF1EEBB
:10A9600010FA38D5DFED1E6A9FED207A01E0F0EE97
:10A97000407AF4EEC77AF1EE10FA37EEA60AF6D472
:10A98000DFED1B7AB4EEE70AF1EE10FA14DDDFED2D
:10A99000137A37EEC00A60EE006A9FED166A9FEDEB
:10A9A000167ADFED167AA6EE867A20EE266AE6EEB5
:10A9B000877AA6EE270A7047DFED117AB4EEE70A30
:10A9C000F1EE10FA44BFDFED087A37EEC00AE2E795
:10A9D000F0EE407ABFE7B0EE670AD1E7DB0F4940FF
:10A9E000DB0FC940E4CB1641DB0F49C0E4CB16C1F5
:10A9F000DB0FC93F92E741B99730083C15A82ABE42
:10AA0000DB0FC9BF41404A0011F0800F82F0D5032F
:10AA1000D2B2DBB208BF1346590013F0800F81F0A9
:10AA2000D502C9B2D2B208BF0A46510012F0800F57
:10AA300081F0D503C9B2DBB208BF0B46590013F051
:10AA4000800F81F0D502C9B2D2B208BF0A465100C8
:10AA500012F0800F81F0D503C9B2DBB208BF0B46FC
:10AA6000590013F0800F81F0D502C9B2D2B208BFED
:10AA70000A46510012F0800F81F0D503C9B2DBB253
:10AA800008BF0B465A0082F0D50013F0800FD2B2F7
:10AA9000C0B208BF1046704780EAE073A3EBE073D2
:10AAA0008B4205DB002801DD401A704702D1704758
:10AAB000002070470844704709B909E0194690FB27
:10AAC000F1F301FB13030846002BF7D1084670474A
:10AAD0000146FBE7F0EEC07AB0EEE07AB4EEE77A3A
:10AAE000F1EE10FAB4BFB0EE676AB0EE476AB5EEA9
:10AAF000406AF1EE10FA46D0B4EEE77AF1EE10FAC1
:10AB00008CBFF0EE675AF0EE475AC5EE866A9FEDAD
:10AB10001F3A9FED1F6A9FED1F4A9FED1F5ADFED01
:10AB20001F3ADFED1F4ADFED1F5AA6EEC36AE6EEBD
:10AB3000A34AA6EE864AB7EE006AA6EE845AA6EEAF
:10AB4000A46AE6EE855AC5EE866AB4EEE77AF1EEBF
:10AB500010FA48BFDFED147AF5EEC00A48BF77EE71
:10AB6000E66AF1EE10FA48BFDFED107AB5EEC00AE2
:10AB700048BF77EEE66AF1EE10FA48BFF1EE666A7A
:10AB8000B0EE660A7047DFED076ADEE739094E3D31
:10AB9000E3B59E3E88FA163E45FE7F3F99FB243F73
:10ABA00069A2163EA7DFA834DB0FC93FDB0F49407F
:10ABB000DFED317A30EE277AFDEEC76A16EE903A75
:10ABC0002033402B02D99FED2D0A7047B4EEE70ADF
:10ABD000F1EE10FA4DDD9FED2A6ADFED2A6A01E001
:10ABE000B0EE677AB4EEE67AF1EE10FA77EE467AD6
:10ABF000F6DC9FED257AF4EEC77AF1EE10FA35D542
:10AC0000DFED1F6A9FED217A01E0F0EE407AF4EE6D
:10AC1000C77AF1EE10FA37EEA60AF6D4DFED167A0F
:10AC2000B4EEE70AF1EE10FA1BDCDFED197AB4EEB0
:10AC3000E70AF1EE10FA44BFDFED137A37EEC00AEF
:10AC400060EE006A9FED136A9FED137ADFED137AD1
:10AC5000A6EE867A20EE266AE6EE877AA6EE270A28
:10AC60007047DFED0F7A37EEC00AE9E7B0EE670A0A
:10AC7000D4E7F0EE477ABCE7DB0FC93F00000000E5
:10AC8000DB0FC940E4CB1641DB0F49C0E4CB16C152
:10AC9000DB0FC9BF92E741B99730083C15A82ABE1F
:10ACA000DB0F4940FDEEC07A17EE903A2033402B7F
:10ACB00051D8DFED2D7AB4EEE70AF1EE10FA50DD4F
:10ACC000DFED2A6A9FED2A7A01E0B0EE670AB4EE62
:10ACD000C70AF1EE10FA70EE667AF6DC9FED257A7F
:10ACE000F4EEC77AF1EE10FA38D5DFED206A9FED69
:10ACF000227A01E0F0EE407AF4EEC77AF1EE10FA33
:10AD000037EEA60AF6D4DFED1D7AB4EEE70AF1EECF
:10AD100010FA1BDCDFED1A7AB4EEE70AF1EE10FA56
:10AD200044BFDFED147A37EEC00A60EE006A9FED93
:10AD3000156A9FED157ADFED157AA6EE867A20EE7C
:10AD4000266AE6EE877AA6EE270A7047DFED067AD6
:10AD500037EEC00AE9E79FED0E0A7047B0EE670ACA
:10AD6000D1E7F0EE407AB9E7DB0F4940DB0FC9408D
:10AD7000E4CB1641DB0F49C0E4CB16C1DB0FC93F62
:10AD8000DB0FC9BF92E741B99730083C15A82ABE2E
:10AD90000000000010B507EE901A2DED028BB8EE02
:10ADA000678ADFED227A28EE008A044628EE278A99
:10ADB000B0EE480A35F0ECFDF0EE408AB0EE480AFD
:10ADC00035F048FDF7EE007A9FED197AF0EE675AFC
:10ADD000E8EE875A0023A361B0EE676AC7EEA56A62
:10ADE00063612362E361A3626362A8EEC76ABDEC9C
:10ADF000028B77EEC07AB6EE007AF8EE005A27EEB4
:10AE0000877A20EE250A27EE267A26EE266A67EE56
:10AE1000A67A20EE260A84ED046AC4ED017A84ED58
:10AE2000007A84ED027A84ED030A10BD27D4D2366D
:10AE3000F304353F10B44C09012250F8243001F0DE
:10AE40001F0102FA01F10B4340F824305DF8044B76
:10AE5000704700BF4B0901F01F0150F82320012368
:10AE600003FA01F1114214BF18460020704700BFD9
:10AE70002DE9F84FDFF8B480DFF8B4A0DFF8B49024
:10AE8000274E0123102088F8003033F02DFEDAF829
:10AE90000000FEF757FE052033F0D4FD002033F00C
:10AEA000D1FD062033F0CEFD002033F0CBFD99F824
:10AEB0000040042044F0010433F0C4FD204633F088
:10AEC000C1FD33888BB1174D174F002415F804B01E
:10AED000072033F0B7FD584633F0B4FD2A5D3388C0
:10AEE0003A550134A4B2A342F0D8072033F0AAFDAA
:10AEF000FF2033F0A7FD99F80040042033F0A2FDB5
:10AF0000204633F09FFDDAF80000FEF721FE042012
:10AF100033F0EAFD002388F80030BDE8F88F00BF69
:10AF200048020020D8470020204D0020094D002075
:10AF30007C990020114D00202DE9F0414A4E10204F
:10AF400033F0D2FD3068FEF7FDFD484B1B78012B36
:10AF50007BD062D3022B0AD1DFF83081082388F836
:10AF600000300D254FF4C373414F3B8010E0DFF8F4
:10AF70001C813F4F98F8003003F04003002B14BFB2
:10AF80004FF4F0734FF4C3733B8014BF10250D25AD
:10AF9000002404F11000C0B233F054FD013401204C
:10AFA00033F050FDA3B2AB42F3D398F80040314DDB
:10AFB000002033F047FD204633F044FD2E4B1C7833
:10AFC000022033F03FFD204633F03CFD2B4B1C7834
:10AFD000032033F037FD204633F034FD284B1C7836
:10AFE0000420044333F02EFD204633F02BFD30685F
:10AFF000FEF7AEFD042033F077FD3A8821480021AA
:10B0000037F087FD2B7B33B11F4B1B7833B3002305
:10B010002B73BDE8F081BDE8F081A02033F012FD74
:10B02000002033F00FFD00F00603022BDFF85C80F8
:10B0300007D000F00500012803D1482388F800302C
:10B0400008E0082388F800308BE7DFF840804823C9
:10B0500088F8003010254FF4F07385E7FFF708FFFC
:10B0600000232B73BDE8F0817C990020809900209B
:10B0700048020020000000208799002088990020C5
:10B08000114D0020204D0020094D002050020020CD
:10B09000F8B50B4C074620680E461546FEF752FDE4
:10B0A00047F0800033F0CEFC3346294600220548A5
:10B0B000FDF744F92068FEF74BFD0120F8BD00BF05
:10B0C000C8860020003C004070B582B06A46062168
:10B0D000F720FFF7DDFF9DF801209DF804309DF873
:10B0E00000609DF803509DF802409DF80500074957
:10B0F00012011B0142EA063243EA053342EA141206
:10B1000043EA10134A600B6002B070BD7424002043
:10B110000C4B984213D0A3F5806398420FD003F5EF
:10B12000804398420BD003F58063984207D003F523
:10B130008063984203D0044B186840087047024B64
:10B140001868704700040140E06F0020F0B5774BAD
:10B15000774A87B01968914200AF00F0DB80002386
:10B16000744A3B607B60136843F48033136003E0F0
:10B170003B68B3F5A04F09D0136803F400337B603C
:10B180003B6801333B607B68002BF1D0694B1B6847
:10B1900013F4003318BF01237B607B68012B7BD045
:10B1A000654D644B654AEA606549586F654A0860B9
:10B1B000AA605E6B644C654A654826F080065E6353
:10B1C0005E6F46F080765E67196B0C431C63596BAB
:10B1D0005963996B9963196C41F05B5141F47B1190
:10B1E00041F41F6141F00F011964596C07F1180413
:10B1F0000A4348F2FF715A6444F8101D00262146A4
:10B200000123FB733E737E73BE732AF059FD214602
:10B210004FF6FF734F48BB602AF052FD4FF6FF73A5
:10B2200021464D48BB602AF04BFD21464B482AF091
:10B2300047FD21464A482AF043FD214649482AF065
:10B240003FFD214648482AF03BFD214647482AF069
:10B2500037FD214646482AF033FD20462AF03AFEC3
:10B26000444B454C1B68BA6844484549A4FB03431A
:10B270009B09A0FB0202013B920CB3F1807F0A60A4
:10B2800007D2404AF0200721536085F823009660DA
:10B2900011601C37BD46F0BD264B3B4C1A6C3B4938
:10B2A00042F080521A6420684A690D69896940F445
:10B2B00040402060986898609868120640F400400A
:10B2C000986042EA8512986842F48002490842F088
:10B2D0000802013942EA014240F4A05098605A60E5
:10B2E0001A6842F080721A601A689201FCD52849E7
:10B2F000104A40F205700860996821F003019960D6
:10B30000996841F002019960936803F00C03082BDF
:10B31000FAD145E700221A6062B61E4B1B6883F320
:10B3200008881D4B1B689847FEE700BFFCFF012003
:10B33000EFBEADDE0038024000ED00E00005FA058A
:10B3400054AA002000000008FF916700335F070047
:10B35000000002400004024000080240000C0240CD
:10B36000001002400014024000180240001C02407D
:10B3700000200240E06F0020D34D621083DE1B43AB
:10B3800054D4002010E000E00070004000000020D5
:10B39000003C02400000FF1F0400FF1F08B5054BE2
:10B3A0001B6803B19847044B044A1A6072B6FDF754
:10B3B00017FC00BF60690020FCFF0120EFBEADDE7E
:10B3C00008B5034B1B6803B1984772B6FDF708FC3C
:10B3D00060690020084B10B507281B68C8BF1438E7
:10B3E00018440C46007EFEF785F820B12146BDE8E2
:10B3F0001040FEF7B3BB10BDA086002030B5044658
:10B40000806D61718389A26823F400531B041B0CB7
:10B41000838185B0A379009213F0040230D04FF4F9
:10B42000805213F00203ADF8042056D1ADF8063077
:10B430004FF480630022ADF8083011F00103ADF83D
:10B440000C2028D1ADF80A3008238D07694648BF83
:10B45000ADF80A302AF088FDA279A36DD10724D473
:10B4600012F0080F9A8A1BD122F008021204120C63
:10B470009A829A8992B242F400529A8105B030BD04
:10B4800013F00203ADF8042024D04FF40055134606
:10B49000ADF80650CEE70423ADF80A300C23D4E70C
:10B4A00092B242F008029A82E3E70D498B420FD034
:10B4B000A1F548418B4209D00A498B42D0D10520E1
:10B4C0000121FFF787FFA279A36DC9E70220F7E703
:10B4D0000020F5E7ADF80630ACE74FF40053A5E7E0
:10B4E000001001400014014010B50446806DA160B9
:10B4F000838923F400531B041B0C8381A37984B03C
:10B5000013F00402009135D04FF4805213F002037F
:10B51000ADF8042056D1ADF806304FF4806362795F
:10B52000ADF80830D1074FF00003ADF80A30ADF8A0
:10B530000C3045BF0423ADF80A3008230C236946BC
:10B54000920748BFADF80A302AF00EFDA279A36D2C
:10B55000D1071FD412F0080F9A8A16D122F00802E0
:10B560001204120C9A829A8992B242F400529A8181
:10B5700004B010BD13F00203ADF804201FD04FF447
:10B5800000511346ADF80610C9E792B242F0080226
:10B590009A82E8E70D498B420FD0A1F548418B42D2
:10B5A00009D00B498B42D5D105200121FFF712FFAD
:10B5B000A279A36DCEE70220F7E70020F5E7ADF80A
:10B5C0000630ACE74FF40053A5E700BF0010014080
:10B5D0000014014038B50D4B07281B68CCBFA0F103
:10B5E0001404044623440546187EFDF783FF58B132
:10B5F00001342722C47182710121FEF70DF928461A
:10B600000021BDE83840E5E638BD00BFA086002037
:10B61000064A00235168814202F11C0204D0013322
:10B62000102BF7D100207047D8B27047740000206B
:10B6300070B50F4C0F4DC0EBC00004EB8004286BBD
:10B6400026693043286382B09209667BA160002599
:10B65000012101A863618DF804608DF805208DF843
:10B6600006508DF8071033F0F5F802B070BD00BF3A
:10B670007400002000380240074BC0EBC00030B41B
:10B6800003EB8000054C0569236B2B432363017694
:10B69000427630BC704700BF740000200038024082
:10B6A0002DE9F04F534C54F8204083B0002C00F0AB
:10B6B0009C80E56D002D00F09A8017464E4A984612
:10B6C000064604F162032869226004F26222636183
:10B6D000A2614FF400736A68A160E3602361A26510
:10B6E000A24668B1FFF794FF721CD2B20C21FFF79B
:10B6F000C3FFA36DA9682A6922630433A16363654C
:10B70000E868A0B1FFF784FF721C8146D2B20B211A
:10B71000FFF7B2FF2346EA7F38494846FFF788FF24
:10B72000A36DA968EA6862630433E163236594F852
:10B730006100FDF7DFFE814694F86000FDF7DAFE58
:10B740008346287F00284DD118F0080F36D1BA075C
:10B750000DD5B9F1000F0AD00B22731C89F8062011
:10B7600089F8073048466A7F2221FDF789FFFB07E9
:10B7700015D4A36B7BB995F82020A97F8DF80630EE
:10B7800001A8930901228DF805308DF804108DF879
:10B79000072033F05FF8504603B0BDE8F08FBBF1EF
:10B7A000000FE6D001360C238BF807608BF80630CB
:10B7B00058466A7F2221FDF763FFDAE70136F6B2C9
:10B7C000B9F1000F04D00B2389F8076089F806301F
:10B7D00018F0100F484614BF022112216A7FFDF7AE
:10B7E0004FFFC6E733F058F8AEE7A246D3E7AA46C4
:10B7F000D1E700BF04380020C42C0408058C0008E1
:10B800000348D0F8AC3113B100F5D2701847704737
:10B81000740000200348D0F8903113B100F5C470D3
:10B8200018477047740000200348D0F8743113B1F2
:10B8300000F5B67018477047740000200348D0F830
:10B84000583113B100F5A8701847704774000020F4
:10B850000348D0F83C3113B100F59A70184770478F
:10B86000740000200348D0F8203113B100F58C702B
:10B8700018477047740000200348D0F804310BB11A
:10B88000FC301847704700BF740000200348D0F810
:10B89000E8300BB1E0301847704700BF740000205B
:10B8A0000348D0F8CC300BB1C4301847704700BF04
:10B8B000740000200348D0F8B0300BB1A83018470E
:10B8C000704700BF740000200348D0F894300BB1DB
:10B8D0008C301847704700BF740000200248836F07
:10B8E0000BB1703018477047740000200248C36DD8
:10B8F0000BB1543018477047740000200248036CA5
:10B900000BB1383018477047740000200248436A72
:10B910000BB11C3018477047740000200248836840
:10B9200003B11847704700BF74000020431C00F0AB
:10B9300019812DE9F04F4FEAC00B0BEB00039B0080
:10B94000DFF8908258F803A087B008EB0304BAF13F
:10B95000000F00F00481143308EB03010022DAF831
:10B96000047048F803204A608A60CA60A568D4F869
:10B970000C90431CDBB215B11522EB71AA71B9F121
:10B98000000F04D0162289F8073089F806200190AC
:10B990009AF80E0032F080FFBB8823F440731B043A
:10B9A0001B0CBB802846FEF7D3F84846FEF7D0F8BC
:10B9B00011212846FDF730FF11214846FDF72CFFE5
:10B9C0000826642404E00A203CB104F0EBFD013CAD
:10B9D0002846FEF7E5F80028F5D02846FEF7B2F82D
:10B9E0000A2004F0DFFD2846FEF7B2F80A2004F032
:10B9F000D9FD013EECD14846FEF7A4F80A2004F038
:10BA0000D1FD2846FEF79EF80A2004F0CBFD28461B
:10BA1000FEF79EF80A2004F0C5FD4846FEF798F8A8
:10BA2000019B0BEB030408EB84042846637C002B8A
:10BA30000CBF122132210422FDF722FE637C002B71
:10BA40000CBF1221322148460422FDF719FE584B43
:10BA50009F4200F09880574B9F4200F09E80564BCB
:10BA60009F4200F08680BB880199544A544C23F4CD
:10BA700040731B041B0CBB803B888B4408EB8B087A
:10BA80009BB243F0010398F810103B80BD8802A8D8
:10BA9000002918BF14462AF01DFA049A4948B2FB3F
:10BAA000F4F325F03F05A0FB02122D04900C2D0CA1
:10BAB0000543BD80444C39884FF4967202FB00F276
:10BAC00084FB02409BB2D217002BC2EBA01221F0E4
:10BAD000010108BF01230904013243F40043090CAA
:10BAE00092B239803A84BB833B889BB243F0010316
:10BAF0003B803B8823F4816323F002031B041B0C6F
:10BB00004FF4804243F480633B803A813B8823F0CA
:10BB100080031B041B0C3B809AF810308DF8083012
:10BB2000002402A801258DF809408DF80A408DF8FF
:10BB30000B5032F08FFE9DF80B209AF80F308DF8E5
:10BB400008308DF809408DF80A4062B95A09203250
:10BB500003F01F031D4905FA03F341F8223007B033
:10BB6000BDE8F08F704702A832F074FE07B0BDE860
:10BB7000F08F174A136A43F4000313624FF4000076
:10BB80002AF0F2F86FE7124A136A43F400131362C3
:10BB90004FF400102AF0E8F865E70D4A136A43F401
:10BBA000800313624FF480002AF0DEF85BE700BFE9
:10BBB0000054004000580040005C0040009F2400FA
:10BBC000804F120083DE1B43D34D621000E100E082
:10BBD0000038024020D20020F0B5C60033189B0088
:10BBE000254DEA585468A28A83B092B20192019A14
:10BBF0002B4412F4706F1CBF01221A75019B13F4C1
:10BC0000E06F07460CD1A38A3E4423F4706305EB32
:10BC100086051B041B0C0022A3826A7503B0F0BDCD
:10BC2000238BA38823F480631B041B0CA380019B3C
:10BC30009B05E8D423889805E5D42388D9050ED53B
:10BC40002388DA05FCD423889BB243F40073238055
:10BC500023889B05FCD43846FFF768FED3E723888A
:10BC60009BB243F400732380A38823F440731B0426
:10BC70001B0CA380C7E700BF20D20020F0B583B023
:10BC8000441C8DF8073001D0032802DD002003B0EA
:10BC9000F0BDC700244E3B1806EB83035D68002D02
:10BCA000F4D04900C9B2997501240021DA755C7697
:10BCB00099761C765C751975A9880DF107028905BE
:10BCC000DA611A6214D42B88DA050CD44FF480544C
:10BCD00001E0013C1ED02B889B05FAD42B889BB237
:10BCE00043F480732B80AB889BB243F44073AB80EA
:10BCF000074406EB87024FF4805401E0013C09D071
:10BD0000537D002BFAD106EB87073C7D84F00100C0
:10BD100003B0F0BD054A138801339BB21380FFF7CF
:10BD200005FE2046B3E700BF20D200208CD20020C1
:10BD30002DE9F043322083B004F08EFC1123002261
:10BD40001E210120FFF79AFF0122104660231E21C9
:10BD5000FFF794FF642004F07FFC6846FDF7C4FA07
:10BD60000024DFF85481254626460A270123184679
:10BD700002221E21FFF782FF322004F06DFC68468C
:10BD8000FDF7B2FABDF900E0BDF90210BDF90420DB
:10BD90008E457346A8BF0B469342A8BF1346434542
:10BDA0004FF0010076440D44144479DBFDF792FB1B
:10BDB000013FDBD14FF00109122300221E21012097
:10BDC000FFF75CFFDFF8F0800A2701231846022204
:10BDD0001E21FFF753FF322004F03EFC6846FDF7BA
:10BDE00083FABDF900E0BDF90210BDF904208E45CB
:10BDF0007346A8BF0B469342A8BF134643454FF076
:10BE00000100A6EB0E06A5EB0105A4EB02044ADB3C
:10BE1000FDF760FB013FD8D107EE906AF8EEE76AC4
:10BE200007EE905AB8EEE77A07EE904ADFED1F5A18
:10BE30009FED1F5A1F4EF8EEE77A85EEA66A702333
:10BE400000221E210120C5EE876A85EE277AB0EE1A
:10BE5000C66AF0EEE66AF0EEC77A86ED006AC6EDD5
:10BE6000016AC6ED027AFFF709FF0122104620237E
:10BE70001E21FFF703FF002302221E210120FFF7EE
:10BE8000FDFE642004F0E8FBB9F1000F04D14FF08F
:10BE90007E5333607360B360012003B0BDE8F0836C
:10BEA0004FF0000988E74FF00009B5E700406F4602
:10BEB00001C05E460000002001F0FFFF012318468C
:10BEC00048227721DAE600BF01231846582277215D
:10BED000D4E600BF134601200A466821CEE600BF23
:10BEE0000220FCF77DBF00BF022075E60120FCF7B1
:10BEF00077BF00BF01206FE60020FCF771BF00BFD5
:10BF0000002069E61549164B16480A6910B48C6979
:10BF10001549B2FBF4F203FB02F30360D1F8882069
:10BF2000124B134C42F47002C1F888201A680020AA
:10BF300042F001021A6098601A6822F0847222F4BA
:10BF400080321A605C601A684FF0006422F480222C
:10BF50001A60D8608C605DF8044B704700000020C8
:10BF600040420F00E06F002000ED00E0003802408A
:10BF700010300024044B4FF4F07002210A221861A3
:10BF800099615A61FFF7BEBF000000202DE9F04F14
:10BF900005462DED048BB0F9080008815FFA80F8A2
:10BFA00097B040460C46914602F0B8FC40B10123E0
:10BFB0001A461846628117B0BDEC048BBDE8F08FBD
:10BFC000A8F10A03E72B00F2EA80DFE813F0250668
:10BFD000E800E800E800E800E800E800E800E80021
:10BFE000E800E800E800E800E800E800E800E80011
:10BFF000E800E800E800E800E800E800E8003706AC
:10C00000E800E800E8006806E800E800E8007906D3
:10C01000E8007E06E800E906E8000207E8000E07EF
:10C02000E8001307E8003907E800E800E8008D01A0
:10C030009401E8009C01E800E800A501E800E800A0
:10C04000E800E800E8008001E800E800E800E80017
:10C05000AD01E800C801E800E9010F02E800E800CE
:10C06000E800E800E800E800E8001903E800EF0253
:10C07000E8005C03E8003F02E8008802E800E8000E
:10C08000E800E8009802BD028A039203E303F50387
:10C090001B0431044A04E80058049104E800E80055
:10C0A000E800E800AE04E800E800BA04E800E800B0
:10C0B000E800DC04ED0406053F05E800E800E800C0
:10C0C0007E058F05A305E800E800E800E800E80029
:10C0D000E800E800E800E800E800E800E800E80020
:10C0E000E800E800E8009802E800E800E800E8005E
:10C0F000E800E800E800E800E800E800E800E80000
:10C10000E800B405E800E800E800E800E800E8001E
:10C11000E800E800E800E800E800E800E800E800DF
:10C12000E800E800E800E800E800E800E800E800CF
:10C13000E800E800E800E800E800E800E800E800BF
:10C14000E800E800E800E800E800E800E800E800AF
:10C15000E800E800E800E800E800E800E800E8009F
:10C16000E800E800E800E800E800E800E800E8008F
:10C17000E800E800E800E800E800E800E800E8007F
:10C18000E800E800E800E800E800E800E800E8006F
:10C19000E800E800E800E800E800ED05FA05B8F17D
:10C1A000740F58D0B8F1770F0DD12B686A689A4296
:10C1B0001EBF5A1C2A601978984A08BF00212046E1
:10C1C00002F042FFF3E6B8F1F50F01F07087B8F125
:10C1D000760F4ED095E88400A8F12103BF1A362BC4
:10C1E00000F25C87DFE813F060065A075A075A0727
:10C1F0005A075A075A075A074A065A075A075A0748
:10C200005A075A075A075A075A075A075A075A0726
:10C210005A075A075A075A073F065A075A075A0732
:10C220005A075A075A075A075A075A075A075A0706
:10C230005A075A075A075A075A075A075A075A07F6
:10C240005A075A075A075A075A075A07A3065A079E
:10C2500081065A07D7062B686A689A421EBF5A1C85
:10C260002A6019786E4A08BF0021204602F0ECFED1
:10C270009DE62B685A1C2A601B78002B01F0A787CB
:10C28000102B07BF674A92E8220000252946226842
:10C29000501C206013702046FEF722FA29462046E3
:10C2A000FEF71EFA604B20461968FEF719FA0021C6
:10C2B0002046FEF72DFA00212046FEF729FA2168D4
:10C2C00000204A1C012322601A46087071E6236888
:10C2D00000255A1C2260294620461D70FEF700FAF0
:10C2E00029462046FEF7FCF900212046FEF7F8F922
:10C2F00001231A465DE6216801200A1822600346E0
:10C300000246087055E62268484B501C9978206018
:10C31000117021685878D4E7082245492046FEF775
:10C32000AFF901231A4644E62368424D591C2A7886
:10C3300021601A7023686A78591C21601A70698814
:10C340002046FEF7E5F923682A79591C21601A7006
:10C35000E9882046FEF7DCF92168287AB1E7364EF5
:10C360003378002B3FF423AE344D0027A8462368D2
:10C3700015F81720591C21601A7098F8011001EB6C
:10C38000810101EB810101F2EE2189B22046FEF725
:10C39000BFF9337801379F4208F10208E7DB06E670
:10C3A0002368274D01269A1922601E7026F044F852
:10C3B000002841F05587234B2268511C21601070E2
:10C3C000226841F2B410511C185C216041F27811CE
:10C3D000107059582046890AFEF782F9E96B204609
:10C3E0004908FEF77DF901231A46E2E52168164A5D
:10C3F0000123481C20600B7021689078CD182560BF
:10C40000087021681078CD18256008702168507870
:10C41000CA1822601A460870CBE500BF69E500081B
:10C4200031E8000894250020E8280020E845002095
:10C4300078740020FC410020908500208079002045
:10C44000A0C7002018B3002078D10020002120468A
:10C45000FEF75EF900212046FEF75AF9002120463A
:10C46000FEF756F92268B74D0023511C2160137066
:10C4700022682968501C91F82F10206011702268E2
:10C480002968501C91F83A102060117022682968C0
:10C49000501C91F83B10206011702268511C2160E3
:10C4A00013702268511C216013702268511C216096
:10C4B00013702B682046D98FFEF72AF92B68204687
:10C4C000998FFEF725F923682A68591C92F83120C4
:10C4D00021601A702B68216893F83200F1E6236816
:10C4E000994A9A49D0789A4A5D1C25601870236849
:10C4F0000978581C206019702168D078E1E60DF1A8
:10C50000180900250695DFF880A2924B0495059541
:10C51000C9F8045001214FF6FF7B05E001350B2DD2
:10C5200001F02E851AF9011F4E1CF7D04BFA05F2C7
:10C53000D007F3D51A882A41D207EFD54846019390
:10C54000FEF778FC019BE9E7834E338AB3F5007F61
:10C5500006F1340594BF01270427403655F8041B23
:10C5600091FBF7F1204689B2FEF7D2F8B542F5D13A
:10C570007A4D7B4F05F10C06B5EC010AD7ED087A30
:10C5800080EE270A34F0B8F981B22046FEF7C0F8F1
:10C59000B542F1D1734D05F10C0655F8041B204648
:10C5A00089B2FEF7B5F8AE42F7D100E56E4EF378EA
:10C5B000002B01F0FF8523680822591C21601A70A6
:10C5C00023680122991821601A702368674D591C4D
:10C5D0002A7921601A702368AA78591C21601A7080
:10C5E00029882046FEF794F8698A2046FEF790F8DD
:10C5F0002368F279591C21601A702168E87860E696
:10C600002BF09EFEFF28064601F0338616A9002572
:10C6100001F84A5D0DF10D008DF80D502BF070FE04
:10C6200016A800F8495D2BF05FFE16A800F8485DDB
:10C630002BF04EFE16A820F8405D2BF03DFE23683F
:10C640005A1C22601E7023689DF80D20591C216021
:10C650001A7023689DF80E20591C21601A702368F7
:10C660009DF80F20591C21601A7023689DF8102036
:10C67000591C21601A70BDF818102046FEF748F8C2
:10C6800001231A4695E4384D23686A792D4E591CCA
:10C6900021601A7033682046198CFEF739F8336828
:10C6A0002046598CFEF734F869892046FEF730F8A9
:10C6B000A9892046FEF72CF833682046998CFEF7AE
:10C6C00027F833682046D98CFEF722F8E9892046FE
:10C6D000FEF71EF8298A2046FEF71AF801231A46AB
:10C6E00067E4102222492046FDF7CAFF01231A46BB
:10C6F0005FE4204D204EDFF89480DFF89490DFED6A
:10C700001F8ADFED1F9A9FED1F9A05F1200708E0B1
:10C7100020460435FDF7FCFFBD4206F118063FF444
:10C7200046AC717C0029F3D095ED008AB0EE480A42
:10C7300034F0E2F898F80030002B41F04D8581B2DA
:10C74000E6E700BFE8830020DC440020D445002059
:10C75000DC450020E48300209C83002054690020F5
:10C760002C6100205085002018610020E46F00201B
:10C770003046002040460020F06D0020000040427E
:10C780000040744400E082441C2D04080C7000201A
:10C7900058AA0020994E3378002B3FF408AC984FEC
:10C7A000002537F8021F2046FDF7B2FF3378013528
:10C7B0009D42F6DBFFF7FBBB924B22681B78924D44
:10C7C000511C03F002032160137023682A78591C5E
:10C7D00021601A7069682046FDF782FFA96820462B
:10C7E000FDF77EFFA9892046FDF792FF698A204662
:10C7F000FDF78EFFA98A2046FDF78AFF01231A461E
:10C80000FFF7D7BB814B20461988FDF781FF804B8E
:10C8100020461988FDF77CFF7E4B20681978421C62
:10C8200001F00101012322601A460170FFF7C1BB2C
:10C83000794D20462988FDF76BFF69882046FDF772
:10C8400067FFB5F904307549DA1781FB0313C2EBB2
:10C85000A30399B22046FDF75BFF01231A46FFF7B9
:10C86000A8BB6F4B20461968FDF73AFF6D4B204679
:10C870001988FDF74DFF01231A46FFF79ABB6A4D51
:10C8800023682A68591C127821601A702B68226864
:10C890009978531C2360002311702A6821681A4478
:10C8A00001335279481C032B20600A70F5D12368AC
:10C8B0002A68591C127A21601A7023682A68591C48
:10C8C000D27821601A7023682A68591C1279216075
:10C8D0001A702B6820465989FDF71AFF23682A68C9
:10C8E000591C527A21601A702B6821685878E8E444
:10C8F0004E4E00232268306803EB4301551C405C18
:10C9000025601070326820680A44451C5278256002
:10C910000270326820680A4401339278411C0A2B65
:10C9200021600270E6D1FFF742BB414952232268E1
:10C93000501C2060137011F8013F002BF7D1FFF756
:10C9400036BB3C4D05F16006A9882046FDF7E0FEA8
:10C95000E9882046FDF7DCFE29892046FDF7D8FE50
:10C960002368AA7A591C21601A702368EA7A591C34
:10C9700021601A7055F80C1B2046FDF7B1FEAE423F
:10C98000E2D1FFF714BB2C4D20462988FDF7C0FEED
:10C9900069882046FDF7BCFEA9882046FDF7B8FE51
:10C9A00001231A46FFF705BB2268244B2249187859
:10C9B000551C2560107022685878551C2560107031
:10C9C00022689B78501C20601370C9882046FDF7B0
:10C9D0009FFE01231A46FFF7ECBA2368184A19494B
:10C9E0001078194A5D1C2560187023688978581CD6
:10C9F000206019702168907863E400BF9085002062
:10CA000052C9002065830020688300209CD100204B
:10CA10000E7B0020004A0020948300206766666633
:10CA20008C83002090830020EC830020E88300208A
:10CA3000EC2C040828D00020E4410020CC45002044
:10CA400018610020DC440020DC450020DFF848E3CA
:10CA50000027FEB2714600232268501C2060167029
:10CA60002268501C20601370226811F8010F0133F6
:10CA7000551C062B25601070EED10137062F0EF1E4
:10CA8000060EE6D1B14900232268501C20601770C1
:10CA90002268501C20601370226811F8010F0133C6
:10CAA000551C0B2B25601070EED12368A84A581C2A
:10CAB00007212060197023680021581C206019701C
:10CAC000216892F8F000FFF7FCBBA24D2046A98A2E
:10CAD000FDF71EFEE98A2046FDF71AFE298B204647
:10CAE000FDF716FE01231A46FFF763BA22689A4B38
:10CAF000501C19782060117022685978501C2060F1
:10CB0000117022689978501C206011702168D878C3
:10CB1000FFF7D7BB914B9249B3F9003081FB03215A
:10CB2000DB17C3EBA10189B22046FDF7F1FD01231C
:10CB30001A46FFF73EBA2368DFF860C2591C9CF81A
:10CB4000002021601A709CF80030002B3FF42FAABF
:10CB5000844E854D854886490022236816F8017F5A
:10CB600003F1010EC4F800E01F70236815F8017F7F
:10CB700003F1010EC4F800E01F70236810F8017F74
:10CB800003F1010EC4F800E01F70236811F8017F63
:10CB900003F1010EC4F800E01F709CF80030013270
:10CBA0009A42DADBFFF703BA724D2046A989FDF7F6
:10CBB000AFFD69892046FDF7ABFD01231A46FFF75B
:10CBC000F8B96D4B03F1700522681978501C20608C
:10CBD000117022685978501C206011702268997871
:10CBE000501C206011702268D978501C2060117090
:10CBF00022681979501C2060117022685979501CE4
:10CC000020601170226899790733501CAB42206074
:10CC10001170D9D1FFF7CBB9584832F001FD002887
:10CC20007FF7C5A9554B1D18226813F8011B501C2E
:10CC3000AB4220601170F7D1FFF7B9B9504D514F99
:10CC400005F15006002128784F4A0B4607E00133D2
:10CC5000242B02F10C0201F0728112F80C1C8842A4
:10CC6000F5D103EB4303226807EB8303511C93F8D0
:10CC700044302160137023686A78591C21601A704F
:10CC80002368AA78591C21601A702368EA78043551
:10CC9000591CAE4221601A70D4D1FFF788B93B4DC0
:10CCA00020462988FDF734FDA9882046FDF730FD90
:10CCB00029892046FDF72CFD01231A46FFF779B993
:10CCC000334B21681878FFF7FCBA324D23682A7A73
:10CCD000591C21601A70A98B2046FDF719FD298B7C
:10CCE0002046FDF715FD698B2046FDF711FD2368F1
:10CCF000EA7C591C21601A70E98C2046FDF708FD7A
:10CD0000298D2046FDF704FD2368AA7F591C216068
:10CD10001A70236895F82020591C21601A70A98C7C
:10CD20002046FDF7F5FC2368EA7A591C21601A7049
:10CD3000E9682046FDF7D4FC23682A7C591C216051
:10CD40001A70216895F82100FFF7BBBA8F7A00208E
:10CD5000AC790020E46F0020184B0020DC45002057
:10CD600067666666334B0020434B0020634B002010
:10CD7000534B0020DC44002068CE0020157B0020AF
:10CD80007C460020EC2C0408342D040834380020A4
:10CD900078460020787400206B7A0020314B002008
:10CDA000AF4D05F14006B5F880102046FDF7B0FC08
:10CDB000236895F88220591C21601A70236895F821
:10CDC00083200435591CB54221601A70EBD1FFF75E
:10CDD000EEB8A44D05F1800655F8041F2046FDF776
:10CDE0007FFCB542F8D1FFF7E2B89F4B2168587D30
:10CDF000FFF767BA9D4B03F15A0522685979501C19
:10CE00002060117022681978501C2060117022680F
:10CE10005978501C2060117022689978501C20604D
:10CE200011702268D978501C20601170226819791D
:10CE30000633501CAB4220601170DED1FFF7B7B84B
:10CE40008B4D8C4E05F1300795F902100023F256F8
:10CE50008A4201F077800C33482BF8D10835AF4275
:10CE6000F2D1FFF7A4B8531C2B6013780A2B01F002
:10CE70008E824FF0FF331A46FFF79BB8531C2B608E
:10CE800013780A2B01F00D82502BF2D12846FDF7C2
:10CE9000EBFB794E30802846FDF7E6FB4FF0FF3381
:10CEA00070801A46FFF785B81346511C2960734EEF
:10CEB00013F8021B71702B6053783370D31C2B60F6
:10CEC0009378B3702846FDF7CFFB2B68F0801A46A5
:10CED000591C296012F8021B31712A605B7873714A
:10CEE0004FF0FF331A46FFF764B8531C2B601678D7
:10CEF000FF2E01F00783FE2E01F0E0812846FDF7AA
:10CF0000B3FB2B686A68D21A002A06DD5A1C2A6015
:10CF10001B7813B90B2E41F21783242EA9D8584A37
:10CF20004FF0FF3322F816001A46FFF742B8531CA1
:10CF30002B6010787A1E0328D2B29AD8411EC9B24B
:10CF4000504E514B01EB410106EB410118704978FD
:10CF500000288ED08A428CD10021C3F80610C3F875
:10CF6000021099725AB1013229681A440133013111
:10CF7000296011F8010C03F8010F9342F7D1434BDC
:10CF80001B78002B3FF475AF2CF03AFD4FF0FF33C8
:10CF90001A46FFF70EB8531C2B6012F8377B0DF1C1
:10CFA000170101332B6013F8010C01F8010F9A42AD
:10CFB000F7D1DFF8E09099F80050002DFDD1DFF8AF
:10CFC000D8A00126102089F8006031F08DFDDAF834
:10CFD0000000FCF7B7FD2E4B28461E7031F032FDE5
:10CFE000284631F02FFD092031F02CFD384631F074
:10CFF00029FD06AF3D460DF14E08EE1BF6B20A20A4
:10D0000031F020FD304631F01DFD15F8016B0B208D
:10D0100031F018FD304631F015FD0020FCF75AFACA
:10D02000A845EAD1082031F00DFDA02031F00AFD1D
:10D03000A02031F007FD002031F004FD10F02005A4
:10D04000F6D1DAF80000FCF783FD042031F04CFD46
:10D050004FF0FF3389F800501A46FEF7AABF00BF11
:10D06000AC790020A879002078740020EC3A0020E8
:10D0700090990020CCB20020CC2900208083002091
:10D0800010D10020E8320408048E0020742900200A
:10D09000124D0020094D00207C990020A8F10B00C2
:10D0A000EF283FF6E6AE01A353F820F03FDA000880
:10D0B00073CE000873CE000873CE000873CE00084C
:10D0C00073CE000873CE000873CE000873CE00083C
:10D0D00073CE000873CE000873CE000873CE00082C
:10D0E00073CE000873CE000873CE000873CE00081C
:10D0F00073CE000873CE000873CE000873CE00080C
:10D1000073CE000873CE000873CE0008DBD9000888
:10D1100073CE0008C1D9000873CE00089FD900085B
:10D1200073CE000873CE000873CE00088DD90008B6
:10D1300073CE0008EDD8000873CE0008BBD80008F5
:10D1400073CE000895D8000873CE00083FDC0008B5
:10D1500073CE0008EBDB000873CE00089DDB0008EF
:10D1600073CE000873CE000873CE000873CE00089B
:10D17000AFBF000873CE000881DB000873CE000843
:10D1800073CE000867DB000873CE000873CE00087A
:10D1900073CE000873CE000873CE000873CE00086B
:10D1A00073CE000873CE000873CE000873CE00085B
:10D1B00027DB000873CE0008DDDA000873CE000814
:10D1C00073CE000873DA000873CE000873CE00082F
:10D1D00073CE000873CE000873CE000873CE00082B
:10D1E00073CE0008F9DD000873CE0008F7DC0008F4
:10D1F00073CE0008AFDC000873CE000851DC0008D5
:10D2000073CE000817DF000873CE000873CE000845
:10D2100073CE000873CE000873CE000873CE0008EA
:10D2200073CE000873CE000873CE000873CE0008DA
:10D2300073CE000873CE000873CE000873CE0008CA
:10D2400073CE000873CE000873CE000873CE0008BA
:10D2500073CE000873CE000873CE000873CE0008AA
:10D2600073CE000873CE000873CE000873CE00089A
:10D2700073CE000873CE000873CE000873CE00088A
:10D2800073CE000873CE000873CE000873CE00087A
:10D2900073CE000873CE000873CE000873CE00086A
:10D2A00073CE000873CE000873CE000873CE00085A
:10D2B00073CE000873CE000873CE000873CE00084A
:10D2C00073CE000873CE000873CE000873CE00083A
:10D2D00073CE000873CE000873CE000873CE00082A
:10D2E00073CE000873CE000873CE000873CE00081A
:10D2F00073CE000873CE000873CE000873CE00080A
:10D3000073CE000873CE000873CE000873CE0008F9
:10D3100073CE000873CE000873CE000873CE0008E9
:10D3200073CE000873CE000873CE000873CE0008D9
:10D3300073CE000873CE000873CE000873CE0008C9
:10D3400073CE000873CE000873CE000873CE0008B9
:10D3500073CE000873CE000873CE000873CE0008A9
:10D3600073CE000873CE000873CE000873CE000899
:10D3700073CE000873CE000873CE000873CE000889
:10D3800073CE000873CE000873CE000873CE000879
:10D3900073CE000873CE000873CE000873CE000869
:10D3A00067DD0008C5DE00085DD8000873CE000800
:10D3B000DBD70008C1D7000853D7000873CE000898
:10D3C00039D70008D3D60008ABD6000899D6000894
:10D3D0003BD6000873CE00080DD6000873CE0008B7
:10D3E00073CE0008EBD50008BDD50008A9D500080C
:10D3F00081D5000861D500083FD5000813D5000885
:10D40000FBD4000873CE000873CE000873CE00086A
:10D4100073CE000873CE000873CE000873CE0008E8
:10D4200073CE000873CE000873CE000873CE0008D8
:10D4300073CE000873CE000873CE0008E1D4000854
:10D4400073CE000873CE000887D4000873CE00089E
:10D4500073CE000873CE000873CE000873CE0008A8
:10D4600073CE000873CE00086DD40008C04B1B7843
:10D47000DB073FF5FEAC01F0B3FE02F065FD0123D2
:10D480001A46FEF796BD531C2B6013780F2B3FF600
:10D49000F0AC911C2960C3EBC303B6495078C85463
:10D4A000D01C28600B4491785970111D2960D178E7
:10D4B0009970511D29601179D970911D2960517998
:10D4C0001971D11D29609179597102F10801296002
:10D4D000D2799A7130F07CF801231A46FEF769BDC3
:10D4E0002846FDF7C1F8A44EB0812846FDF7BCF8E8
:10D4F000012370811A46FEF75CBD2846FDF7B4F89B
:10D500009E4900EB8000420001230A801A46FEF784
:10D5100050BD1146531C2B60994B11F8020B18702B
:10D52000296051785970D11C296091789970111D2A
:10D530002960D278DA7001231A46FEF73ABD2846F0
:10D54000FDF792F88F4EB0822846FDF78DF8F082F5
:10D550002846FDF789F8012330831A46FEF729BDD6
:10D560001346511C296013F8020B2B60D31C517811
:10D570002B60927823F0B4FC00287EF418AD78E498
:10D580001346511C2960804913F8020B08702B6068
:10D59000794953788B70D31C2B60784B92789A70B2
:10D5A00001231A46FEF705BD784B794918684A22CF
:10D5B00032F098FF01231A46FEF7FBBC1146531CBC
:10D5C0002B60744B11F8020B187029605178597058
:10D5D000D11C296092789A702846FDF745F86E4A6A
:10D5E0000123D0801A46FEF7E4BC2846FDF73CF83C
:10D5F000694E30802846FDF737F870802846FDF7E1
:10D6000033F80123B0801A46FEF7D3BCDFF8A881B7
:10D6100098F80030002B3EF4CAAC604F0026284634
:10D62000FDF722F812F032FE98F80030A7EC010A5C
:10D6300001369E42F3DBFEF7BABC0F2F7FF419AC24
:10D64000531C2B601678072E3FF613ACDFF86C8165
:10D6500028460C27FDF708F807FB06F708EB070636
:10D66000B0802846FDF700F8F0802846FCF7FCFF64
:10D670002B6830811A46591C296012F8021BB172BE
:10D680002A605B78F3722846FCF7D6FF012348F83E
:10D6900007001A46FEF78DBC2846FCF7E5FF404A16
:10D6A000012310801A46FEF784BC531C2B601078AF
:10D6B000060600F1FF862E4B1B78DD073EF577ACA2
:10D6C000032828BF002001F06FFD01231A46FEF752
:10D6D00070BC531C2B60284692F80090FCF7ACFFFE
:10D6E00080462846FCF7A8FF07462846FCF7A4FF1B
:10D6F00006462846FCF7B8FF2846FCF7B5FF2B681E
:10D7000001332B60B9F1000F00F0BF86B9F1100FA3
:10D710007EF44DAC234BC3F800805F600EB1224B0A
:10D720001E602249224B0222081F1A702AF0FAFCBE
:10D7300001231A46FEF73DBC0D4B1B78D8073EF57A
:10D7400036AC01F001FE02F0FFFB01231A46FEF7A2
:10D7500030BC074B1B78DA073EF529AC15490A782F
:10D76000012342F004020A701A46FEF722BC00BFF1
:10D77000CC81002068CE0020DC440020DC45002065
:10D78000184B0020E46F002018610020E88300207F
:10D79000CC340408CC450020E4410020EC400020BB
:10D7A000144B002094250020E82800209825002014
:10D7B000024A0020658300205E75002028D00020EA
:10D7C000B74B1B78D9073EF5F2ABB64A4FF4C87198
:10D7D000012311801A46FEF7ECBB092F7FF649ABF7
:10D7E000DFF8F4821346511CD8F80060296013F862
:10D7F000021B31702B605378B370D31C2B6093786D
:10D80000642B02F10401A8BF642373712960D378EB
:10D81000642B02F10501A8BF6423B3712960137959
:10D82000F371931D2B605379642B28BF6423D11DA2
:10D83000337229609379F37002F108032B60D37976
:10D8400033712846FCF710FF0A2F708140F00186E3
:10D850002EF03AF901231A46FEF7ABBB924B18683B
:10D86000D31C014621329E1E2E6013F8036C0E70ED
:10D870005E1E2E6013F8026C4E702B6013F8016C64
:10D880008E7003339A4201F10301ECD130F07AF843
:10D89000FEF78DBB531C2B6016781F2E3FF6E9AAAE
:10D8A000052F7FF4E6AA2846FCF7C6FE7F4B43F817
:10D8B00026001AF0ABFDFEF77ABB7C4E06F140075E
:10D8C0002846FCF7D1FE2B68A6F88000591C1A46A2
:10D8D000296012F8021B86F882102A605B7886F8AD
:10D8E00083300436B742EBD1FEF761BB531C704E58
:10D8F0002B60137833722846FCF7B6FEB0832846B7
:10D90000FCF7B2FE30832846FCF7AEFE2B6870832E
:10D910005A1C2A601B78F374082F7EF648AB284601
:10D92000FCF7A2FEF0842846FCF79EFE0C2F308503
:10D930007EF63DAB2B681A46591C296012F8021B73
:10D94000B1772A605B7886F820302846FCF78CFE99
:10D95000102FB0847EF62BAB2B685A1C2A601B78E4
:10D96000F3722846FCF768FE2B68F0605A1C2A60A8
:10D970001A783274162F7EF61AAB9A1C2A605B78DE
:10D9800086F8213001231A46FEF713BB531C2B6087
:10D99000484B12781A7001231A46FEF70ABB284634
:10D9A000FCF762FE444E30602846FCF75DFE706076
:10D9B0002846FCF759FE0123B0601A46FEF7F9BA73
:10D9C0003E4E002333602846FCF736FE32680123C2
:10D9D000024332601A46FEF7ECBA531C2B601078F3
:10D9E00013283FF646AA931C2B605678344B00212F
:10D9F00005E00131242903F10C033FF43AAA1F7A10
:10DA0000B742F6D12F4E304B0C2707FB0161D61CD5
:10DA100091F83C1003F820102E6003EB80039178FE
:10DA20005970111D2960D0789870501D28601E49CA
:10DA300012790868DA702DF0D5FFFEF7B8BA234BDB
:10DA4000102F4FF0000228BF10271A605A609A600A
:10DA5000DA601A74002F3EF4AAAA2A681744013229
:10DA60002A6012F8011C03F8011BBA42F7D1FEF735
:10DA70009EBA174B1B78012B3EF699AA1146531CF0
:10DA80002B60144B11F8020B9870296051781970B3
:10DA9000D11C296092785A7001231A46FEF789BA80
:10DAA000CC810020C2CA0020E8830020AC7900208D
:10DAB0007874002078460020343800201853002065
:10DAC000282D0408EC2C04087C460020157B00203F
:10DAD0001C53002078D10020EC830020531C2B60C5
:10DAE0001778112F3FF6C5A9931C2B60B44E5378BD
:10DAF00006F817302846FCF7B7FD40F6CA039842EF
:10DB0000A8BF184640F2EE23984206EB4706B8BF7E
:10DB100018460123A0F2EE211A46192091FBF0F1DC
:10DB20007170FEF746BA1346511C2960A54E13F8D2
:10DB3000021B31702B60537873702846FCF794FDFC
:10DB40002B6870805A1C2A601B7833712846FCF7BA
:10DB50008BFD2B68F0805A1C2A601B7833720123DE
:10DB60001A46FEF726BA984B02F1080101322A60E4
:10DB700012F8010C03F8010F9142F7D1FEF717BA22
:10DB80001346511C2960914913F8020B88702B60D1
:10DB900053784B7001231A46FEF70BBA0723B7FBE5
:10DBA000F3F3C3EBC301791A7FF463A9DBB203F18A
:10DBB000FF395FFA89F9002B3EF4F9A9DFF810A2CA
:10DBC00009F101098846531C2B6092F90020804B13
:10DBD000002693F90210914200F0AC830136062E24
:10DBE00003F10803F5D1FFF744B9531C2B601378F8
:10DBF0000E2B3FF63EA9911C29605678032E3FF666
:10DC000038A97448062101FB03F14318D71C5E7143
:10DC10002F6096784654111D2960D1785970511D96
:10DC2000296011799970911D29605179D970D11DA0
:10DC3000296092791A7101231A46FEF7BAB9531C6A
:10DC40002B60654B12785A7501231A46FEF7B1B95D
:10DC50002846FCF709FD2846FCF706FD2846FCF798
:10DC600003FD2B685D4E9A1CD6F800802A605A7816
:10DC700088F82F20DA1C2A609A7888F83A201A1D32
:10DC80002A60DA7888F83B2007332B602846FCF7B7
:10DC9000EBFCA8F83E002846D6F80080FCF7E4FC30
:10DCA000112FA8F83C0000F289833068EEE5531C80
:10DCB0002B604A4EDFF828811378D6F8009088F858
:10DCC00005302846FCF7D0FCA9F820002846D6F8F5
:10DCD0000090FCF7C9FC052FA9F8220000F27C8314
:10DCE00001F088FA1BF0E0FF306812F003F901231D
:10DCF0001A46FEF75EB91346511C2960384E13F8D8
:10DD0000021BB1702B60374953780B70D31C2B600A
:10DD1000354F93783B71131D2B60D378092BA8BF27
:10DD200009232846BB70FCF79FFC2B686A68388083
:10DD3000D11A012905DD2846FCF796FC2B686A6894
:10DD400078829A4240F0958301F054FA2B686A6811
:10DD50009A423EF42CA95A1C2A601B78FB700123BE
:10DD60001A46FEF726B9C7F34707122F3FF681A8D8
:10DD7000B7B116AB0DF1160803EB4706C146423E9C
:10DD80002846FCF771FC29F8020F4E45F8D1174BD5
:10DD900038F8022F23F8022FC845F9D1112F09D8DE
:10DDA000134A7B00023B13440021223223F8021F56
:10DDB0009A42FBD10F49012213460A70FEF7F9B8C7
:10DDC00080790020FC41002077740020E845002085
:10DDD00090990020EC3A002078740020E88300201D
:10DDE00018610020C8450020E46F00208E770020D5
:10DDF00090770020B47700202846FCF735FC0646D3
:10DE00002AF09EFAFF283EF4D2A8B6F57A7F80F079
:10DE100009830DF15809002309F8403DF7084946E8
:10DE200004A88DF8103001372AF06AFA9DF81030F6
:10DE3000FFB206F00706BB4206F1010603D19DF8CA
:10DE40001830B34203D0314638462AF065FA2B68C1
:10DE50006A68D21A012A7EF7AAA85A1C16A82A6054
:10DE600000221E7800F8482D2AF03EFA9DF8103066
:10DE7000B3420AD0BC4B1B683BB19A79B24204D37F
:10DE80001B681B690BB1304698472B685A1C2A60E7
:10DE9000484600221D788DF818202AF019FA9DF8BE
:10DEA0001830AB423EF483A8AF4B1B68002B3EF406
:10DEB0007EA81B685B69002B3EF479A8284698472A
:10DEC000FEF775B8531C2B601378A849002B00F09F
:10DED000D8820B7843F00203901C0B70A44E28608C
:10DEE000537833702846FCF7A7FB70602846FCF790
:10DEF000A3FBB0602846FCF7B7FBB0812846FCF7CF
:10DF0000B3FB9C4970820A78012342F002020A7036
:10DF10001A46FEF74EB81346511C2960964913F86D
:10DF2000020BC8702B60954953780B70D31C2B6083
:10DF3000934B9278DA7001231A46FEF73AB8002321
:10DF40001B7AFFDE23685A1C22601970298820463C
:10DF5000FCF7DEFB2368EA78591C21601A702368FD
:10DF60002A79591C21601A702368AA79591C2160EA
:10DF70001A7023686A79591C21601A70FEF76EBF07
:10DF8000DFF82CB200254FF0080A0135242D1AD0F5
:10DF9000C5F120020AFA02F22BFA05F6A5F12003D8
:10DFA00016432AFA03F31E4306F00102002313432B
:10DFB000EBD0E8B22DF010FD0028E6D02946484607
:10DFC000FCF738FFE1E76F4B1B78DF0700F1648156
:10DFD00000256D4E2F4602E00135242D0DD0294637
:10DFE0003046FCF737FF0028F6D029464846FCF7B4
:10DFF00031FF002856D10137EEE7644B644DB3F88A
:10E0000050102046FCF784FB624B1988204689B2E9
:10E01000FCF77EFB604B1A68530103F02001C2F34A
:10E0200040030B43C2F3800143EA4103C2F3C00142
:10E0300043EA8103C2F3401143EAC10102F0100236
:10E0400011432046FCF764FB04A904222046FCF798
:10E0500017FB23682978514A581C206019701188D1
:10E060006429A8BF64212046FCF752FBB8F1960F43
:10E0700000F0078100212046FCF74AFB2168B7F138
:10E08000190348BFA7F11203A3F3C4034A1C22607B
:10E0900020461A460B7005A9FCF7F2FA01231A462E
:10E0A000FDF787BF394604A8FCF7C4FEA3E72B6839
:10E0B0006A689A4240F01581334BFF221A724FF082
:10E0C0000008374D16F038F941463022354885F8BA
:10E0D000008034F01EFD8DF818809DF818300B2B51
:10E0E00000F26A81304F2F4E42469DF8183003EB04
:10E0F000430307EBC3035B7CE3B19DF8183003EBEC
:10E10000430307EBC3035B69A3B19DF8183003EB2E
:10E11000430307EBC3032021586946F82200FBF7AD
:10E120007BFB2B7856F82300FBF712FD2A7801328F
:10E13000D2B22A709DF818300133DBB28DF8183056
:10E140009DF818300B2BD0D92368591C21601A7008
:10E15000B9F1000F3DF42BAF144BC9F80030012387
:10E160001A46FDF726BF00BF287B002065830020EC
:10E1700068830020004A0020DC440020D4450020B1
:10E18000DC450020CC81002088240020B01D002028
:10E19000107B00208CD20020646900207643002090
:10E1A00007CD00209C780020F06D0020FDCE0308F4
:10E1B00090E33FF42368B178C44A581C206019707A
:10E1C00023681278591C21601A70FEF7FEB9C04A04
:10E1D00092E82200FEF75BB8D9F8003013F48053C0
:10E1E000B4EEE88A63D0F1EE10FAC0F2CD80B4EE5E
:10E1F000C98AF1EE10FA0DD8DFEDB67A9FEDB67A46
:10E2000077EEC87AB4EEC78AF1EE10FAB0EE678AFC
:10E2100000F2BA80F7EE007A78EE677AB6EE007A0E
:10E22000F0EE696AE7EE876A40F2E932FDEEE67ADF
:10E2300017EE901AB1F5FA6FA8BF4FF4FA61914248
:10E24000B8BF114689B2002B3EF462AAB5EE408AEF
:10E25000F1EE10FA40F2DC5308BF1946FEF758BA47
:10E2600095F824209D4B002A40F085803046FEF72B
:10E27000A3B821680123CA1822601A460870FDF766
:10E2800098BE23680322591C21601A7023686A789B
:10E29000591C21601A70F1E6069B43F001030693B6
:10E2A00096E62846FCF7E0F98D4EFEF7F3BDF1EE59
:10E2B00010FAAFDA4FF47A71FEF72ABA931C2B608A
:10E2C0005678022E3EF6D5AD2846FCF7CDF9854AA4
:10E2D00002EB46024FF0FF33A2F85E001A46FDF74C
:10E2E00068BE5A1C19462A607F4811F8022B027238
:10E2F00029605B784372042A03D9FF2A7DF4DFAFDB
:10E30000DDE67A490978994205D8022A7DF4D7AF2B
:10E31000FF2B7DF4D4AF22680123D1182160137044
:10E32000B9F1000F3DF443AE714AC9F800201A4616
:10E33000FDF73FBE0AEBC6072846BA70FCF794F912
:10E340002B682AF836001A46591C296012F8021B5D
:10E35000F9702A605A783A71DA1C2A609A78BA7190
:10E360001A1D2A6008F10108DB787B71C1457FF432
:10E370002AACFDF71CBE5978022917D003290CBF1F
:10E3800004203046FEF718B84FF47A715EE7931C0C
:10E390002B60584B51781970D11C296091785970B5
:10E3A000111D2960D2789A70FEF763BD042A34BF2C
:10E3B00002200320FEF700B84246C5E62B6831680C
:10E3C000581C1A46286012F8020B81F831002A60A6
:10E3D0005B7881F8323068E42846FCF745F9A8F804
:10E3E0000A002846FCF740F9A8F80C002846D6F8A1
:10E3F0000090FCF739F9A9F824002846D6F80090D7
:10E40000FCF732F90D2FA9F826007FF669AC2846F3
:10E41000FCF72AF9A8F80E002846FCF725F9A8F819
:10E4200010005DE40DF11809484629F045FFBDF8DC
:10E430001830B3423FF40BAD2F4B1B68002B3FF459
:10E4400006AD1B689B69002B3FF401AD3046984731
:10E45000FDE42B68D8F80020591C29601978517206
:10E460000B2F3FF4F5A9991C29605B785370FFF7D7
:10E47000EFB95A1C2A601B78003318BF0123F371CF
:10E4800062E40B7803F0FD0326E5114B1020C3F87E
:10E4900000805F6025F038FA184A137843F00103D2
:10E4A0001370002E3DF483AD154A012316601A4601
:10E4B000FDF77FBD00F07F00032828BF002015F086
:10E4C0007BFF01231A46FDF774BD00BFC84500203D
:10E4D000444A002000C0884400C0824418B3002091
:10E4E000C445002010D10020882400205E75002043
:10E4F00059E80008F7510020287B002065830020A0
:10E50000E8280020931C2B60154B51781970D31C00
:10E510002B60144E937886F85C30131D2B60D378F3
:10E5200086F856302846FCF79FF8A6F8580028468B
:10E53000FCF79AF82846FCF797F84FF0FF33A6F857
:10E540005A001A46FDF735BD064B00301E4418BF71
:10E5500001204FF0FF3386F84A001A46FDF729BD27
:10E560008499002010D1002003680A7A591C0160A8
:10E570001A70704738B50B4C23688BB15A68821AF1
:10E58000002A054604DA0CE05A68AA1A002A07DBBA
:10E590009A68226018461A6890472368002BF3D1C6
:10E5A00038BD38BD884500200B4B002210B40272E4
:10E5B00003F59074032102E0072A09DC99798907A1
:10E5C00002D51979815401329C4203F11803F3D129
:10E5D0005DF8044B704700BFD4550408282303702E
:10E5E000704700BF012310B431213224102244703F
:10E5F0004171C2700370037183705DF8044B704702
:10E600002DE9F0410B78047BDB43DEB200F1100210
:10E6100000F1380342F8044F9342FBD1DFF89CC06D
:10E6200000F16001002243F8042F8B42FBD14FF030
:10E63000140E0521002546FA01F303F00103002B17
:10E640001D4414BF4FF019084FF00A0811F0010FD4
:10E65000EDB214BF2746002700220EEB02039BB247
:10E6600000EB8303013242455F61F6D1013A92B279
:10E67000013201390EEB02034A1C9BB201D09E46C7
:10E68000D9E715F0010F14BF19250A2500215A18E2
:10E6900092B200EB82020131A9425461F7D10B44DE
:10E6A0009BB21A1D00EB8202013300219BB2516024
:10E6B000ACF800300361BDE8F08100BF9424002075
:10E6C000254B5B880B332DE9F04F8A4601F1060B91
:10E6D0001FFA83F94FF00108002100271AF801EB17
:10E6E0003E464C460122A4F10B039BB207E00133E6
:10E6F0009BB2B0F80CC0C5F814C09C420AD000EB25
:10E700008305002AF3D100EB830501339BB29C42C1
:10E710006A61F4D1231D00EB83030136092FF6B2A1
:10E7200059600CD0092E14D008FA07F313EA0E0F23
:10E7300014BF012200220C34A4B20137D3E709F13F
:10E740007809DA451FFA89F9C7D1034B5980BDE82A
:10E75000F08F0022EFE700BF942400202DE9F0475E
:10E76000DFF85C80B8F8043004338A461FFA83FC73
:10E7700001F109094FF0010E1AF8017B64460026E9
:10E78000231F0EFA06F29BB23A40BAB1818900EB20
:10E79000830501339BB29C426961F6D10136043492
:10E7A000082EA4B2ECD10CF1200CCA451FFA8CFC47
:10E7B000E2D10023A8F80430BDE8F0871146E6E76F
:10E7C0009424002010B4037B01681F2B09D9203B3F
:10E7D00020224C6802FA03F31C4214D15DF8044B6A
:10E7E000704720220C6802FA03F31C42F6D00C4A50
:10E7F00040680024147002685DF8044B22F00102A6
:10E8000002608B607047064A4068002414700268FA
:10E810005DF8044B22F001020260CB60704700BF3C
:10E82000008E002008B511F067FDFCF7C9FD00BFA0
:10E8300070B54E680546304630F0F2FE314604466B
:10E840000246286831F04EFE2A68131901333B2135
:10E850002B60115570BD00BF024A034B1278197826
:10E8600029F08ABD9024002091240020038A2DE9FC
:10E87000F0478589ADB21D4029D00F4606464FF0BE
:10E8800000484FF00009B5FA85F328FA03F2D243A5
:10E8900091B21B3B15403182042B16D8DFE803F000
:10E8A0003129211903007B6A002B32D003F1FF3A92
:10E8B0001FFA8AFAC7F824903C6A34B123682046CC
:10E8C000514698476468002CF8D1002DDBD1BDE893
:10E8D000F0873868716B036889B29847002DD2D1F0
:10E8E000F5E77868B16B036889B29847002DCAD103
:10E8F000EDE7B868F16B036889B29847002DC2D183
:10E90000E5E7F868316C036889B29847002DBAD101
:10E91000DDE7F36A1FFA83FACEE700BF38282DE956
:10E92000F04700F097810C462ED9802800F0F68041
:10E9300074D8522800F0898040F24C81542800F0AD
:10E94000B2816E2840F0AC81B04B0A681B88B04D94
:10E95000FF2BA8BFFF23511C21601370A96881F30E
:10E960001001204689B2FBF7D3FEAA4B2046198836
:10E97000FBF7CEFE296801F30F01204689B2FBF7B1
:10E98000C7FE0120BDE8F087042800F04E8240F267
:10E99000EE80202800F0A18040F22481242800F09D
:10E9A000D381282840F07C810B68DFF89C829A4E46
:10E9B000591C022221601A70236806275A1C226003
:10E9C0001F7023680A22591C21601A7023680125D0
:10E9D0005A1922601D70B8F800102046FBF798FE07
:10E9E000B8F802102046FBF793FE23685A192260FC
:10E9F0001F7023685022591921601A702368002261
:10EA0000591921601A7031882046FBF781FE204693
:10EA10007188FBF77DFE2846BDE8F08782282FD05D
:10EA2000C0F0AC81A02800F09781FE2840F038812A
:10EA30007A4D05F1080635F8021B2046FBF768FE03
:10EA4000B542F8D10120BDE8F0870A68744E531C26
:10EA50000321236006F10C071170334606200121C3
:10EA60002268551C2560117022689F4202F1010145
:10EA70002160107000F0EA819979D8790633EFE7C8
:10EA80000B68684A624D1178674A581C20601970FB
:10EA9000D1882046FBF73CFE5C4B22681B88FF2B8D
:10EAA00002F10101A8BFFF2321601370A96881F35F
:10EAB0001001204689B2FBF72BFE296801F30F01F4
:10EAC000204689B2FBF724FE2368584A591C127865
:10EAD00021601A700120BDE8F0870B68524D591C67
:10EAE0006A7821601A7023682A78591C21601A708C
:10EAF0002368AA78591C21601A70E9882046FBF720
:10EB000007FE23682A79591C21601A7023686A79E4
:10EB1000591C21601A700120BDE8F087DFF82C81B4
:10EB2000434F444EDFF828A108F10D090A2515E0EE
:10EB3000322D34D0A5F13C00C0B2132835D90023C2
:10EB40002268511C216015702268C84502F101013C
:10EB5000216013703FF476AF18F8015B0A2DE7D1FE
:10EB6000BAF80030FF2BA8BFFF23DBB2E8E702288A
:10EB700000F09C8100F28981012840F091800B68AF
:10EB80000022591C21601A7023685A1C22601870D8
:10EB900023682422591C21601A70BDE8F08733884D
:10EBA000FF2BA8BFFF23DBB2CAE71EF0ABF900289A
:10EBB000C5D003780A2B00F28181B0F9023087FBBF
:10EBC0000312DB17C3EBA2039BB2FF2BA8BFFF23EB
:10EBD000DBB2B5E7442863D1002A3FF433AF164BCC
:10EBE00013602FE705285BD120460B221349FBF762
:10EBF00047FD204608221249FBF742FD2046072226
:10EC00001049FBF73DFD0120BDE8F0879476002018
:10EC1000D481002098D10020CC29002070750020DC
:10EC2000E8320408A676002080830020A8D10020C6
:10EC300067666666E429002025E80008306104085C
:10EC40003C61040848610408C4450020ED2E040816
:10EC5000142A00200B689A4A01205C1C0C60187072
:10EC60000B6805241D180D601C700B680A241D1804
:10EC70000D601C700B6800241D180D601C700B6863
:10EC800014781D180D601C700B6854781D180D60E9
:10EC90001C700B6892781C180C601A70BDE8F08725
:10ECA0000020BDE8F0870B68864A874F581C112169
:10ECB0002060197023681278591C21601A7023682B
:10ECC00097F85C20591C21601A70236897F8562029
:10ECD000591C21601A70B7F858102046FBF718FD30
:10ECE00000212046FBF714FDB7F85A102046FBF729
:10ECF0000FFDBD1E07F1480635F8021F2046FBF741
:10ED000007FDAE42F8D12268704B0C21501C2060E8
:10ED10005D181170226813F8011F501C9D4220607D
:10ED20001170F7D123680222591C21601A70B7F8BC
:10ED30005E102046FBF7ECFC2046B7F86010FBF7AE
:10ED4000E7FC0120BDE8F087614B08461968FBF736
:10ED5000C7FC0120BDE8F0875E4B08461968FBF749
:10ED6000BFFC5D4B20461968FBF7BAFC5B4B2046A5
:10ED70001968FBF7B5FC0120BDE8F087DFF8789152
:10ED8000574F09F10E064FF00A081DE0B8F1500F79
:10ED900032D0B8F1320F31D0A8F13C00C0B2132804
:10EDA0002FD90025294623685A1C2260204683F863
:10EDB0000080FBF7ADFC29462046FBF7A9FC4E4539
:10EDC0003FF440AE19F8018BB8F10A0FDED1454B84
:10EDD0009D68196805EB85054FF6FF736D009D4230
:10EDE000A8BF1D469942A8BF194625EAE57521EA44
:10EDF000E171ADB289B2D6E73B4BE9E797E8220073
:10EE0000E8E71EF07FF80028CBD003780A2BC8D89B
:10EE1000B0F90430B0F9061003EB830383F3500517
:10EE200021EAE171ADB289B2BDE702462F49204621
:10EE3000FBF726FC20460021FBF76AFC2368022230
:10EE4000591C21601A700120BDE8F087284B216809
:10EE50001A78481C20600A70002A3FF4F3AD013A8A
:10EE6000D2B202EB420206EB42025278002A3FF491
:10EE7000E9AD0132D5180133226813F8011F501C87
:10EE80009D4220601170F7D1DCE50B680222591C0D
:10EE900021601A70236801201A18226018702368F4
:10EEA0000022191821601A70BDE8F0870846042274
:10EEB0001049FBF7E5FB0120BDE8F087002387E65A
:10EEC000F75100208499002010D1002059D1002052
:10EED00018530020107AFF1F147AFF1F187AFF1FA3
:10EEE000DC29002090290020D02900202861040876
:10EEF000048E002020610408DD2E0408F0B54B4B81
:10EF00004B491A68096883B00123570200935CBF1C
:10EF100003F180530093D6005CBF43F010030093CD
:10EF20008C0744BF43F0C6030093480744BF43F037
:10EF3000080300930F0748BF43F020033D4948BF33
:10EF40000093160648BF43F44063097848BF009316
:10EF5000D40548BF43F0006301F0EF0048BF0093C1
:10EF600008286D4655D00E2953D0D0033248009B57
:10EF700000784CBF43F4204343F40053D7044CBF04
:10EF800043F0C84343F0884300280CBF07200F20FC
:10EF9000960648BF43F48073540748BF43F40033D8
:10EFA00043F400245205009402D5244A1279A2BBEE
:10EFB000182936D001900027012639462846FCB290
:10EFC000FBF748FF60B11E4B002203F5D87103E048
:10EFD0008B420FD013F80C2CA24203F10C03F7D193
:10EFE0000137242FE9D195E80300164B83E803008D
:10EFF00003B0F0BD7A0904F01F0455F8223006FA78
:10F0000004F4013723EA0404242F45F82240D4D124
:10F01000E9E743F480530093A7E743F4C013009358
:10F02000C6E7009B43F060730093C3E758AA002033
:10F0300064690020784600200C700020987600203B
:10F04000342D0408882400202DE9F84F4E014FF09C
:10F05000000B174D8146904606F120075C46594645
:10F0600028465FFA8BFAFBF7F5FEC0B1A64215D829
:10F07000A74213D900200F4A014604E00131242998
:10F0800014D012F80C0C504502F10C02F6D10A4BC8
:10F0900001EB410103EB81014846C04701340BF10C
:10F0A000010BBBF1240FDAD1BDE8F88F0021F3E7A3
:10F0B00088240020342D0408282D040800210A4A41
:10F0C0000B4604E00133242B0BD012F80C1C8842B1
:10F0D00002F10C02F6D1054803EB430300EB830079
:10F0E00070470020704700BF3C2D0408282D0408FD
:10F0F00000210A4A0B4604E00133242B0BD012F8FE
:10F100000C1C884202F10C02F6D1054803EB4303C4
:10F1100000EB830070470020704700BF342D0408C7
:10F12000282D04081C4C08B501210220FAF71EFD09
:10F13000237803F00502052A29D003F00903092BDF
:10F1400008D000210120FAF711FD00210846FAF746
:10F150000DFDFEE7114A124B11681A680B68114C3D
:10F1600023F001030B601388206823F001031B04C4
:10F170001B0C138018B1292200238271C371022253
:10F180004A21FAF77DFA2068FAF7DCFCD9E711F09A
:10F1900063F92378D1E700BF0038002080290020E0
:10F1A00084290020582A0020022828BF022010B4F9
:10F1B000084C094B207000EBC00200EB82020749AB
:10F1C0005DF8044B013003EB4203C0B20B6024F046
:10F1D00083BB00BF107B002008520020E883002082
:10F1E00008B51EF027FFFBF72FF8BDE808401EF01A
:10F1F00009BF00BF38B5384B5A899989914224BF5D
:10F2000000225A81198ADA89914224BF0022DA81C8
:10F21000DA788AB1072A0FD0304C3148A278012120
:10F220000025062A01709970DD714CD92379DFED34
:10F230002D6A002B36D138BDDA799B78284807EE45
:10F24000103A002A44D0DFED276A0178234CB8EE4B
:10F25000C77A07EE901AA278F8EEE77A27EE267AB8
:10F26000062A67EE877A2BD81F4B03EB8203D3ED78
:10F27000086AF4EEE76AF1EE10FA10DDC6EE877A5E
:10F28000FDEEE77A17EE903A102BA8BF1023012B62
:10F29000B8BF0123DBB28B4228BF0B460370237932
:10F2A000002BC8D0013A032AC5D8B7EE000A80EE79
:10F2B000260A31F021FB2388984238BF208038BDD0
:10F2C000DFED086AD5E7DFED097AB0EE677ACBE7C4
:10F2D000DFED076AB9E700BF18610020E46F002086
:10F2E000C84500206F120338DC2E04086F12833AE1
:10F2F0006F12033938B50D4C0D4DAC4206D2616822
:10F3000020461434FAF724FFAC42F8D3094B0A4CD8
:10F310000A481860002525702EF0EEF9084B094ABE
:10F3200065701A60BDE8384019F070B890010008A7
:10F3300018060008E8830020107B002008520020F7
:10F34000EC8300206685002008B5FFF7D3FF1EF090
:10F3500071FEFAF779FFBDE808401EF053BE00BF0A
:10F36000F0B50C2934D8DFE801F0893333335E334C
:10F370003333343333330700048C9689B2F802E018
:10F380001788734D24F480542404240C0484038CC3
:10F390008488818B23F4005321F4E6411B04090483
:10F3A0001B0C46EA0E06090C43EA063341EA072124
:10F3B000A8429BB2A4B289B200F09E8005F5806598
:10F3C000A84200F09980926884808183026403845B
:10F3D000F0BD048C9589B2F802C0B2F800E05C4F31
:10F3E00024F480742404240C0484038C8688818B88
:10F3F00023F400731B0421F073011B0C45EA0C0479
:10F40000090443EA0423090CB8429BB2B6B241EAAC
:10F410000E015CD04F4CA04259D092688680818307
:10F42000C2630384F0BD048C9589B2F802C0B2F8BF
:10F4300000E0474E24F010042404240C0484038CC0
:10F440008788018B23F0200321F4E6411B04090483
:10F450001B0C45EA0C04090C43EA041341EA0E2193
:10F46000B0429BB2BFB289B25DD03A4CA0425AD0F2
:10F4700092688780018382630384F0BD048C97893E
:10F48000B2F802E01688324D24F001042404240C62
:10F490000484038C8488018B23F002031B0421F075
:10F4A00073011B0C47EA0E0709043B43090CA842F1
:10F4B0009BB2A4B241EA060125D005F58065A842B9
:10F4C00021D092688480018342630384F0BDD58992
:10F4D000148A578A23F4006343EA05254FF6FF3365
:10F4E0002B40958826F440563C4343EA052346EAE0
:10F4F00004169BB2B6B290E7158A24F4804444EA1D
:10F500008514A4B25FE7D689158A578A23F00803C9
:10F51000334324F4407496883D4323F004032C4382
:10F520003343A4B2CDE7D489158A568A23F08003E9
:10F5300043EA04134FF6BF741C40938827F44067D6
:10F54000354344EA031347EA85079BB2BFB28FE70E
:10F5500000000140000401402DE9F84F4FF4A07273
:10F5600000219348934CDFF87492934D934E944F3F
:10F57000DFF86C8233F0CDFA92489349DFF864E209
:10F58000DFF864C200221359834200F0F980B3F11E
:10F59000804F00F0F780AB4200F0F680B34200F0FD
:10F5A000F580BB4200F0F480734500F0F3806345C2
:10F5B00000F0F280434500F0F180DFF830A25345BF
:10F5C00000F0EE800AF5806A534500F0EB800AF502
:10F5D000806A534500F0E880AAF5983A534500F058
:10F5E000E5800AF5806A534500F09C800AF5806A40
:10F5F000534508BF0D2300F096801832B2F59C7F6A
:10F60000C1D1DFF8B081714E08F59C774FF0030A45
:10F610004FF0020998F804301C09013C032C03F058
:10F620000F0378D86A4A32F8140040FA03F2D2077E
:10F6300071D5012505FA03F3013B184030F00AFDAE
:10F64000644B1B5D184416EBC00264D056F8303092
:10F65000614C98F8081003F13F4000F57E00800AE5
:10F66000205C00F01F044009032805FA04F500F0AF
:10F670008180042878D0022804D15348406C054387
:10F6800051484564B2F804E0BEFA8EF2C2F11F029E
:10F6900092B2D00803EB800002F00702046A9200E5
:10F6A0000F25954024EA05040462046A01FA02F277
:10F6B0002243002502624FF0010C2A4603E0102A83
:10F6C00005F1020527D00CFA02F030EA0E0102F132
:10F6D0000102F4D11C680AFA05F1C9430C401C6010
:10F6E000D3F800B009FA05F444EA0B041C609C68E6
:10F6F0000C409C609C689C605C6824EA0000586038
:10F7000058685860D8680140D960D968D960102A13
:10F7100005F10205D7D108F1180847457FF47AAF03
:10F72000BDE8F88F0C2309EBC3034FF0010A93F8EF
:10F73000403003F01F0B5B09032B0AFA0BFA09D0C8
:10F74000042B0CD0022B7FF458AF4B6C4AEA030316
:10F750004B6452E70B6C4AEA03030B644DE70B6BF7
:10F760004AEA03030B6348E71748006B0543164852
:10F77000056387E71448006C05431348056481E777
:10F780000023D0E70123CEE70223CCE70323CAE717
:10F790000423C8E70523C6E70623C4E70723C2E717
:10F7A0000823C0E70923BEE70A23BCE70B23BAE717
:10F7B000CC860020D4550408000400400008004016
:10F7C000000C00400000014000380240C0D2002080
:10F7D000545F0408505F0408EC520408DC2E04084F
:10F7E00000040140001000400014004000400140AF
:10F7F00001490248FFF73AB8E487002000180040AA
:10F8000001490248FFF732B8BC87002000400140A0
:10F8100001490248FFF72AB89487002000040140FC
:10F8200001490248FFF722B89487002000040140F4
:10F8300001490248FFF71AB86C870020000C00400D
:10F8400001490248FFF712B8448700200008004031
:10F8500001490248FFF70AB81C8700200004004055
:10F8600002494FF08040FFF701B800BFF486002046
:10F8700001490248FEF7FABFCC8600200000014093
:10F8800001490248FEF7F2BFCC860020000001408B
:10F89000F0B50468A30AA3F58013502B2AD8DFE83B
:10F8A00003F02A7A8E9229297E29292929292929B2
:10F8B00029292929292929292929292929292929B8
:10F8C00029292929292929292929292929292929A8
:10F8D0002929292929292929292929292929292998
:10F8E00029298286292929292929292929292929D2
:10F8F00029298A00F0BD4FF0480E01264779B00053
:10F900004FEA970C00296BD063460227A5899F40D8
:10F9100083190CEB43032F4303F1040C3A4DBFB2A0
:10F9200045F8231045F82C20A781EFF311815022D0
:10F9300082F31288821905EBC2021369002B46D0AC
:10F9400013620433821905EBC202576917B11F60B5
:10F9500053690433821905EBC202976917B11F601E
:10F9600093690433821905EBC202D76917B11F608E
:10F97000D36904330027CAB21F6082F31188304470
:10F9800005EBC000036A2BBBA38923F001031B0412
:10F990001B0CA381F0BD4FF0700E0226AEE74FF4B2
:10F9A0009C7E0726AAE74FF0200E0026A6E74FF020
:10F9B000E80E0526A2E74FF4887E06269EE74FF064
:10F9C000980E03269AE74FF0C00E042696E705EB43
:10F9D0000E03B7E7A3899BB243F00103A381F0BDF7
:10F9E0000223BF0803FA07F7A389074D9BB223EA56
:10F9F000070387190CEB470CA3810CF1040345F8AE
:10FA00002C1045F8232090E7CC86002010B5036821
:10FA100083480139834282B089B200F0CB80A0F5DF
:10FA20008060834200F0C68000F58040834200F091
:10FA3000B88000F58060834200F0B38000F58060FC
:10FA4000834200F0AE80774C188824686408B4FBC9
:10FA5000F2F4013CA4B282B2B3F1804F0AD07248F2
:10FA6000834207D000F58060834203D000F58060B8
:10FA7000834202D122F0700292B26C48834200F0BD
:10FA8000A28000F58060834200F0A78022F44072DB
:10FA900000F56C4092B283421A80D9621C854FD027
:10FAA0005F4A93424CD001229A821A8892B242F065
:10FAB00001021A80B3F1804F00F099805A4A9342B4
:10FAC00000F0978002F58062934200F0948002F586
:10FAD0008062934200F0918002F58062934200F0D0
:10FAE0008E8002F58062934200F08B8002F57042B6
:10FAF000934200F0888002F57052934200F08580B6
:10FB000002F58062934200F0828002F580629342A7
:10FB10007FD0A2F5983293427DD002F58062934265
:10FB20007BD002F58062934208BF0D2215D002A857
:10FB30004FF0012340F8043D2EF08CFE02B010BDC2
:10FB40000122002119869A821A88394892B242F01D
:10FB5000010283421A80ADD10A46364B03EBC20341
:10FB600001A893F841408DF80440012300228DF84C
:10FB700005308DF807308DF806202EF06BFE1B2C1B
:10FB800008D02E2CDAD12C4B019301A82EF062FE66
:10FB900002B010BD294B019301A82EF05BFE02B00C
:10FBA00010BD204C18882468B4FBF2F4013CA4B2C8
:10FBB00082B251E71B4C18882468B4FBF2F4013C74
:10FBC000A4B282B256E701201A80D9621C859882BD
:10FBD0001A8892B202431A8070E701201A80D96213
:10FBE0001C8598821A8892B202431A8062E7012229
:10FBF000B3E70222B1E70322AFE70422ADE7052213
:10FC0000ABE70622A9E70722A7E70822A5E7092212
:10FC1000A3E70A22A1E70B229FE70C229DE700BF82
:10FC200000040140E06F002000040040001000408C
:10FC300000000140DC2E04082C0100011901000124
:10FC40002C4B98423DD0B0F1804F3CD0A3F57C4383
:10FC500098423AD003F58063984238D003F5806328
:10FC6000984236D003F58063984234D003F5806320
:10FC7000984232D003F57043984230D003F5705368
:10FC800098422ED003F5806398422CD003F5806310
:10FC900098422AD0A3F59833984228D003F5806380
:10FCA000984207D003F58063984208BF0D2202D026
:10FCB000002070470C22104B03EBC20393F8400066
:10FCC00070470022F7E70122F5E70222F3E703225B
:10FCD000F1E70422EFE70522EDE70622EBE7072232
:10FCE000E9E70822E7E70922E5E70A22E3E70B2232
:10FCF000E1E700BF00000140DC2E04082DE9804848
:10FD0000013085B0C3B203938A4D8B4F8B4C8C4E20
:10FD10000A230293DFF82C9228F084FD4FF4FA7A3C
:10FD20004FF0100C4FF47A70D9F80430C3F3080385
:10FD3000002B40F0C180EFF31183002B40F0BC801A
:10FD40002968A26800BF2B689942F9D1D7F800E072
:10FD500000FB0EF39B1AB3FBFEF300FB01314FF0E7
:10FD6000010E0191D9F80430C3F30803002B40F0D1
:10FD70008780EFF31183002B40F082802B68A1680D
:10FD800000BF2A689342F9D1D7F800B000FB0BF20C
:10FD9000521AB2FBFBF200FB0323019A9B1AB3F544
:10FDA0007A7FDFD3BAF1010ABED1039B002B40F06A
:10FDB000BD804FF47A7ADFF88C9150464FF0100CEA
:10FDC000D9F80430C3F30803002B40F09280EFF31E
:10FDD0001183002B40F08D802968A26800BF2B683A
:10FDE0009942F9D1D7F800E000FB0EF39B1AB3FB60
:10FDF000FEF300FB01314FF0010E0191D9F8043000
:10FE0000C3F3080303BBEFF31183EBB92B68A168BD
:10FE100000BF2A689342F9D1D7F800B000FB0BF27B
:10FE2000521AB2FBFBF200FB0323019A9B1AB3F5B3
:10FE30007A7FE3D3BAF1010AC2D1029B013B02935C
:10FE40007FF468AFFBF7BCFAEFF311888CF31288EC
:10FE5000A1682368DB0344BFC6F800E0A1682B68F3
:10FE600032685FFA88F888F31188D7F800801A445E
:10FE700000FB08F35B1AB3FBF8F300FB0233D4E793
:10FE8000EFF311888CF31288A1682368DB0344BF69
:10FE9000C6F800E0A1682B6832685FFA88F888F33A
:10FEA0001188D7F800801A4400FB08F35B1AB3FBF3
:10FEB000F8F300FB023370E7EFF311828CF3128842
:10FEC000D4F808E02368D90303D501233360D4F8BC
:10FED00008E02B683168D2B282F311883A6819447D
:10FEE00000FB02F3A3EB0E03B3FBF2F300FB0131C3
:10FEF00035E7EFF311828CF31288D4F808E0236819
:10FF0000D90303D501233360D4F808E02B683168A6
:10FF1000D2B282F311883A68194400FB02F3A3EBD2
:10FF20000E03B3FBF2F300FB013164E718462EF039
:10FF300001FE3EE750D4002054D4002010E000E041
:10FF40004CD4002000ED00E02DE9F047AD4FAE4E5F
:10FF50001EF070F8BE421ED2DFF83883DFF8389307
:10FF60004446258862197DB14A450DD2052D0BD92D
:10FF700033886188C3F30B03994200F0D88014469C
:10FF800025886219002DEFD1716830461436FAF7D2
:10FF9000DFF8BE42E4D39D4B5A78022A40F2EC804F
:10FFA00000225A701A789A489A490160022A00F28F
:10FFB000DD8002EBC201984B02EB810203EB4202AF
:10FFC000964C104622602DF097FB954A1378A3F1CA
:10FFD000170102290FD9934911F83300002840F086
:10FFE0000381D8000144497829B18F4911F8333091
:10FFF0000BB9182313708D4B9A78042A00F0EB800C
:020000040801F1
:1000000032B91A88B2F5F07F84BF4FF4F0721A80CB
:10001000874D884A2B681A40002A00F0EE80DE07E0
:1000200000F1B580580400F1B980190700F1BD80D6
:100030009A0100F1C1809B0400F1C68023689A8C6C
:10004000D98C914224BF00229A84FFF7D3F81BF089
:1000500065FA10B9784822F02BFA2BF035FD002113
:100060003022764832F055FD754B256803F150017A
:1000700002E0043399427DD01A78002AF9D19C78A5
:10008000D8788442F5D26F496F4B0A7028461D60BC
:1000900028F0AAF86D4B6E4A1E786E496E486F4B79
:1000A0001160C825642212FB06526D4C006B31F8BA
:1000B000041C5A60002221809A60DA601A615A6139
:1000C0009A61DA6183F8202083F8212008B116F0C4
:1000D0008BFB644B9FED645A1B88644A9FED646AF6
:1000E000557B644C64496548086006EE903AF8EE2A
:1000F000E66A1389C5EE265A07EE103A5389127B39
:10010000C4ED005A07EE903AB8EEC77A5C4BF8EEB1
:10011000E77A1D725A7227EE067A67EE867ABDE894
:10012000F04783ED017AC3ED007A1DF06BBF637970
:100130009B077FF424AF716894F804A03046FAF767
:1001400007F83388BAEB133F0BD173887068AA1F86
:10015000C3F30B039A4204F10601A8BF1A4630F01C
:10016000C1F91436BE42FFF4FBAE14E700221A7048
:10017000294A25E7012286E72649254802EB420263
:1001800001EB82011A780160022AEFD811E73D489D
:10019000FAF714F82B6858047FF547AF3A48FAF796
:1001A0000DF82B6819077FF543AF3848FAF706F8C2
:1001B0002B689A017FF53FAF46F20900F9F7FEFF81
:1001C0002B689B047FF53AAF3148F9F7F7FF4020E1
:1001D000F9F7F4FF32E71A8BB2F57A7FBFF418AF64
:1001E0004FF47A721A8313E7D8000D186D68002D4A
:1001F0007FF4F8AE17251570F4E643F008032B6082
:100200000DE700BF1806000890010008107B0020D1
:10021000EC8300206685002008520020E88300203F
:100220007846002038570408A85D0408E46F0020D1
:100230001853002009600002909900205C250020DE
:100240007C4600209022002090250020FC410020C8
:10025000F0250020E04400209C830020E07A00206C
:10026000EA440020F4280020C0C9FB489424002060
:1002700017B7D138F8280020C03A00203661023D77
:100280009C3A002008600002092000020160000280
:1002900009400002074000080080000808B51DF072
:1002A000C9FEF9F7D1FF1DF0ADFEFFF74DFE0120AD
:1002B000BDE8084023F010BB2DE9F04F013085B0B8
:1002C000C3B203930B4602918B4C8C4E002B00F073
:1002D00099808B4D8B4FDFF8309228F0A3FA4FF4C2
:1002E000FA7A4FF0100C4FF47A70D9F80430C3F357
:1002F0000803002B40F0DE80EFF31183002B40F069
:10030000D9802968A26800BF2B689942F9D1D7F833
:1003100000E000FB0EF39B1AB3FBFEF300FB013180
:100320004FF0010E0191D9F80430C3F30803002BFC
:1003300040F08780EFF31183002B40F082802B6820
:10034000A16800BF2A689342F9D1D7F800B000FB3A
:100350000BF2521AB2FBFBF200FB0323019A9B1A29
:10036000B3F57A7FDFD3BAF1010ABED1039B002B2C
:1003700040F0BD804FF47A7ADFF88C9150464FF010
:10038000100CD9F80430C3F30803002B75D1EFF338
:100390001183002B71D12968A26800BF2B68994294
:1003A000F9D1D7F800E000FB0EF39B1AB3FBFEF384
:1003B00000FB01314FF0010E0191D9F80430C3F375
:1003C000080313BBEFF31183FBB92B68A16800BFCF
:1003D0002A689342F9D1D7F800B000FB0BF2521A09
:1003E000B2FBFBF200FB0323019A9B1AB3F57A7F61
:1003F000E3D3BAF1010AC4D1029B013B0293002B63
:100400007FF467AF05B0BDE8F08FEFF311888CF390
:100410001288A1682368DB0344BFC6F800E0A16826
:100420002B6832685FFA88F888F31188D7F8008063
:100430001A4400FB08F35B1AB3FBF8F300FB02332A
:10044000D2E7EFF311888CF31288A1682368DB03ED
:1004500044BFC6F800E0A1682B6832685FFA88F8EC
:1004600088F31188D7F800801A4400FB08F35B1A60
:10047000B3FBF8F300FB023370E7EFF311828CF368
:100480001288D4F808E02368D90303D50123336028
:10049000D4F808E02B683168D2B282F311883A6848
:1004A000194400FB02F3A3EB0E03B3FBF2F300FBD2
:1004B00001317FE7EFF311828CF31288D4F808E062
:1004C0002368D90303D501233360D4F808E02B68EF
:1004D0003168D2B282F311883A68194400FB02F302
:1004E000A3EB0E03B3FBF2F300FB013118E7184650
:1004F0002EF020FB3EE700BF10E000E04CD40020CF
:1005000050D4002054D4002000ED00E0204B5B6864
:10051000C3F3080330B4BBB9EFF31183A3B91D4B88
:100520001D4C1868A16800BF1A689042F9D11B4B96
:100530001C684FF47A7202FB04F3591AB1FBF4F110
:1005400030BC02FB00107047EFF31182102383F3DD
:10055000128811498C680B6813F4803F104B02D04D
:10056000012018608C680B49D2B20D68186882F3BC
:1005700011880A4B19684FF47A72284402FB01F380
:100580001B1B30BCB3FBF1F302FB0030704700BF14
:1005900000ED00E050D4002010E000E054D4002032
:1005A0004CD400202DE9F84F8046FFF7AFFF254ED1
:1005B0002549DFF8A0E0254A254D844610274FF451
:1005C0007A740120DEF80430C3F30803D3B9EFF3E3
:1005D0001183BBB90B68D2F808A000BFD1F8009016
:1005E0004B45F7D1D6F800B004FB0BF9A9EB0A098B
:1005F000B9FBFBF904FB0393A3EB0C034345E1D3E5
:10060000BDE8F88FEFF3118A87F31288D2F808B0AB
:100610001368DB0344BF2860D2F808B00B68D5F834
:1006200000905FFA8AFA8AF31188D6F800A09944FC
:1006300004FB0AF3A3EB0B03B3FBFAF304FB09334C
:10064000DAE700BF54D4002050D4002010E000E0CE
:100650004CD4002000ED00E02DE9F04FDFF830C170
:10066000474A4849484E494D8046102718F1FF38FF
:10067000C0F08480DCF80430C3F30803002B5CD1A5
:10068000EFF31183002B58D10B68946800BF086802
:100690008342F9D1D6F800904FF47A7000FB09FE3E
:1006A000AEEB040EBEFBF9FE00FB03EEDCF80430FB
:1006B000C3F308034FF47A740120FBB9EFF31183FD
:1006C000E3B90B68D2F808A000BFD1F800904B4501
:1006D000F7D1D6F800B004FB0BF9A9EB0A09B9FB76
:1006E000FBF904FB0393A3EB0E03B3F57A7FBDD2B2
:1006F000DCF80430C3F30803002BDFD0EFF3118ADA
:1007000087F31288D2F808B01368DB0344BF28606F
:10071000D2F808B00B68D5F800905FFA8AFA8AF32D
:100720001188D6F800A0994404FB0AF3A3EB0B034D
:10073000B3FBFAF304FB0933D5E7EFF3118487F336
:100740001288D2F808901368D80303D501232B60D0
:10075000D2F808900B682868E4B284F31188D6F8C0
:1007600000A04FF47A7400EB030E04FB0AF3A3EB32
:100770000903B3FBFAF304FB0E3E97E7BDE8F08FE5
:1007800010E000E050D4002054D400204CD40020CD
:1007900000ED00E030B4EFF31183102282F31288F1
:1007A0000649074C0A680748013200250A6025609F
:1007B000DBB2026883F3118830BC704750D400204C
:1007C0004CD4002010E000E00F4B1B88014643B9D9
:1007D0000E4B0F4A1B7810680BB981F00101F9F735
:1007E000BDB90C4B5A691AB118B91A68106058741F
:1007F0007047094A18681188084A92FBF1F20121F2
:1008000002605974704700BF28D400202AD4002009
:100810002CD4002030D4002048D4002020A1070090
:1008200038B5254B5C69236B73B1A36D626BCAB19C
:10083000998A1A88C90592B201D5D20700D438BD69
:100840004FF6F7721A8038BDA36D99891A88890608
:1008500092B2EBD59206E9D5E26ACAB1988880B225
:100860009047E2E799891A880D0692B2E0D5100602
:10087000DED5A26A616A8A4219D0A1692569885CBD
:1008800098800132B2FBF5F105FB1122A262CFE79D
:100890009B88E2696169DBB28B54E269E068A36D11
:1008A0000132B2FBF0F100FB1122E261BEE7DA682F
:1008B00022F08002DA60BBE70438002038B5254B0F
:1008C0009C68236B73B1A36D626BCAB1998A1A8855
:1008D000C90592B201D5D20700D438BD4FF6F772E0
:1008E0001A8038BDA36D99891A88890692B2EBD512
:1008F0009206E9D5E26ACAB1988880B29047E2E7E9
:1009000099891A880D0692B2E0D51006DED5A26A42
:10091000616A8A4219D0A1692569885C9880013290
:10092000B2FBF5F105FB1122A262CFE79B88E269D9
:100930006169DBB28B54E269E068A36D0132B2FBFE
:10094000F0F100FB1122E261BEE7DA6822F08002DA
:10095000DA60BBE70438002038B5254B1C68236BF0
:1009600073B1A36D626BCAB1998A1A88C90592B234
:1009700001D5D20700D438BD4FF6F7721A8038BDC2
:10098000A36D99891A88890692B2EBD59206E9D5AA
:10099000E26ACAB1988880B29047E2E799891A88DA
:1009A0000D0692B2E0D51006DED5A26A616A8A42CF
:1009B00019D0A1692569885C98800132B2FBF5F1F4
:1009C00005FB1122A262CFE79B88E2696169DBB275
:1009D0008B54E269E068A36D0132B2FBF0F100FBD9
:1009E0001122E261BEE7DA6822F08002DA60BBE73A
:1009F000043800202DE9F04F9A4A9B49137895B0AE
:100A00000446099000F59C4020300C900860002BB3
:100A100000F03284954909688C4240F296809449EE
:100A2000059109689348944DDFF888B20391013B22
:100A3000137001F4805302900893002B40F09480CF
:100A4000029B5B7D002B40F06083039B180400F148
:100A50006386039BD9050BD5099A884BDFF858A20A
:100A60009A429AF8022001F21D80002A41F01E806D
:100A7000834B0493834C039B13F4805740F0A4836F
:100A8000029BBBF906605B8B9E42B4BF0026012629
:100A90007D4B1B6813F0805373D0049A127812F0C8
:100AA000010275D002987949808C91ED037A07EEA6
:100AB000900AF8EEE77AB4EEE77AF1EE10FA80F2F7
:100AC0000487002E69D195F8A410002965D17048DB
:100AD0007049006890F830004FF0000EC1F800E057
:100AE000C1F804E0C1F808E06B49002856D108704D
:100AF000002A57D0039AD00654D5684A1278D106F6
:100B000050D4002F4ED1002B4CD1039B5A0249D414
:100B100094F800C0BCF1000F01F05286604B9B7846
:100B2000002E41F076863BB15E4A5F4B12681B682F
:100B30009B1A002BC1F29B86102022F0B9FD0123E5
:100B400085F8A53094F800C02EE0494B05931B684A
:100B50000393484A484D029203F48053DFF854B19E
:100B60000893002B3FF46CAF00214748FAF772F965
:100B700000287FF465AF12F06FFF059B1B6803939D
:100B80005EE7039A520288D4049A127802F00102B6
:100B9000002185F8A410002E99D03F49012008704B
:100BA000002AA7D194F800C0029ABBF900E0508B4C
:100BB000918BBBF902208645CCBF8027002747F0E8
:100BC00040038E45A8BF3B469B0843F08007824206
:100BD000C8BF3B4643F040078A42B4BF3A461A4674
:100BE0009208BBF904E0BBF9067042F08003864529
:100BF000C8BF1A4642F040038E45A8BF13469B0863
:100C000043F080028742D4BF1846104640F04002AD
:100C100095F8A6308F42ACBF014611468B4200F0DA
:100C20008F84002385F8A61085F8A730BCF1000F4B
:100C300000F0F885059B1D4A1B68039203F004032E
:100C4000002B40F02C840DF14808194C0023C8F803
:100C5000043004F15009129340F6330A192740F288
:100C600083362EE0E07800208C770020DC780020AE
:100C700058AA002078740020AC240020404B4C007F
:100C8000CC81002090220020ACD10020A87600204A
:100C9000E8830020F8450020183A002065830020F2
:100CA000E845002050D400207C43002064690020E7
:100CB0007C46002054C90020E07A002004344C45D2
:100CC00020D0A278E3789A4217FB0261F6D26278CC
:100CD000043217FB03633BF912205245A8BF52466A
:100CE000B2F5617FB8BF4FF461728A42E6DD9A4285
:100CF000E4DC21782329E1D840460434FAF79AF855
:100D00004C45DED1AD4B98E803001E78AC4B83E830
:100D10000300002E00F053830121A948FAF79AF846
:100D2000002840F00D81059B1B68D90500F1038167
:100D3000A44C23881EB226F001061FFA86F843450C
:100D4000A4F8008000F070849F4E02270F204FF01F
:100D5000140A4FF0FF09377086F801A086F8029058
:100D600022F0A6FC39469648B4F80080FAF772F8EB
:100D7000002840F0DE8728F002039BB24345238021
:100D80000BD0914B1421FF2202260F201E705970A8
:100D90009A7022F08DFCB4F800808C4BDFF848A2EA
:100DA0001978DAF80400029318F0030F08BF81F0F5
:100DB0000201C1F34001F8F7D1FE039B1B6813F059
:100DC0000A0F1DD005217E48FAF744F8002800F0EC
:100DD00014852688730740F1518779480621FAF770
:100DE00039F8002800F0F684770640F1648707217F
:100DF0007348FAF72FF8002840F0A781039B1B687F
:100E0000980600F1B28126886D480C21FAF722F885
:100E1000002800F0B48046F48073B342238009D0E8
:100E2000694B02251421FF220F201D7059709A7002
:100E300022F03EFC664B1B78082B00F0AC800E2B9A
:100E400000F0A980059B1B685E0542D5614B1B79AC
:100E5000002B58D014215A48F9F7FCFF002856D12E
:100E600025F0F2FF012022F075FB90B3DFF87C81C2
:100E700000254FF0CC0902E0DDB2022D29D809FB94
:100E800005F76B1C58F80760002EF5D1C378524A5D
:100E900090F9020052F823300196032200920121BA
:100EA000324621F031FB034605EB450000EB001014
:100EB000059353B1314608EB8000CC2231F029FE76
:100EC000059B48F807300135EDB228F033FE0028C5
:100ED000D3D1049B1B78DD0740F18A803F49404A0B
:100EE00001230B701370029BDAF80000197801F0EF
:100EF0000101F8F733FE039B1B685A0700F1E880F5
:100F000015B0BDE8F08F049B1B78D807A8D53C200E
:100F100029F046FB0028DCD008F002FF3C2029F035
:100F2000E1FA0028D5D008F0FBFE3C2029F0DAFADF
:100F30000028F1D1CDE72B4BDB78002B3FF4F8AE46
:100F4000039B1B689A077FF5F3AE1E4CB4F8008034
:100F500018F0010F7FF40FAF48F00103984523808C
:100F60003FF409AF184B1421FF2202260F201E70F8
:100F700059709A7022F09CFBB4F80080FBE626F4CE
:100F800080739BB2B34223807FF44AAF104B1B782F
:100F9000082B7FF454AF228822F040039BB29A4280
:100FA00023803FF44FAF084B02251421FF220F206E
:100FB0001D7059709A7022F07BFB43E7084D0020AA
:100FC000ACD10020E48300200842002018D4002087
:100FD000784600209876002038550408CD810020FE
:100FE000FC280020E07A00201CD400203CC5002012
:100FF000814B93F80090B9F1000F5FD1DFF8748254
:101000007E4F18F8030C3E784146A8F103052AF0FC
:10101000B9FC002800F02883002E40F07A8305F107
:10102000080168792AF0AEFC002841F05282744928
:10103000A87A2AF0A7FC002800F02983022E41F0AC
:101040004C827049E87B2AF09DFC002841F03182F7
:101050006D49287D2AF096FC002800F02983042E93
:1010600041F02B826949687E2AF08CFC002841F00F
:1010700028826749A87F2AF085FC002800F0298390
:10108000062E41F02282634995F823002AF07AFC6B
:10109000002840F06D87604995F828002AF072FC1E
:1010A000002800F02983082E40F078875B4995F8E6
:1010B0002D002AF067FC002840F02983584B0122BC
:1010C0001A702AF0E4FE039B1B685A077FF518AFDD
:1010D00003202AF081FC002800F04086238813F0CA
:1010E00008047FF40DAF082022F026FC4D484E4D39
:1010F0004E494F4A4F4BBBF8066000682E8008608F
:1011000014601C6015B0BDE8F08F029A013BD27DDF
:101110003BF91330002A40F09E83A3F57A73B3F5B0
:101120007A7FA8BF4FF47A7323EAE37307EE903A0D
:101130009FED417AF8EEE77A67EE877A3F4AFCEE58
:10114000E77A17EE903A138083E43D4B3D4AB3F9BA
:1011500004303D4982FB0302DB17C3EBA202039B71
:101160000A801B6898067FF54EAE384B1B789907AE
:1011700004D5374F3B78042B00F28B86268816F077
:10118000300F3FF441AE102022F0BEFB202022F0B1
:10119000BBFB304B268800221A702F492F48304F56
:1011A000304D00220A6030493A6000232A604260D4
:1011B0008261036083604361C3610B604A608B603E
:1011C0004B618A61CB611FE61D212848F9F742FE79
:1011D00000287FF455AC264A029BD2881B8BBBF9B2
:1011E0000660991A8E4240F33F8613449E42B4BF74
:1011F000002601264CE400BFCD8100202C000020F9
:10120000DF3B0020E43B0020E93B0020EE3B0020D8
:10121000F33B0020F83B0020FD3B0020023C002077
:10122000FC2800208C830020DC280020E8280020F7
:10123000E0280020D8280020AAF1823F98D1002081
:101240009483002067666666D028002065830020AE
:1012500068830020024A0020F44A0020A44A0020AB
:10126000EC39002058290020CC4A0020ACD10020C5
:10127000E4410020D53B00209A4D9B4B2E780293F1
:101280009A4F002E00F0F082B6B1DFF8A092DFF89E
:10129000A0B2DFF85882CA460024072C4046E1B2CB
:1012A0007B6841F35082984700B20134A6422BF884
:1012B000020F0AF1040AF0D18D4B05931A460999E1
:1012C0008C4B12680392A3FB013E42F201031340D0
:1012D0004FEA9E1E079300F0C3828748874A884BD7
:1012E00000788849069012781A70069B08702BB116
:1012F000834B93F800B08BF001030693824A029966
:10130000127838781090B1F82680088D91F822C0B4
:101310000B92098B0B9A119195F829107B4B0E902B
:1013200008461146A3FB01135B0803EB4303D31AE2
:10133000DBB20D93039B2C78754EDFF8F8B1DFF824
:10134000F891CDF810800F220CF1040C03F48053B7
:1013500085F828200A955FFA8CFC109D0F92A24612
:1013600008930021804610972CB9AC4599BFE246FE
:101370006446AA462C46A14280F22583069B002B98
:1013800000F0D682634B049833F9112097B287425C
:101390004FEA410303D30E98874240F20F8359F876
:1013A0002120964580F0CE823BF90320079F002F35
:1013B00040F0E2822BF8032001310636D4E7DFF853
:1013C0007C91554F09F15A044FF00108494619F82C
:1013D000010C2AF0D7FAF8B199F8040099F8023014
:1013E00099F803E000EB400105EB8101013BD1F8E6
:1013F000B42003EB43033B4493420DD095F8E02027
:1014000081F8B0E008FA00F022EA0000C1F8B43038
:10141000C1F8B86085F8E00009F106094C45D5D15E
:101420003E493F4A374B0968D2F8009093F800A034
:101430003C4C0691002663685BB31F784FB3A268EB
:10144000A9EB0202002A0ADB95F8E0200121B14055
:1014500022EA010209F5FA7185F8E020A160BAF1EB
:10146000000F16D0227859780432D2B2002940F009
:10147000318202993BF91220098B01F1C8008242A6
:1014800040F3C68495F8E0209B783241D20740F1C2
:1014900046850136042E04F10C04CCD13CE495F8C9
:1014A000AB3053B1049B1B78D90706D5029BBBF91F
:1014B00006205B8B9A4200F3248511211A48F9F724
:1014C000C9FC002800F0E88195F8AE302BB995F8FA
:1014D000A93013B93223A5F8AC30012385F8AE301A
:1014E000FFF7B1BBAC240020787400209085002069
:1014F00058AA0020D34D621068770020281C0020D5
:10150000291C0020A97A0020E1780020ABAAAAAA11
:10151000D8240020B0240020882F0408EC83002069
:1015200050D400205C250020ACD100204C79002054
:10153000AE24002054C90020E4780020ED3A0020B9
:1015400095F8A790B9F1F90F00F2B88109F10109F6
:101550005FFA89F985F8A79085F8A610BCF1000F0D
:1015600000F06181B9F1140F7FF464AB5F2940F0A2
:101570006D81049E337813F0010300F0558712F05B
:101580006BFA337803F00103002B7FF453AB95F82B
:10159000A620572A00F0B886059B1B6813F00403A9
:1015A00002D05A2A00F0FE845D2A00F01E875B2AD2
:1015B00000F036875E2A00F0B884562A00F0B7871C
:1015C00023782BB16F2A00F0A287CB4B0021196042
:1015D000972A00F0A087A72A00F086840021BB2A62
:1015E000129101F06180B72A01F03E80BE2A01F01D
:1015F0005E80BD2A01F06480792A01F09D807A2AFC
:1016000001F093809E2A01F089809D2A01F07E805E
:10161000AE2A01F06780AD2A7FF40CABFF210020D9
:1016200024F004FDFFF706BB0221B448F9F712FCD1
:1016300000283FF4A0AB268018F0020F7FF4ADAB7A
:1016400048F00203434523803FF4A7ABAC4B022292
:1016500014211A700F20FF2259709A7022F028F876
:10166000B4F80080FFF799BB08F1050168792AF00A
:1016700089F900283FF4DBAC012E40F02A8705F100
:101680000D01A87A2AF07EF9002840F026879D49AE
:10169000E87B2AF077F900283FF4DAAC032E40F01B
:1016A00008879949287D2AF06DF9002840F00587C0
:1016B0009649687E2AF066F900283FF4DAAC052ED8
:1016C00040F0FF869249A87F2AF05CF9002840F09C
:1016D000FC86904995F823002AF054F900283FF43D
:1016E000DAAC072E40F044848B4995F828002AF0A4
:1016F00049F9002840F05284884995F82D002AF0D5
:1017000041F900283FF4DAAC092E3FF4D7AC4FF092
:1017100009094B4600F02FBCD5F88C30099AD31A32
:10172000002BFFF696A97E4A95F89030517C7D4AB1
:10173000029C32F811200C98A17DC5F88C00013371
:1017400003F00F0385F890302B4492B292FBF1F234
:1017500083F8942095F8940095F8951095F89620C4
:1017600095F8973001440A4495F8980095F8991037
:101770001344184495F89A2095F89B3001440A4484
:1017800095F89C0095F89D101344184495F89E20F8
:1017900095F89F3001440A4495F8A00095F8A110EF
:1017A0001344184495F8A23095F8A32001440B4443
:1017B0001A4442F30B12642AE17DA8BF642213B2DB
:1017C00009B1C2F1640307EE903A9FED577AF8EE43
:1017D000E77AB1E426F040039BB2B34223803FF4A2
:1017E00006AB474B02261421FF220F201E705970B2
:1017F0009A7021F05DFFFFF7FABA238823F0040600
:10180000B6B2B34226803FF4E8AA3D4B022614212B
:10181000FF220F201E7059709A7021F049FF268810
:10182000FFF7DBBAE14600213448F9F713FB30B388
:10183000002385F8A83011F041FC95F8A730142B4F
:101840007FF4F8A92378002B40F0DF87049B1B78F6
:1018500003F0010398E6C3F53B6308331BB25CE475
:10186000324B1B78069342E593F822303E780433DE
:10187000DBB2B3428EBF2E702B701E4604E5049B74
:101880001D4A1B781060DB0700F12185B9F1140FA8
:101890003FF47DAEFFF7CEB995F8A930002B3FF4A9
:1018A000D2A9049B1B7813F001037FF4CCA9012279
:1018B00085F8A93085F8AA20FFF7C5B985F8A630C4
:1018C000BCF1000FAFD0FFF7B5B9012185F8A41026
:1018D000FFF763B9012900F0368595F8E020012370
:1018E000B34001361343042E85F8E03004F10C04B4
:1018F0007FF4A1ADFFF710BA80430020ACD10020E7
:1019000008420020E43B0020E93B0020EE3B0020A1
:10191000F33B0020F83B0020FD3B0020023C002070
:101920007C8600209886002014AE2341A97A0020EE
:10193000049B002B40D059F8212096454FEA4103E3
:10194000FFF432ADB84AB848D25CC718002A00F09C
:10195000BA81022A40F065817A7802EB820202EBBA
:10196000820202F2EE2292B2032940F39280079F94
:1019700012B2002F3FF41EAD0D985F1807440A986D
:1019800000EB4707BA85B8F1000F03D10B98022886
:101990007FF610ADB6F802803288B788424417440B
:1019A000A24A3FB282FB0702A148A2EBE772C752EC
:1019B00012B24FF00108FDE41A464B000EF596777F
:1019C00049F82170F2E40F990A9D9A4B109F85F80F
:1019D00000A00F2942460CBF0122002285F8298071
:1019E00085F828101A7006D11B219348F9F732FAAE
:1019F000002800F0E5849148914B82681968914B6A
:101A0000C1608A1A0121197043688F4E9A42029A66
:101A1000317088BF002392F8226088BF80F821309F
:101A2000089B3878B2F826C0B2F818E00436F6B24F
:101A3000002B00F0558186427B4A40F2C781834EDD
:101A4000174600210CB982460446A14218DA12F862
:101A5000113083B1022B0CD17B7803EB830303EBB2
:101A6000830303F2EE239BB226F8023B01310237D7
:101A7000E8E73388F8E7CBB2032BFAD87346F3E7ED
:101A800085F800A00B9B724A01331370089BFEF788
:101A9000D4BF012000FA01F70F9820EA070012B224
:101AA0000F9083E412B901228AF80220694B049353
:101AB0001C789AF8218004F001031B20039329F07D
:101AC0008BFFB8F1010F079000F0D18104F0020301
:101AD00006939AF82020604CDFF884915F4E584FAF
:101AE000052A00F29580DFE802F08579032F3E5148
:101AF000B8F1010F04BF05238AF82030039B002BA7
:101B000000F0BA80029B3868B3F91810B9F80230B7
:101B1000002261F30F0263F31F42002361F30F03FE
:101B200061F31F43DAF81410CBF804208142CBF89C
:101B3000003080F01E810323069347F230520323C6
:101B4000CAF81C208AF82030338843F0020333801F
:101B500011F082FF3A68DAF81C3013440422CAF804
:101B600018308AF82020B8F1010F40F037843B6824
:101B7000DAF818209A424BD2207818B929F02CFFB5
:101B8000002845D1338823F0020333803A68B9F83E
:101B90000630642101FB03234FF4806000228AF8A1
:101BA00020208AF80320CAF8103021F0ADFE9AF800
:101BB000202095E729F03CFF012800F07084079B66
:101BC000002B40F05781B8F1010F21D03B68DAF8C3
:101BD00010209A4246D301238AF82030B8F1010F31
:101BE000D4D099F80830012B3CD00FF0B3F89AF814
:101BF000202075E7039B002BDCD1079B4FF480600E
:101C0000002B00F0A88021F097FE0022CAF81020D7
:101C1000069B002B40F0A980059B1B680393FEF7F1
:101C20002BBF3BF803209FE6807900205655555581
:101C30002025002079510020ACD10020E07A00203E
:101C400050D40020281C0020291C002054C900204A
:101C5000E1780020CC81002090220020E283002047
:101C6000FC4100200FF076F8032240F6B8338AF8E2
:101C70002020CAF81C3067E73B685EE746F00403A3
:101C80009E4223800AD0AE4B02261421FF220F2051
:101C90001E7059709A7021F00BFD2688A94BAA4A34
:101CA000B3F90430A94982FB0302DB17C3EBA2039B
:101CB0000B80FFF792B846F04003B34223807FF4D5
:101CC00090ADFFF794B8CAB2022A40F2FD82032A0F
:101CD000A7D1119A0898049F002808BF3A4643E606
:101CE000864219469A4A4CD89A4817460CB9B246C9
:101CF00034468C427FF7C4AE12F8113083B1022B08
:101D00000CD17B7803EB830303EB830303F2EE2315
:101D10009BB220F8023B01310237E7E70388F8E77E
:101D2000CBB2022B03D9032BF8D16346F1E77346FC
:101D3000EFE728F001039BB2434523803FF47CACDE
:101D40000F20377086F801A086F8029021F0B0FCD1
:101D5000B4F8008070E421F0D7FD56E7082021F0A8
:101D6000D3FDFFF7CDB803230693069821F0A0FC1E
:101D700052E7B8F1010FF6D103239AF82020069319
:101D8000AEE6744E17460CB982460446A142BFF631
:101D900077AE12F8113083B1022B0CD17B7803EBB4
:101DA000830303EB830303F2EE239BB226F8023B8B
:101DB00001310237E7E73388F8E7CBB2022B03D9CA
:101DC000032BF8D16346F1E77346EFE76148174606
:101DD00000210CB9B24634468C427FF751AE12F85E
:101DE000113083B1022B0CD17B7803EB830303EB1F
:101DF000830303F2EE239BB220F8023B013102374A
:101E0000E7E70388F8E7CBB2032BFAD87346F3E78A
:101E1000C8398A425BDA95F8E0209B783241D007D6
:101E20003FF537ABC3F10008012021F055FD7A1EC4
:101E3000162A00F25F81DFE812F0F1010502DA01F3
:101E40003F0123023402B2019F018A017501600142
:101E50005D013F014F013402B2019F012B011701C7
:101E60000301C501ED00D9000126FEF711BE0023D4
:101E700006932EE699F80430002B3FF4A4AE0EF042
:101E800069FF03224FF47A738AF82020CAF81C30C5
:101E90005AE60A2029F0A0FD26888046002800F096
:101EA000A882F20640F1CF8395F8F080B8F1000FD8
:101EB0007EF4AAAF0E2021F0FBFB012385F8F03061
:101EC0002688B8F1000F7FF468A9FEF79DBF95F84A
:101ED000E0300122B24023EA020309F5FA7285F8E4
:101EE000E030A260FFF7D5BA1B49059B0A781B6852
:101EF00042F004020A7003F00403184A0392FEF74A
:101F00009FBE00211648F8F7A5FF00287FF4D5AA48
:101F1000322385F8AB00A5F8AC30FFF7CEBA98466F
:101F2000002B0CBF012002207FE70E4B0222032072
:101F30000D4C0E4922700B6021F0CEFCFEF77ABEEC
:101F4000084200209483002067666666144B0020D8
:101F50008079002054C90020658300206469002036
:101F6000ACD100209C520020107B0020E883002090
:101F70004FF007094B4603EB83031D4487F800909D
:101F8000A978687826F0C8F9049BB84A1B78012123
:101F90001170D9077FF595A8FEF7A5BF4FF0080986
:101FA0004B46E8E795F8A920002A40F0918395F880
:101FB000AB2082F0010285F8AB20002A40F0838339
:101FC000AB49096811F4003104D0AA490979002904
:101FD00040F047840A46A848845C0D2C02F10C02AC
:101FE00000F0D58301311529F6D186E7D5F8E40054
:101FF000A24B90F83A109A7841446429A8BF642112
:1020000021EAE17180F83A10002A40F019842BF09F
:10201000B9FC62E4D5F8E400984B90F83B109A784C
:102020004144FE29A8BFFE2121EAE17180F83B105E
:10203000002AECD0162029F02DFDD5F8E400E6E7C3
:10204000D5F8E40081788D4B4144C829A8BFC82148
:1020500021EAE17181709B78002BD8D0142029F0FF
:1020600019FDD5F8E400D2E7D5F8E4004178834BB8
:102070004144C829A8BFC82121EAE17141709B7879
:10208000002BC4D0132029F005FDD5F8E400BEE7ED
:10209000D5F8E4000178794B4144C829A8BFC8218C
:1020A00021EAE17101709B78002BB0D0122029F059
:1020B000F1FCD5F8E400AAE70698704B81799A788C
:1020C00041446429A8BF642121EAE1718171002A99
:1020D00040F097830D2F0DD00698684B41799A7880
:1020E00041446429A8BF642121EAE1714171002AB9
:1020F00040F0B083D5F8E40089E7D5F8E4005F4B01
:10210000017A9A784144C829A8BFC82121EAE1711F
:102110000172002A3FF47BAF0B2029F0BBFCD5F8FD
:10212000E40074E7D5F8E400544BC1799A7841444F
:10213000C829A8BFC82121EAE171C171002A3FF472
:1021400066AF0A2029F0A6FCD5F8E4005FE7D5F8D1
:10215000E4004A4B81799A784144C829A8BFC82134
:1021600021EAE1718171002A3FF451AF092029F081
:1021700091FCD5F8E4004AE7D5F8E4003F4B4179FB
:102180009A784144C829A8BFC82121EAE171417168
:10219000002A40F03083112F7FF454AF37E7D5F891
:1021A000E400364B01799A784144C829A8BFC82178
:1021B00021EAE1710171002A40F04683102F7FF47B
:1021C00055AF24E7069A2D4B51784144B1F5967FDF
:1021D000A8BF4FF4967121EAE17151709B78002BF2
:1021E00088D0152029F056FCD5F8E4000FE7069AB0
:1021F00017794744642FA8BF642727EAE777177148
:1022000029F062FC1D4B9B78002B3FF473AF032039
:10221000394629F03FFCD5F8E400F8E6069A174B5A
:1022200011784144FA29A8BFFA2121EAE17111701D
:102230009B78002B3FF45EAF012029F02BFCD5F8F2
:10224000E400E4E6069A0D4B917841446429A8BF66
:10225000642121EAE17191709B78002B3FF44AAF31
:10226000022029F017FCD5F8E400D0E6FC28002075
:10227000E43A002080830020B839040878D1002097
:102280000698B24BC1799A78414481F30801C17133
:10229000002A3FF42FAF052029F0FCFBD5F8E4001D
:1022A000B5E6D5F8E400A94BC1789A784144C8292D
:1022B000A8BFC82121EAE171C170002A40F09582CF
:1022C0000F2F7FF4E7AEA2E6119AFFF74DBBA04BAC
:1022D0001B78002B3EF4AEAC9E4BDB78002B7EF4DB
:1022E000A9AC95F8A8300133DBB2032B85F8A830F0
:1022F0007EF6A0AC984B5B7813B9002E7EF49AACB6
:1023000011F0AAFBFFF799BA944B95491A684FF45C
:102310007A73B3FBF2F3C3EB431203EB8203059A28
:102320001268DB001606A1F8A83000F1E3808D4B9F
:1023300003931B68580700F1D480059B1B6803F0CA
:102340000403FEF77DBC3BF912209978B2F5617F5A
:102350004FF4966393FBF1F3C0F2988040F633019B
:102360009142A8BF11460C2FA1F5617191FBF3F8C2
:1023700000F07781182F7FF4B0AA5FFA88F1C8299E
:102380000B46A8BFC823D5F8E400C27DDFB2974250
:102390003FF4A3AA9B1A6D4AC77548BF0733DB10E9
:1023A00092785F1CFFB23AB9002F3FF496AA3846E4
:1023B00021F092FAFFF791BA182029F06BFBF3E7AE
:1023C0006449694BCA681B688B609B1AC82B7FF6EF
:1023D00059AB012381F82130FFF754BB3968DAF893
:1023E0001C200A44CAF8182012E4604B0022012085
:1023F0009EE5F30600F108810B2029F0EDFA002894
:1024000040F0CC80B70600F1548195F8F030002BF5
:102410003FF450ADB8F1000F7EF4BFAEFEF7F4BC50
:10242000534B0122022083E5524A1268970304D5D8
:10243000514A1279002A40F05D81504819461A46E7
:10244000465C0B2E01F10C0107D00132152AF7D1A1
:10245000002285F8A720FFF797B8494ED6F800E08C
:102460005100BEF1000F07D08F1800EB87079EF8D0
:1024700001E07F787745EBD20A44424F424900EBB6
:1024800082020020326038800860E1E70C2F00F003
:10249000C580182F7FF421AA00210B4673E73A6804
:1024A000B9F80630642101FB0323CAF81030FFF7A6
:1024B00086BB4FF003094B465DE54FF004094B46E0
:1024C00059E54FF005094B4655E54FF006094B46D7
:1024D00051E54FF001094B464DE54FF002094B46DF
:1024E00049E5059B294A1B680A21118003F0040372
:1024F000FEF7A6BB264B1B789C077FF518AF254B34
:102500001B78042B7FF613AF25F096FD0FE710F034
:10251000D5FDFEF78FBB059B1F4A1B684FF4C871A2
:102520001180104A039203F00403FEF789BB1BF0ED
:1025300081FDF7F789FE1BF065FDFDF705FD012024
:1025400021F0CAF995F8A620FFF73AB878D1002013
:10255000A97A0020E07A0020E84500205069002098
:102560002C6100206469002050D400200852002013
:1025700052520020E43A002080830020B839040839
:10258000C43900205E3A0020603A0020C0CA002012
:102590006583002068830020C2CA0020B94ABA4B74
:1025A000528993ED007A07EE902AF8EEE77AB0EEC2
:1025B000C77AB4EEE77AF1EE10FA7FF523AF93ED28
:1025C000017AB0EEC77AF4EEC77AF1EE10FA7FF72F
:1025D00019AFB3063FF519AF202021F0ADF9AB4993
:1025E0007A68BB68C5F8E820081FC5F8EC3025F00C
:1025F00099FDA74B01221A7095F8F030002B00F0DE
:10260000F0802688FEF7C9BD102021F07DF9A04B8F
:10261000268883F800804FF00108EDE60027B846D1
:102620009C4B5B78BB423FF458A9384611F0C4FE7E
:10263000994B9B7823B15FFA88F10C2029F02AFA94
:102640000137FFB2B0E6102021F076F9202021F00A
:102650005BF99249081F25F065FD8D4B02221A7027
:10266000CAE75FFA88F7DBE70B464FF6FE718C4A44
:102670008C4854890390908923440144538191816B
:102680001BF0D8FCF7F7E0FD1BF0BCFCFDF75CFC91
:10269000012021F021F9059B1B68002203F00403AF
:1026A00085F8A720FEF7CCBA0B460221DFE702230C
:1026B000DDE7202021F028F9754B00221A709BE7F6
:1026C0004FF6FE73D3E70C2020F0F2FFFEF7B2BA0C
:1026D0000122002185F8AA20724A85F8A9100392E8
:1026E000FEF7AEBA0121002023F0A0FC95F8A62049
:1026F000FEF791BF6C4A1278002A7FF49EAE20F05C
:10270000BBFF049B1B7803F00103A1E60021FF201F
:1027100023F08CFC95F8A620FEF77ABF012023F069
:1027200085FC95F8A620FEF770BF604A137A43F047
:1027300001031372FEF77EBA5C4A137A23F0010399
:102740001372FEF777BA029A115D9847032C1BDCCF
:1027500040F2EE2240F6CA0C00283EF4A6AD39F84D
:1027600024E0BAF802104FF47A73A0EB0E0003FBDA
:1027700000F0A1EB0E0190FBF1F018449042B8BFBD
:1027800010466045A8BF604600B2FEF78EBD484EB9
:1027900037684A003FB1541800EB84047F786478AE
:1027A000BC42BFF4AAAB0A4400EB8202414F424C48
:1027B000326000213B4A398021600392FEF740BA23
:1027C000002E3EF4B9A995F8A5C0BCF1000F3EF467
:1027D000EBA920F051FF94F800C085F8A570FEF732
:1027E000E3B94FF00108FFF765BB0F2029F052F95C
:1027F000D5F8E40064E5112029F04CF9D5F8E4009F
:10280000C9E40D2029F046F964E495F8A610FEF716
:10281000ADBE3BB129492A4A09684FF47A7000FBE2
:102820000313136095F8A530002B3EF4BDA920F0EA
:1028300023FF002385F8A53094F800C0FEF7B4B953
:10284000172029F027F955E4102029F023F9D5F8AD
:10285000E400B3E40E2029F01DF9D5F8E400FFF7F9
:10286000D6BB1149097849B11146FFF7B4BB11F045
:10287000F3F8002385F8A530FEF794B920F0FCFEAC
:10288000FEF7D8B9984A0020A876002098250020A5
:10289000024A0020107B002078D10020484A002006
:1028A000DC44002064690020A676002064510020EA
:1028B000C43900205E3A0020603A002050D4002045
:1028C0007C430020F8B55D4B1B78DB072DD55C4BB6
:1028D0005C4D1C785C4E012C49D079D3022C1BD066
:1028E0006B7A7BB1EB886BB1584B1B7853B106F018
:1028F000E5F900287CD0AB7A83422CBF012300236A
:10290000337000E0337852492A7A9C4238BF1C4623
:102910000C70002A53D1F8BD4E494F4A09881288DD
:102920009142DDD901241C70DAE74A4B4B48454DF2
:102930001988EC78B0F8F230A142A1EB030303F15F
:10294000020223D32B788B4220D33D4B1C78032CDF
:1029500051D03D4E424A1278022A04D13B4F414A9F
:102960003F78D7809480012CA0F8F210B5D13A4A74
:1029700038491288E87A0988121A914235DD3A4AB4
:1029800012888A42ACD200241C70A9E7B1EB440F34
:10299000DBDC2B4B1C78032CDBD0042AD9D82A4E45
:1029A000DFF8A8C0DFF8C0E02B4F0022032434700A
:1029B0001C708CF80020AEF800203A80CAE7012C89
:1029C00036D0022C10D10720BDE8F84020F070BEB0
:1029D000254A20491288E87A0988121A91423FF75D
:1029E0007FAF01241C707BE7F8BD02241C7077E7E1
:1029F0000223337087E7042AABD82A7891FBF2F2DE
:102A00000132082ADFF844E06C78AE78164FA8BF90
:102A100008228EF8002092B216FB02F614FB02F296
:102A20000D4C3E80084E2280002434701C7091E7CB
:102A30000820BDE8F84020F03BBE00BFCC8100205C
:102A4000442A0020808300204A2A0020A676002005
:102A5000A8D1002094760020482A0020AC24002031
:102A60006D75002070750020462A00202DE9F04F7A
:102A7000B74B1E788BB0002E40F08180B54BB64C22
:102A80001D78B64FDFF8FCB205F00105A4F10A0984
:102A900054F80A0CB8B14FF0CC0808FB0698F6F7CA
:102AA000FBFC80B154F80A0CF6F7EEFC14F8023C7B
:102AB000024683B924283BD075B354F80A0CF6F7C4
:102AC000EBFC0028EED10136032E04F1CC04DFD15B
:102AD0000BB0BDE8F08F012B2ED0022B33D0032B8F
:102AE00040D0042B00F06681052B00F05481062BAA
:102AF000E3D114F801ECBEF1000F00F0D581BEF176
:102B0000010F00F01A8201360023032E04F8023C64
:102B100004F1CC04BCD1DBE7232A54F80A0C00F002
:102B20007F818F4B93F832309342B8D1F8F736FC5F
:102B3000012304F8023CC0E74D2800F06481002323
:102B400004F8023CB9E700233C2804F8023C00F0FA
:102B500054813E28B1D10122032304F8012C04F84A
:102B6000023CAAE7C028EAD80021042304F8050C97
:102B700004F8040C04F8061C04F8023C9DE7794BA9
:102B800018680028A4D0F7F775FA774B774D03F54E
:102B90001C7A774B1868F6F77FFC002898D0744BA6
:102BA0001868F6F771FC09281BD03F2819D02B684C
:102BB000002B67D1042800F0B8810C2800F0E480D5
:102BC0007F28E6D0A0F12002D2B25E2AE1D80BB96C
:102BD0002028DED067495A1CC8542A6028F0FAF829
:102BE000D7E72C68002C5AD12646DFF87C8100E01C
:102BF000984608F11003002E08BF46465345F7D308
:102C0000002E6CD03068D8F80020075D135D9F421D
:102C1000204402EB040140F04581564F04F1FF3E91
:102C2000BE4422460BB9FD2A5DD90EF8013F0132A0
:102C30002A6010F8013F11F801CF9C45F2D00AB18B
:102C4000B04512D04C4828F0CDF8B04508D356F81E
:102C5000100B28F0C7F8092028F0BCF84645F6D933
:102C6000464828F0BFF82A680024944291D2444E86
:102C7000264416F8010F28F0ADF82B6801349C4269
:102C8000F7D386E70C287FD00A2833D00D2831D01F
:102C90007F2800F0BC80FF2B3FF67BAF92E7324FDE
:102CA000DFF8D0B04FF0000807F51C79464602E087
:102CB00010374F450DD22246396858462FF074FF21
:102CC0000028F5D1B846002EF2D13E4610374F45C8
:102CD000F1D3002E96D1B8F1000F3FF45AAF264839
:102CE00028F080F8B3E7511C2020B85429607B54A9
:102CF0000A46A5E71F4F28F0E2F8384623212FF0B7
:102D00003DFF002800F00F81C01B286080B1431EEA
:102D1000F95C202940F00F81FA1843B112F8011D27
:102D2000202903F1FF3050D10346002BF6D12B6050
:102D30004FF4807200210F482FF0EBFE044B1B78FC
:102D4000002B3FF4C5AE0D4828F04CF821E700BF3A
:102D5000084D0020CC81002046C50020AC24002076
:102D600090990020043C0020603604087043002045
:102D70006C42002070420020546104085C61040829
:102D80006F420020D02F04087A4828F02BF87A48A8
:102D900028F028F8FDE614F8063C14F8051C9942C2
:102DA00074D814F8043C83427FF4C9AE062304F8B7
:102DB000023C9EE614F8043C04F8030C5A40052338
:102DC00004F8042C04F8023C77E62B606B4C6C4E44
:102DD000002204F51C79FA5402E010344C4551D21B
:102DE000216830460FF064F90028F6D04C4549D2EE
:102DF000E368984700232B609AE7032204F8013C1C
:102E000004F8022C59E6022304F8023C55E6013B83
:102E10005B4A5C482B600021D15427F0E3FFB8E601
:102E2000594B5A49DB785A4ADFF888E11060003381
:102E300018BF01230B70574B574ACEF80030574B41
:102E4000C7F8F8204FF0400E0121C7F8F400C7F88A
:102E5000FC0087F800E1524887F80151197028F00A
:102E60004FFB454827F0BEFF4E4A4F49138891F863
:102E7000321043F08003232913803FF457AE14F837
:102E8000023C34E6494827F0ADFFB3E714F8041CD0
:102E900008EB03005140013304F8041C04F8063C1D
:102EA00082720AE62246CAE69BE80F000DF1280C62
:102EB0000DF1080888E80F004CF824ED14F8053CE3
:102EC00014F803AC0694624623444FF0010C4146CB
:102ED00006A8ADF822E00793ADF820A08DF824C035
:102EE000F9F754F840B1029A314B03924146A4F1EC
:102EF0000A00029306F01EF9DDF80480002304F8AE
:102F0000023CB8F1000F3FF4DEAD54F80A0C06F0B5
:102F10003FFE013654F80A0CC047032E04F1CC04DE
:102F20007FF4B6ADD4E52868F0E615480EF0AAFCAB
:102F30000BB0BDE8F08F034648E714F8053C14F8E1
:102F4000032C0694234407936E2A4FF00003089342
:102F50000993ADF820207FF4D6AD631C06A8069334
:102F6000F7F782FB06A8F7F77FFB06A8F7F77CFBCD
:102F7000C9E500BF646104085C61040860360408A8
:102F8000704200208C610408107B0020C42A0020BD
:102F90006C420020A425002089810008084D0020F3
:102FA00090610408E2830020909900207061040879
:102FB00070D50020043C00202DE9F047B74C636831
:102FC00020469847002800F09F80B54B1B780122CF
:102FD000042B84F8402000F09980B4F91210B4F961
:102FE0001420B4F916306163A263E363AD4B1B8810
:102FF000002B69D0AC4DD4ED0D7AD5ED004A95ED9E
:10300000090A95ED015A95ED0A7AD5ED035A95ED29
:10301000026AF8EEE76AD5ED047AA4EEA60AA5EEF8
:10302000267A67EEC07AA5EEC07AE6EE267A85EDBE
:10303000097AC5ED0A7A2DF05FFCD4ED0E6AD5ED64
:103040000B4A95ED140A95ED0C5A95ED157AD5EDD0
:103050000F7AD5ED0E5A95ED0D6A6063F8EEE66ACB
:10306000A4EEA60AA5EE267A67EEC07AA5EEC07A8F
:10307000E6EE267A85ED147AC5ED157A2DF03CFC46
:10308000D4ED0F6AD5ED164A95ED1F0A95ED175A46
:1030900095ED207AD5ED1A7AD5ED195A95ED186A85
:1030A000A063F8EEE66AA6EEA40AA6EE857A67EEBD
:1030B000C07AA0EE657AE6EE867A85ED1F7AC5EDD8
:1030C000207A2DF019FCE063784EA17E784813F049
:1030D0000DFB3288002A61D1764DD5F84431764A0D
:1030E0001268520720D404F1340007C8B3F9005025
:1030F000401B6063B3F90200091AA163B3F90430FD
:10310000D21AE263BDE8F087BDE8F0876B4BB4F9F3
:103110001200B4F91410B4F91620188060635980B5
:10312000A1639A80E26361E7B5F8AC10322900F040
:103130008980002967D195F8AA20002AD3D0D5F834
:1031400060115F4E5F4886FB0172C917C1EB221107
:103150001980D5F8641186FB0172C917C1EB2211E1
:103160005980D5F86821278A86FB0261D217C2EB05
:103170002112D21B9A800023C0F80A3085F8AA30A9
:103180001AF058FFF7F760F81AF03CFFFCF7DCFE86
:10319000012020F0A1FBD5F84431A4E7454D616B37
:1031A000D5F84431B2F5C87F4FF0000262631A804F
:1031B000308814BFD5F848710027B0F5C87F18BF14
:1031C000D5F84C21A06B39443788C5F848114FF029
:1031D000000E0244B7F5C87FC4F838E0C5F84C21AA
:1031E000A3F802E052D0D4F83CC0D5F85001C4F89E
:1031F0003CE06044012FA3F804E0C5F8500165D01D
:10320000013F37806BE7D5F86061626B0020324484
:10321000C5F8602160631880D5F86461A26BA06373
:103220003244C5F864215880E26BD5F86861E063E8
:1032300032440129C5F86821988073D00139A5F876
:10324000AC1078E71A8820481E4E676BA5F8542109
:103250000022B3F802E0B3F804C0D6F80A60426076
:1032600082606263C5F860711A80A06BC5F8640162
:10327000A2635A80E06BC5F86801E263A5F856E1E5
:10328000A5F858C1C5F85C619A80D7E7E26BC5F82C
:103290005021C4F83CE0A3F804E0B1E79C8300208F
:1032A0006D750020EA440020EC440020C2CA0020D2
:1032B000D0830020AC24002058AA00207075002084
:1032C0001F85EB51DC4400200C260020DFF8108124
:1032D000DFF8FCC0C83188FB01A9C832C917C1EBAF
:1032E000E91188FB02A9D217C2EBE9125A801980B2
:1032F000C83088FB0028218AC217C2EBE812521A94
:103300009A80CCF80AE01AF095FEF6F79DFF1AF0C5
:1033100079FEFCF719FE384620F0DEFA3788D5F83A
:1033200044316DE7274A85F8AE00126885F8A91088
:1033300012F4003203D0244A1279002A35D1104603
:10334000224E375C0C2F00F10C0011D00132152AEF
:10335000F7D1B5F854011E4A1880B5F85671B5F882
:103360005861D5F85C015F809E80C2F80A0065E76D
:10337000184FD7F800C05000BCF1000F09D000EB87
:10338000020E06EB8E0E9CF801C09EF801E0E645A9
:10339000DFD20244DFF84CE00F4806EB8206002241
:1033A0003E60AEF800200260D3E70C4A12780AB102
:1033B0000246C5E720F060F9D5F84431B5F8AC1005
:1033C000C7E700BFE43A002080830020B839040832
:1033D000DC440020C4390020603A0020A67600209A
:1033E0001F85EB515E3A00202DE9F04F2DED028B49
:1033F00091B0054623F028FD814B1F7827B111B00D
:10340000BDEC028BBDE8F08F7E4B1A685205F6D5F5
:103410007D4A1278002A40F098817C4B1B78002B63
:103420006DD07B4C7B4AD4F81C31EB1A934201F2ED
:103430006C8494F82471A7BBDFF80C82D8F80000E4
:10344000F6F72AF8C0B201280ED9022841F0968674
:10345000714B1A78002A42F07580D4F82821AA1AF4
:10346000B2F57A6F82F02A81D4F82C31002B46D045
:1034700094F82431C3B9694B1B689B7801211E3B2A
:1034800000228B4284F8241184F8382142F2BF8054
:10349000D8F800000221043023F0B2FB94F8303158
:1034A00010E0D4F82C3153B3D4F8343140F6B732AD
:1034B000EB1A934223D994F83031002B01F0808528
:1034C000DFF88481013BDBB284F83031002B01F05E
:1034D0005485D4F82C7194F8382117F8011B94F80E
:1034E0003931D8F80000C4F82C710A44013384F84B
:1034F000382184F83931F5F7D3FFC4F8345122F07C
:103500007BFF474B1B786BB1DFF84091D9F8003057
:1035100043B1444B3E4C1B68D4F83C219A1A632AB1
:1035200000F2F681404C2378022B01F03685DFF85B
:10353000208198F80030032B01F00B853B4B1B7862
:1035400073B13B4F3B685BB1314CFCF7DFFFD4F804
:103550004431019044F61F62C31A934200F2BA82CA
:10356000344B1B78002B75D1334B1B7843B1284C5F
:10357000D4F8943203F5C333A0339D4281F086839F
:103580002E4B1B78002B3FF43AAF214E2C4C2D4D87
:1035900006F2B5272068F5F77FFF00283FF42FAF2C
:1035A0002068F5F771FF2B7880465A1E33B12068EA
:1035B0002A70F5F771FF0028F2D120E7032239467F
:1035C000781E2FF08CFA96F8B43296F8B52286F869
:1035D000B78283F47F4383F0FF039B1A1FFA88F8B6
:1035E0009BB2B8EB132FD5D196F8B622DBB29A4234
:1035F000D0D1781E19F000FD2B7818442870C9E747
:10360000084D002058AA00204C8400205684002039
:10361000182600203F0D03002D000020F483002019
:103620006084002050D4002092780020688400201C
:103630006C840020008500200E850020728400200C
:10364000788400207C840020F0830020B87600205D
:103650009D1C00209D4C2278002A41F00E839C4C3A
:10366000D4F88C3203F5C333A0339D42FFF47CAF12
:10367000984A94F89032C4F88C52D75CFA0701F15A
:10368000E585BB0701F1A085780701F12C863A0793
:103690004FD5914BDFF86C82099310AA1146A3F124
:1036A000210241F8202D0020A3F124020E4603F848
:1036B000240C029102231121517093703046D8F8E6
:1036C0000410F6F7E7FF3046D8F80810F6F7E2FFE7
:1036D000B8F81230814903EBC3039B00053381FB2B
:1036E0000321DB17C3EBA101304689B2F6F7EAFFED
:1036F000B8F8143003EB8303590089B23046F6F76B
:10370000E1FF774B029E1B789B0743BFB8F80C1074
:1037100001F57A7189B24FF47A713046F6F7D2FF2B
:10372000089B98F80020591C089130461A7023F025
:1037300049FB6C4A94F890321178013393FBF1F213
:1037400001FB123384F890320EE7614C664BD4F8DB
:10375000102119688A1A7C2A7FF65FAE94F814212A
:10376000DFF8A4919FED618AC4F81011013284F84A
:103770001421A9F1340A4FF02408404623F0B8FA86
:10378000BAF81030F9EC016A07EE103AF8EEE66A82
:10379000B8EEC77A08F10108C6EE877A5FFA88F8B2
:1037A00067EE887AFDEEE77ACDED017ABDF904B0D7
:1037B0005FFA8BF023F072FACBF3072023F06EFA56
:1037C000B8F1270FD9D1302023F092FA484ADFF818
:1037D0003C91D2F800805FFA88F023F05FFAC8F3DA
:1037E000072023F05BFAD9F800005E21F5F758FEB8
:1037F00094F8142193072DD1D4F8101141F2883296
:10380000914201F22C87142023F072FA394A33498D
:10381000B2F9042081FB02314FEAE278C8EBA1083B
:103820000FFA88F85FFA88F023F038FAC8F3072017
:1038300023F034FA1C2023F05BFA002023F02EFA48
:10384000002023F02BFA5E21D9F80000F5F728FEBE
:1038500094F8142112F0070801F0A685282A7FF4B5
:10386000DCAD214B4FF0000817201F6884F814814D
:1038700023F03EFA404623F011FA1F4B1F4CA3FBE6
:1038800007239B0BA4FB03125209C2EB0212A3EB0A
:103890008203D8B223F002FA182023F029FA184B39
:1038A000A3FB07239B09A4FB03125209C2EB0212DC
:1038B000A3EB8203D8B223F0F1F9404623F0EEF9EE
:1038C000D9F800005E21F5F7EBFDA6E54484002061
:1038D0001826002008850020208400206766666680
:1038E000658300200D85002050D4002000007A441C
:1038F000908300209483002073B2E74589888888EC
:10390000D34D621068830020D0830020F88300200C
:10391000DFF8B0810193412019F048FC644FB8F9F9
:103920000220DFF8A4B187FB0230D217C2EBA0005F
:1039300080B219F01FFCB8F9002087FB0230D217C3
:10394000C2EBA00080B219F015FCB8F9042087FB87
:103950000230D217C2EBA00080B219F00BFC9BF82A
:103960000010D9F80000F5F79BFD94F84071019B19
:1039700017F0010801F07D83DFF844A1DAF8002098
:10398000910640F185804B4ADFF84081127892071A
:1039900041F13A8698F80020042A8CBF03270227B9
:1039A0004720029319F002FCD8F8040019F0AEFB8E
:1039B000D8F8080019F0AAFBB8F812203E49D9F847
:1039C0000000A1FB0232C2F3471211460192F5F743
:1039D00067FD9BF80000DAF80010019A029B424054
:1039E00011F0140F8BF8002041F0A885B8F80C20D6
:1039F000642000FB02F0019319F088FB98F8002086
:103A0000D9F8000047EA8207FFB23946F5F748FDCA
:103A10009BF80020D9F80000574039468BF8007019
:103A2000F5F73EFD94F84071019B8FBBDFF8A08055
:103A300001934F2019F0BAFBD8F8000019F066FB8B
:103A4000D8F8040019F062FB384619F05FFB012139
:103A5000D9F80000F5F724FD16499BF800200F78EF
:103A6000D9F8000007F00107394682F001028BF80F
:103A70000020F5F715FD9BF80020D9F8000057400D
:103A800039468BF80070F5F70BFD94F84071019BF7
:103A90000A4AC4F83C317B1CDBB2A2FB0312D208F9
:103AA00002EB8202A3EB420384F840313AE500BF07
:103AB00067666666658300201F85EB51CDCCCCCC54
:103AC0006469002094830020BC7600206883002075
:103AD000444A002094F84A31002B41F03383E84BEC
:103AE0001B6803F00802002A48F603414AF60B401F
:103AF0004BF60F4249F6074804BF0246884613F0CA
:103B0000040F4FF0190118BF90469B0684F84A1124
:103B100003D548F4804848F02008DA4B1A79C8F3F6
:103B2000090B002A41F0FE855B79002B41F08C8760
:103B3000994664204FF0FF334FF0000ACDF8208003
:103B4000CDF82480CDF828B0ADF82E90ADF8303007
:103B50008DF83E00ADF82CA0CDF832A0CDF836A0FF
:103B6000CDF83AA00DF1200EBEE80F00DFF824C317
:103B700084F805A0ACE80F009EE80F00ACE8070051
:103B80002CF8023B61464FF001081B0C4FF0FE0E73
:103B90001F20C82201F81E3984F802E0A27184F8BF
:103BA0000780E07094F85A01207180F0F10383EAF5
:103BB0000313DAB2130983F0E70343EA022383EA2B
:103BC000C2031BB283EA0312D2B2C3F3072383EA10
:103BD000121343EA022383EAC2031BB283F0C80232
:103BE00082EA0212D2B2C3F3072383EA121343EA32
:103BF000022383EAC2031BB283EA080E8EEA0E1E7A
:103C00005FFA8EFEC3F3072282EA1E1242EA0E22F8
:103C100000EB080382EACE0E0CEB080084F85A3160
:103C2000A4F800E011F8013B83EA0E0383EA0313D2
:103C3000DBB21A0982EA1E2242EA032282EAC303A5
:103C40001BB21FFA83FE8142A4F800E0EAD183F0A0
:103C50007C0383EA0313DBB24FEA131C8CEA1E2CAD
:103C60008CEA032C8CEAC30C0FFA8CFC1FFA8CFA3A
:103C7000DFF82492A4F800A05FFA8CFC4FEA1A2A1D
:103C800084F828A084F827C009F5C17B04F1220834
:103C9000D9F80000D9F80410D9F80820D9F80C3068
:103CA000DE46AEE80F0009F11009C145F346EFD139
:103CB000D9F80000CEF80000DFF8E08199F8043070
:103CC0008EF8043008F1270984F8A9C184F8AAA164
:103CD00018F8011F3868F5F7E3FBC145F8D194F8EF
:103CE0004B21002A41F078816749684B08781B68AE
:103CF0000A2184F84B11002801F05182DFF8A0C19D
:103D00000128BCF80010039141F296860228BCF805
:103D1000029001F04B85BCF804100291032801F0D9
:103D2000A3860428BCF806B001F099860528BCF8E3
:103D300008E001F090860628BCF80A8001F066864B
:103D40000728BCF80C1001D0BCF80E2094F85A01DA
:103D50000893064686F0300383EA0313DBB24FEA8A
:103D6000131C4B4804968CF07A0C4CEA032C008808
:103D700026718CEAC303DFF82CC1C0EB00208CFB5A
:103D800000AC8444C0171BB2C0EB6C200646C3F3E2
:103D9000072C83EA0310039B8DF83560C0B24FF007
:103DA000000A63F30F0A8CEA101303934FF0000C20
:103DB000029B69F31F4A6EF30F0C4FF000094FF09E
:103DC000000E63F30F0961F30F0E039BCDF824A0DF
:103DD00068F31F4C62F31F4E4FF000086BF31F494E
:103DE000CDF82890CDF82CC0CDF830E08DF8348097
:103DF00043EA00230DF1200983EAC00EB9E80F0061
:103E00000FFA8EFE8EF0C80A8AEA0A1ADFF884C01A
:103E100084F805805FFA8AFACEF3072EACE80F002B
:103E20008EEA1A1E4EEA0A2399E8030083EACA03BF
:103E30001BB283F0230E4CF8040B8EEA0E1E5FFAC1
:103E40008EFEC3F3072282EA1E12049B604642EAFA
:103E50000E2203F1010882EACE0E20F814194FF069
:103E60002309FE211622C82384F85A81A4F800E011
:103E700084F807900CF1020CA170E27014E000BF0E
:103E800064690020808300209085002050D40020A9
:103E900098D10020202600201A2600209B270020F1
:103EA00054C9002003082080A37110F8013B83EA65
:103EB0000E0383EA0313DBB21A0982EA1E2242EAE6
:103EC000032282EAC3031BB21FFA83FE6045A4F8F3
:103ED00000E0EAD183F0F40383EA0313DBB21A09AA
:103EE00082EA1E2282EA032282EAC3031BB21FFA7D
:103EF00083FEDFF80C84A4F800E05FFA83FC4FEA4D
:103F00001E2A84F81EC084F81FA0D8F80410D8F820
:103F10000820D8F80000D8F80C3008F5C17EAEE8CB
:103F20000F00D8F81000D8F81410D8F8182004F2B0
:103F3000A119AEE8070004F2831884F8A1A184F85F
:103F4000A0C118F8011F3868F5F7AAFAC145F8D1E1
:103F500094F84E31002B41F0FA80DFF8B0A3DAF884
:103F600000301922980684F84E2140F12083E34B5B
:103F7000DFF89C831B78990741F1D08398F80030D3
:103F8000042B8CBF4FF003094FF00209FCF7BEFA77
:103F9000B8F81430B8F80C20089003EB83035B00EA
:103FA000ADF83A304FF47A70D8F804300A93B8F884
:103FB000121098F800E0D8F808308DF83C9000FB1B
:103FC00002F24FF0000C4FF0FF3008AE8DF83DE0EC
:103FD000CDF824C00C920B93ADF838100D90B1467B
:103FE000B9E80F00DFF82CE30296AEE80F0099E87D
:103FF0000F00AEE807007246182122F81C39E17163
:1040000094F85A1184F805C081F0780383EA031309
:10401000D8B2030983F0F60343EA002383EAC0031E
:104020001BB283EA0310C0B2C3F3072383EA101361
:1040300043EA002383EAC0031BB283F0C80080EA8E
:10404000001C5FFA8CFCC3F3072080EA1C1040EAD6
:104050000C2080EACC0000B280F0180383EA03133E
:10406000DBB2C0F3072080EA131040EA032080EAA5
:10407000C30301F101091E204FF0FE0C4FF0C80BE5
:10408000E0700EF1020E217184F85A91238084F8B9
:1040900002C084F806B0184612F8011B414081EABC
:1040A0000111C9B20B0983EA102343EA012383EA11
:1040B000C10109B288B272452080EDD181F01801AA
:1040C00081EA0111C9B20A0982EA102383EA0123B5
:1040D00083EAC1031BB29AB289492280DBB2120A79
:1040E000039104921E4684F8272084F826308E46D9
:1040F00001F5C17B04F12209DEF80000DEF80410AE
:10410000DEF80820DEF80C30DC46ACE80F000EF1DB
:10411000100ECE45E346EFD1DEF80000CCF80000EB
:10412000DFF8F4919DF8103084F8A86184F8A93183
:10413000CB461BF8011F3868F5F7B2F9714B5B45A8
:10414000F7D1FCF7E3F9DAF80030B8F80C20D8F82A
:1041500004A0D8F808804FF47A7113F0140F01FB13
:1041600002F141F05D828E4694F85AB108908BF0CE
:104170006A00654BDFF8A4C1B3F90420CDF824A090
:1041800080EA0010C0B2030983F0D50343EA00239C
:1041900083EAC0031BB283EA0310C0B2C3F3072350
:1041A00083EA101343EA002383EAC0031BB28CFBAB
:1041B000020CD2174FF0000ACDF82880C2EBAC02F7
:1041C000DDF80880CDF830E083F0C80C0B91ADF835
:1041D0003A20ADF834A0ADF836A0ADF838A08CEA9E
:1041E0000C1C5FFA8CFCC3F3072EB8E80F008EEAB4
:1041F0001C1E4EEA0C2E8EEACC0CDFF818E184F877
:1042000004B00FFA8CFCAEE80F008CF0210398E8A4
:10421000070083EA0313DBB2CCF3072C8CEA131CF0
:104220004CEA03280BF1010C8EE8070088EAC3036F
:1042300084F85AC14FF0210B4FF0FE084FF01C0CD0
:10424000C8220EF10C0E84F805A084F807B084F89B
:10425000028084F803C0AEF11C01A27118462380CD
:1042600011F8012B424082EA0212D2B2130983EA0A
:10427000102343EA022383EAC20212B290B27145CC
:104280002080EDD182F0680282EA0212D2B24FEAB7
:10429000121B8BEA102B8BEA022B8BEAC20B0FFA54
:1042A0008BFB1FFA8BF3DFF858E023805FFA8BFB60
:1042B0001B0A1E4684F8253084F824B00EF5C17A16
:1042C00004F12208DEF80000DEF80410DEF8082011
:1042D000DEF80C30D446ACE80F000EF1100EC645E7
:1042E000E246EFD1BEF80030DFF83480ACF80030A1
:1042F000CA4684F8A6B184F8A76113E0658300205C
:104300001A260020C1270020948300206469002021
:1043100068830020202600209B27002067666666B1
:10432000BF2700201AF8011F3868F5F7B9F8D04503
:10433000F8D194F85AA1E14AE14E84F804A08AF039
:10434000EB0383EA0313D9B20B0983F0C50343EAF5
:10435000012383EAC1031BB283EA0310C0B2C3F393
:10436000072181EA101141EA002181EAC0010CCA4B
:1043700009B281F0C80E8EEA0E1E5FFA8EFE4FF073
:10438000000C0892C1F30721029A0993CDF828C0C6
:1043900081EA1E1343EA0E2307CA83EACE031BB247
:1043A00083F0310E86E807008EEA0E1E5FFA8EFE5D
:1043B000C3F3072383EA1E1343EA0E2383EACE03E3
:1043C00094F808E0607AA27AE17A84F805C01BB21A
:1043D0008EEA030E8EEA0E1E5FFA8EFEC3F30723EB
:1043E00083EA1E1343EA0E2383EACE031BB258402E
:1043F00080EA0010C0B2C3F3072383EA101343EA34
:10440000002383EAC0031BB25A4082EA0210C0B202
:10441000C3F3072282EA101242EA002282EAC002B3
:1044200012B2514081EA0111C9B2C2F3072383EAF3
:10443000111343EA012383EAC10394F80CC094F8F2
:104440000DE0A07BE17B227C94F811801BB28CEA0A
:10445000030C8CEA0C1C5FFA8CFCC3F3072383EA81
:104460001C1343EA0C2383EACC031BB28EEA030E2F
:104470008EEA0E1E5FFA8EFEC3F3072383EA1E1335
:1044800043EA0E2383EACE031BB2584080EA0010B1
:10449000C0B2C3F3072383EA101343EA002383EA7D
:1044A000C0031BB2594081EA0111C9B2C3F307230B
:1044B00083EA111343EA012383EAC1031BB25A4082
:1044C00082EA0212D2B2C3F3072383EA121343EA49
:1044D000022383EAC2031BB288EA030888EA0818A9
:1044E0005FFA88F8C3F3072383EA181343EA082323
:1044F00083EAC803A17CE27C1BB2594081EA011126
:10450000C9B2C3F3072383EA111343EA012383EA01
:10451000C1031BB25A4082EA0212D2B2C3F307238C
:1045200083EA121343EA022383EAC2031BB283F035
:10453000270E8EEA0E12D2B2C3F3072E8EEA121E97
:104540004EEA022E8EEAC20E0AF101030FFA8EFE27
:104550001FFA8EF24FF0310AFE200C2184F85A31F6
:10456000C8234FEA122C06F5BE785FFA8EFE228031
:1045700084F807A0A070E170A371039E84F814E092
:1045800084F815C07168B268F3683068B6F810A096
:10459000A8E80F0028F803AB84F897C184F896E1E7
:1045A00019F8011F3868F4F77BFFC845F8D194F873
:1045B00052C1BCF1000F40F05685424B94F85A911D
:1045C000B3F90010B3F90220B3F904309FED3E6A4D
:1045D00084F805C007EE103A3C4B1B68089389F03D
:1045E0006A0383EA031306EE901AD9B20B0983F02B
:1045F000D50343EA012383EAC1031BB283EA031113
:104600005242C9B207EE902AC3F3072383EA11137B
:1046100043EA0123F8EEE77AF8EEE66AB8EEC77AE5
:1046200083EAC1031BB267EE867A66EE866A27EEDE
:10463000067A002083F0C808CDED0A7ACDED096A2C
:104640008DED0B7A0C900D900E9088EA081E0DF1FE
:10465000200A5FFA8EFEC3F30728BAE80F0088EA43
:104660001E1848EA0E2888EACE08DFF854E00FFA50
:1046700088F8AEE80F0088F01E0C9AE807008CEA74
:104680000C1C5FFA8CFCC8F3072383EA1C1343EA73
:104690000C238EE8070083EACC0CC8214FF0050AF2
:1046A0004FF01E08FE231C2009F10102A17184F8BD
:1046B00052A184F80780A370E07009E0444A00200A
:1046C000202600209483002088C3E43A50D40020A0
:1046D000AEF1100184F804900EF10C0EA4F800C0A5
:1046E00084F85A2111F8013B83EA0C0383EA03138F
:1046F000DBB21A0982EA1C2242EA032282EAC303DD
:104700001BB21FFA83FC7145A4F800C0EAD183F004
:10471000270383EA0313DBB21A0982EA1C2C8CEA12
:10472000032C8CEAC30C0FFA8CFC1FFA8CFADFF80E
:104730001094A4F800A05FFA8CFC4FEA1A2A84F8BF
:1047400025A084F824C009F5C17B04F12208D9F81A
:104750000000D9F80410D9F80820D9F80C30DE464A
:10476000AEE80F0009F11009C145F346EFD1DFF8BB
:10477000E483B9F80030AEF8003008F1240984F879
:10478000A6C184F8A7A118F8011F3868F4F788FEBD
:10479000C145F8D194F853A1BAF1000F40F05E84FE
:1047A000E04B1B68052284F853219A0640F10185ED
:1047B000DD4ADFEDDE7A518A07EE101AB8EEC77ACD
:1047C00013F0140F27EE277A01F0E380D84BDFEDCA
:1047D000D76AD3ED007AF8EEE77A67EEA67A94F816
:1047E0005A91D44BD44AB3F90410B2F90620DFF839
:1047F00068E3D2488DED097A89F0220383EA031336
:104800005FFA83FC4FEA1C1383F0590343EA0C233D
:1048100083EACC03B2F5FA6F1BB2A8BF4FF4FA6279
:1048200083EA031C5FFA8CFCB2F57A7FC3F307239B
:1048300083EA1C13B8BF4FF47A724FF0640843EA5E
:104840000C23A2F57A7208FB02F283EACC0C8EFBF1
:10485000026E80FB01600FFA8CFCC917D217C2EB05
:10486000AE12C1EBA0034FF0000B08A98CF0C80EEC
:10487000CDED0A7AADF83220ADF83030CDF820B069
:10488000CDF82CB088468EEA0E1E5FFA8EFE02919D
:10489000CCF3072CB8E80F008CEA1E1C4CEA0E2C57
:1048A0008CEACE0EDFF8B4C2D8F8008084F8049009
:1048B000ACE80F000FFA8EFE8EF04A0383EA031372
:1048C000DBB2CEF3072181EA1311624641EA0321EC
:1048D00009F1010981EAC303142042F810894FF05D
:1048E000FE0E4FF04A08002184F85A914FF0C80993
:1048F000E07023800CF1040C84F8078084F802E057
:10490000617184F80690184612F8011B414081EA53
:104910000111C9B20B0983EA102343EA012383EA98
:10492000C10109B288B262452080EDD181F0140145
:1049300081EA0111C9B24FEA111E8EEA102E8EEAE9
:10494000012E8EEAC10E7E4B0FFA8EFE1FFA8EFCF0
:104950001E464FEA1C2B5FFA8EFE84F81DB084F8C9
:104960001CE059689A683068DB68A4F800C006F556
:10497000C17CACE80F0030697169B6F818900396F5
:10498000ACE8030004F28318ACF8009084F89FB1FF
:10499000C14684F89EE104F29F1B19F8011F386894
:1049A000F4F77EFDCB45F8D1664B674A1B78127849
:1049B000013B12F00100DBB214BFC0214021172BD4
:1049C00003D8624A134493F808A0614B1A889607EB
:1049D0001ABF002341F01001012312F4027F18BF17
:1049E000022312F0100F18BF062312F0200F18BF79
:1049F0001023002840F029864FF0030994F85AE16B
:104A000008938EF0460383EA0313DAB2130983F0A6
:104A1000920343EA022383EAC2031BB283EA031030
:104A2000C0B2C3F3072282EA101242EA002282EAED
:104A3000C00212B282F0C80C8CEA0C1C5FFA8CFC2B
:104A4000C2F3072282EA1C1200238DF8279003206C
:104A500042EA0C29029A8DF824A08DF825308DF8B1
:104A600026108DF8280007CA89EACC0C0FFA8CFCB6
:104A7000DFF8E890E3718CEA0C1AA9E803005FFA0A
:104A80008AFACCF3072C8CEA1A1C4CEA0A2181EA38
:104A9000CA0A94F808C089F800200FFA8AFA8CEA4A
:104AA0000A0C8CEA0C1C5FFA8CFCCAF3072282EA1F
:104AB0001C1242EA0C22607AA17A94F80BA063716E
:104AC00082EACC0212B2504080EA001C5FFA8CFCF1
:104AD000C2F3072080EA1C1040EA0C2080EACC00D8
:104AE00000B2414081EA0111C9B2C0F3072282EA53
:104AF000111242EA012282EAC10212B28AEA020AD1
:104B00008AEA0A1A5FFA8AFAC2F3072282EA1A12BA
:104B100042EA0A2294F80CC0607BA17B84F804E08E
:104B20001EE000BF64690020688300200AD7233C90
:104B30008C8300209483002054C900206766666639
:104B40001A26002078460020CC810020E02F04089F
:104B5000E48300209B270020D34D621020260020F4
:104B600082EACA0212B28CEA020C8CEA0C1C5FFACE
:104B70008CFCC2F3072282EA1C1242EA0C2282EA6F
:104B8000CC0212B2504080EA0010C0B2C2F3072239
:104B900082EA101242EA002282EAC00212B25140B6
:104BA00081EA0111C9B2C2F3072282EA111242EA74
:104BB000012282EAC102E17B94F810A013B281EADB
:104BC000030282EA0212D2B2C3F3072383EA12136A
:104BD00043EA022383EAC2031BB28AEA030282EA9F
:104BE0000212D2B2C3F3072383EA121343EA022369
:104BF00083EAC2031BB283F0320282EA0212D2B20B
:104C0000C3F3072383EA121343EA022383EAC203AE
:104C10001BB29AB24FF0FE0C0920C8210EF1010E12
:104C2000DBB284F802C04FEA122CE070A17184F864
:104C30005AE1228084F812C06374039E3068716860
:104C4000B268B6F80CB009F5BA7EAEE8070009F50F
:104C5000C2798EF802A0AEF800B084F894C184F84E
:104C6000933118F8011F3868F4F71AFCC145F8D1E0
:104C7000019BC4F84431FEF773BCDA4BDA4918687B
:104C8000F4F7D6FB00232370FEF7E9BC94F89832C2
:104C9000D64AC4F8945202EB8302126A42B310ADB2
:104CA00004F29F23D24E45F8203D002104F2B123A7
:104CB0003180099380211523A52784F89E32284648
:104CC00084F89D1284F89C72904728463188F5F745
:104CD0001FFD089DC74804F527716D1A152DA8BF43
:104CE00015252A462BF0FEFBC34A94F8983215701E
:104CF000C24A013382FB0312A2EBE37202EB4202CF
:104D00009B1A84F89832FEF73BBCDFF828E3BC4AD4
:104D1000BC4BD4F82011DEF800001B8892F80BC0C1
:104D2000B94A401A4FF47A71DFB201FB0CF11B0A49
:104D30009777177588424FF00007D37753759770B0
:104D4000177180F00C82B14BB14E1B68B149DFF88E
:104D5000E89208688968DFF8E4E2DFF8E482DEF8C8
:104D600000E086FB036CDB17C3EB6C1303F5FA73EF
:104D70009BB293761B0AD37689FB003AC01789FB56
:104D80000139CB17C0EBAA0111770912DFF8B4C2C1
:104D900051779F499CF800C0C3EBA9030EF5EA4088
:104DA00081FB0E1982F820304FEAEE711B12C1EB25
:104DB0006911303082F82130974B98F8009083F8D1
:104DC0001A90001278310EF1300E1CF0020F82F8AA
:104DD000230082F8241082F822E000F0BD81D8F888
:104DE00004C08E49D8F808A0DFF85CB28C4A81FB79
:104DF0000C604FEAEC7E81FB0A61CEEBA05E4FEACD
:104E0000EA70C0EBA1510BFB0EC00BFB01AB0BEB2F
:104E10004B0B4FEA4B0600EB40000196400082FB33
:104E2000007B01EB810182FB0672019E92140EEB66
:104E30008E0E01EB81014FEAAB4B04920EEB8E0715
:104E4000B8F8122005914FEAE67EC117B8F80C8039
:104E5000744E03974FEADC7C83F809C0ABEB010C7E
:104E600006FB1C0108F5FA78049E03981FFA88F7E0
:104E70000297A6EB0E086B4F019EDFF8D0E1B9F167
:104E8000050F4FFA8CF909EB8009404607FB1868BB
:104E9000059EDFF8BCC140B200EB860002EBC20207
:104EA0005B4E4FEA82024FEADA7A8CFB02BC83F84F
:104EB0000EA086FB017A86FB08B74FEAE27B9DF8DD
:104EC00008205A75CBEBAC120192029ABEF8006032
:104ED000DFF880E14FEAE8784FEAE1711FFA89F9DB
:104EE00080B2C8EB6717C1EB6A114FEA1228019A2A
:104EF00083F80A904FEA102B4FEA192C4FEA212A27
:104F00004FEA272983F810B0BEF800E083F80BC001
:104F1000D873C2F3072C4FEA162034BF4FF0320B80
:104F20004FF0330B197383F80DA05F7483F8129060
:104F300083F816809DF80420DA7183F808C0DE74C7
:104F4000187583F81BB083F81CE0C4F81C51FEF7F9
:104F500070BA354F386803685B69984700283EF49B
:104F6000EDAA3868036801219B6998470222002353
:104F700088F800202370FEF7E1BA94F8381194F80D
:104F80003931D8F800004A1C013384F8382184F8FC
:104F90003931F4F785FAFEF7B0BAFBF7B7FA234BCD
:104FA0001A6840F6B833801A984200F2EE80204F1B
:104FB0003B793A2B00F0CB8200232370FEF7BEBA78
:104FC000C4F82C3184F82431DFF88C8021F04CFEB9
:104FD00094F83031FEF776BA013A84F84B21FEF7A7
:104FE000B7BF00BF0485002020840020E02F040804
:104FF000D08100204C440020614400205655555576
:105000009876002094760020808400208C830020F5
:105010001F85EB51D4810020AC8400206BCA5F6BEC
:1050200083DE1B4340420F00307900209878002037
:105030008078002050D40020676666669083002048
:105040006883002065830020806967FF9CD1002071
:10505000D34D62100E7B0020F08300200AF1FF3A4E
:1050600084F853A104E60CF1FF3C84F852C1FFF729
:1050700091BBB94A1288D70515D4D00600F1D88261
:10508000910600F19A83570600F18A84100700F117
:105090008B84D10700F1AE8412F0020F0CBF4FF0E9
:1050A00004084FF00C08AD49AD4A0F78D27807F0EC
:1050B00001070AB147F002075320019318F076F870
:1050C000A84A128802EB820202EB8202900080B2B0
:1050D00018F050F8002018F04DF8A34AA3491288A0
:1050E000D9F80000C2EBC212520081FB0231114418
:1050F000D217C2EB61225FFA82FA5146F4F7D0F977
:105100009BF80020D9F800008AEA020248EA070763
:1051100000218BF80020F4F7C3F93946D9F80000D4
:10512000F4F7BEF99BF80020D9F800007A40D2B21B
:1051300011468BF80020F4F7B3F994F84071019B05
:10514000FEF773BC013B84F84A31FEF7C8BD013B52
:1051500084F84E31FFF72BBA2D22DA76F5E6844B30
:10516000DEF800101B78C4F82011013B012B3FF63C
:10517000EAAD1021022391701371E4E521F064FD82
:105180007C4B01221A70FEF76FB97B4AB2F84231AC
:1051900000210133A2F842312170FEF7CFB9014658
:1051A0008046864683460290814603900246FEF77B
:1051B000CDBD9FED727A13F0140F08BFF0EE477A61
:1051C0007FF404ABFFF70BBB6D4B664909930DF100
:1051D0004008A3F1210048F8200D4FF0080E4FF0D1
:1051E00000090A2003F822EC03F8230C03F8249C9E
:1051F00040460988F5F766FA624B63491B6881FBF4
:105200000321DB17C3EBA101404689B2F5F75AFA37
:105210005E4BB3F806A003F051FD089B5A1C0892A0
:1052200083F80090089B4FEA1A22591C08911A70C3
:10523000089B5A1C089283F800A0089B5A1C0892ED
:105240001870404621F0BEFDFEF71EBADFF85091FF
:105250009FED4F8AB9F90230494A099207EE903A18
:10526000F8EEE77A0DF1400867EE887AA2F12403A0
:10527000FDEEE77AA2F12101002048F8201D02F896
:10528000240C0822CDED017A5A701E229A70BDF8C6
:1052900004104046F5F716FAB9F9003007EE903AD7
:1052A000F8EEE77A404667EE887AFDEEE77ACDEDD4
:1052B000017ABDF80410F5F705FAB9F9043007EEE4
:1052C000903AF8EEE77A404667EE887AFDEEE77AA4
:1052D000CDED017ABDF80410F5F7F4F9404621F060
:1052E00071FDFEF7CEB92B4A254B12680993A3F145
:1052F0002408002103F8241C2123D10088F802305F
:1053000040F1008224490326134B1B885A0500F103
:10531000F681D80700F1F58203F002031F4A002B43
:105320001CBF03261146DFF87C90324648462BF01E
:10533000D9F806EB090310A80133A9F1020140F8DE
:10534000203D00225B1A06F8092088F8013021F080
:1053500039FDFEF79CB900BFE4830020CC8100201A
:10536000E07A00209476002098D100200308208065
:10537000A8D100202D0000201826002000000000E9
:1053800020840020D4810020676666668083002028
:1053900058A08B41ACD10020D0610408E061040822
:1053A00094830020FF830020022021F0A1FCFF2035
:1053B00017F0A8FD0278FF2A00F0E98290F90100B9
:1053C0004FEAE0785FFA88F8C0B221F067FC404607
:1053D00021F064FC032021F08BFCFF2017F092FDEC
:1053E0000278FF2A00F0CF82B0F908805FFA88F0D7
:1053F000C8F30728DFF898A321F050FC404621F0BD
:105400004DFC9AF80420002A40F0E781D14A126846
:10541000900640F11081DFF87CA3DFF87C839AF8D6
:105420000020910700F170824FF0000B012021F065
:105430005FFC384621F032FC584621F02FFC092051
:1054400021F056FC002021F029FC002021F026FC50
:10545000B8F8161098F80030B1F5967F0AD994F88C
:10546000142102F00F02072A04D842F20F738B4274
:1054700028BF0B46DFF824B30193052021F038FC48
:105480009BF80820019B002A00F0A482203B07EE35
:10549000903A9FEDB17AF8EEE77AF6EE006A67EEA1
:1054A000877ABEEE007AF5EEC07AF1EE10FA58BFB8
:1054B000B0EE667A77EE877AFDEEE77ACDED017A87
:1054C000BDF904300193D8B221F0E8FB019BC3F38E
:1054D000072021F0E3FB9AF80020002306930793AE
:1054E000930700F16D8194F81831012B00F0688169
:1054F000BBF90030DFED996A07EE103ABBF90230D4
:1055000007EE903AB8EEC77AF8EEE77A27EE267AF9
:1055100067EEA67ABDEEC77AFDEEE77A08A88DEDB4
:10552000087ACDED097A21F0F5FB5E21D9F800006B
:10553000F3F7B6FF94F81421FEF790B9884A106883
:10554000FEF759BAC4F828511F70FDF78DBFBB781C
:10555000DBB103F1FF3C5FFA8CFC0CF1010CBC44A5
:10556000BE4600221EF8013B534083EA0313DBB220
:10557000120AD90042EA0322F44581EA131382EAAF
:105580000302EFD1002A7FF417AD764BDFF810E26B
:105590001968734BD1F830C01B68734ADFF8EC818F
:1055A000CEF83830714BB8F80080CEF86800B3F808
:1055B000423110689268CEF81880CEF82800CEF8F4
:1055C0004820CEF85830BCF1000F00F01782DCF80C
:1055D0000430886C83423BBFCA681B1A1B1A9B1895
:1055E000002B7DF4A4AF0B68DFF8B8819B690846F7
:1055F000022198470423F87888F8003019F0D8F889
:1056000003232370FDF795BF0127FEF7C9B90221D7
:10561000D8F80000F3F72CFF94F83031FDF752BFB3
:105620004F4B1B6803EB83034FEA430EFEF79CBD11
:105630004FF0340837E54E4B93E8030008AB83E89E
:105640000300184621F066FB6FE74A4AD278002A29
:105650000CBF4FF004094FF00509FFF7CFB9DFF891
:1056600000B1DFF844A1102021F042FBDBF800205C
:105670008AFB0238D217C2EB68185FFA88F021F073
:105680000DFBC8F3072021F009FB212021F030FB9E
:10569000DBF800108AFB013ACA17C2EB6A126420D9
:1056A00000FB1212002AD8BF524212B2D0B221F02F
:1056B000F5FA002021F0F2FAFEF7A5B80122D8F899
:1056C00000001A70F3F7E0FE0746D8F80000F3F781
:1056D000DBFE7F067DF4C8AE8A2800F069818E2843
:1056E0007DF4C2AE94F82431002B7DF4DAAE224B67
:1056F000C4F82C312D2384F83031FDF7BCBE0326CD
:105700001E4910E61E4B1F4A1B681F4903F4800305
:10571000002B16BF114604260326F5E54FF00109BC
:10572000FEF734BC19495A790B8803EB830303EB6A
:1057300083034FEA83091FFA89F9002A00F09A814E
:10574000094B1B681BB2029303F0B8FA029B40B2EC
:10575000FEF7F2B964690020E4380E3F0050C347F9
:105760008C83002030790020D4810020182600206E
:10577000E02F0408E07A002080840020D46104082F
:1057800058AA0020D0610408C8610408947600205B
:1057900080830020658300206883002098760020A5
:1057A0002C1C00209D1C00201F85EB5111469046AB
:1057B000964693460292FEF7C9BA4FF0240872E467
:1057C0000121D8F80420D8F8083084F8181106A868
:1057D0000692079321F09EFAA7E6DFF8C0B29BF885
:1057E0000020002A3FF412AEA449B4F816810888BC
:1057F00002914FEA08184FF0640E1FFA88F80EFB6A
:1058000000204FEA420EB0FBFEF048EA00281FFAE3
:1058100088F8C0F3032048EA00080620019221F02E
:1058200067FA5FFA88F021F039FA4FEA182021F080
:1058300035FAB4F81601019A914B0299013080B201
:1058400090FBF2FC02FB1C02587AB1F80080A4F82D
:105850001621012800F0E4805A7B6E2303FB08F830
:10586000152198FBF1F8002A40F0D3803A2021F06E
:105870003FFA1FFA88F84FF0640BB8FBFBF291B2C5
:10588000C8B20292019121F009FA0199080A21F0A7
:1058900005FA3B2021F02CFA029A0BFB128080B211
:1058A0000A22053090FBF2F0C0B221F0F7F9002097
:1058B00021F0F4F9DFF8E0B1282021F019FA4FF0D7
:1058C0000A08DBF8002092FBF8F85FFA88F021F074
:1058D000E5F9C8F3072021F0E1F9042021F008FAE6
:1058E000BAF80620002A7DD1DBF8082082F31008E0
:1058F0005FFA88F021F0D2F9C8F3072021F0CEF941
:1059000084E5604904260EE5112021F0F1F9B8F88C
:1059100012205D494FF4F36B0BFB02F281FB023165
:10592000D217C2EB6132D0B2019221F0B7F9019ADD
:10593000C2F3072021F0B2F9192021F0D9F9B8F803
:10594000122052490BFB02F281FB0230D217C2EB4C
:10595000601281FB0230D117C1EB6011642000FBA3
:105960001120C0B221F09AF9002021F097F99AF89D
:105970000020B8F80CB092077FF556AD5FFA8BF7B0
:105980004FEA1B2B52E54FF00008404632E54046F7
:105990001BE5938907EE903AF8EE677AFEF71FBF92
:1059A0004FF01008FFF77FBB4FF02008FFF77BBBDD
:1059B000374B1B6898067DF557AD94F82431002BC2
:1059C0007DF46FAD334BC4F82C312D2384F8303186
:1059D000FDF751BDD8B221F061F9019B180A21F001
:1059E0005DF978E503F06AF921F058F9002021F01B
:1059F00055F90BE54FF00808FFF755BBCA690B6A6C
:105A00009A423CBFC8681218D31AE9E51146FEF75E
:105A10009DB91FFA88F89BF8002098FBF2F825E75B
:105A2000392021F065F95FFA88F021F037F94FEA63
:105A3000182021F033F93DE71146904696469346EB
:105A400002929146FEF782B9134B9146B3F90030AA
:105A50006420FEF771B811469046FEF777B91146FB
:105A600090469646FEF772B9114690469646934682
:105A7000FEF76CB94FF0FF3364E600BF9476002068
:105A800098760020D861040889B5F8141F85EB5179
:105A900064690020AC840020D4810020A676002018
:105AA0002DE9F04F2DED028BC74B1B7891B0072BE2
:105AB000069001F0118300230893C44B1B680593E3
:105AC0005D0500F1E286C24BD3F8008018F0080FA4
:105AD00040F07986BF4BC04DB3F800B0DFF81CA38F
:105AE0000793BE4BBE491E68B1F906907289914575
:105AF00080F2A784BB4B4FF07E521A60BA4F9AF9DE
:105B00000420B1F900C03C8B9AF800009AF801E03B
:105B1000002AACEB040314BF01224FF0FF32002B2C
:105B200040F3F184B3F5FA7FC0F2F3844FF4FA73D3
:105B30001B1A07EE903AF8EEE77AA445C5ED007A15
:105B400003DAF1EE677AC5ED007AB1F902C0ACEB89
:105B50000403002B40F3E484B3F5FA7FC0F2E6843B
:105B60004FF4FA731B1A07EE903AF8EEE77AA44561
:105B7000C5ED017A03DAF1EE677AC5ED017AB1F984
:105B80000430191B0029D8BFE11AB1F5FA7F80F261
:105B900052847145D8BF4FF0000E00F34E8402FBD3
:105BA0000EF207EE902AF8EEE77AA342059BC5EDC8
:105BB000027ABCBFF1EE677AC5ED027A13F4805326
:105BC000049300F0ED80B9F5FA6F4A46A8BF4FF490
:105BD000FA62B2F57A7FB8BF4FF47A72A2F57A72A0
:105BE0008249DFF81CE281FB0230D317C3EB60135C
:105BF000581C6FF0630C3EF910003EF913E00CFBEB
:105C00000323A0EB0E0003FB00F381FB0321DB1752
:105C1000C3EB61139E440FFA8EFE07EE90EA049BDD
:105C2000B8EEE78A85ED038A002B40F075861BF0FD
:105C3000400F40F038856E4C18F0140F03D01BF461
:105C4000027F40F0F1866B4B1B781BB17B8B4B4581
:105C500080F20B8594F826301BB11BF0030F41F046
:105C60000D8094F82C20FB7F002A40F08286B97FBB
:105C7000002900F0C980022900F0D187032940F0F3
:105C8000B68797F82010C1EB411001EB8001C900E5
:105C900089B20233DBB2002A00F0B087002900F09D
:105CA000AD8755480068B1FBF0F10FFA81F9A4F80F
:105CB0005C90ABB307EE909AF8EEE77AF7EE006AE5
:105CC00086EEA77A012BD5ED007AD4ED1C6A77EE2B
:105CD000E67A67EE877AC4ED187A21D0D5ED017A9D
:105CE000D4ED1D6A77EEE67A022B67EE877AC4ED73
:105CF000197A15D0D5ED027AD4ED1E6A77EEE67AE0
:105D0000032B67EE877AC4ED1A7A09D0D5ED037AB2
:105D1000D4ED1F6A77EEE67A67EE877AC4ED1B7AD8
:105D200029490978092901F06585B9F1000F71DD6C
:105D300093B394ED1C7AD4ED187A77EE877A012B21
:105D4000C4ED1C7AC5ED007A21D094ED1D7AD4ED16
:105D5000197A77EE877A022BC4ED1D7AC5ED017AA8
:105D600015D094ED1E7AD4ED1A7A77EE877A032B4C
:105D7000C4ED1E7AC5ED027A09D0D4ED1F7A94EDF8
:105D80001B7A77EE877AC4ED1F7AC5ED037A013B63
:105D9000022BB8BF0223DBB2002A18BF02233AE06D
:105DA000798B8945C0F27084B9F5FA6FD4BFC1EB25
:105DB0000903C1F5FA634FF47A7202FB03F2C1F5ED
:105DC000FA61B2FBF1F20BE76D75002058AA0020D2
:105DD00064690020E4830020A8760020EC83002082
:105DE00054C90020CC390020787400201F85EB5165
:105DF000D02800209022002074460020CC450020AE
:105E0000A8CA00200AD7233CA4F85C108946002ABF
:105E100000F07281022332785FED066AB17807EEF6
:105E2000902AF8EEE77AB0EE007A67EEA67ADB4ABF
:105E3000F4EEC77AF1EE10FA107840F3C084DFED8B
:105E4000D86A37EEC77AB0EE676AA7EE266AF0EE38
:105E5000466A95ED007A9FEDD36ADFF870E3DFF8CC
:105E600070C327EE066AF0EEC65ACEED005A8CEDEE
:105E7000006A99B107EE101AB8EEC75A9FEDCA7AB8
:105E800066EE064A25EE075AB7EE007A37EE457AF7
:105E900064EEA54AA5EE247A26EE076A9FEDC37A42
:105EA000727926EE877A27EE067AAAB1DFEDBE6A0E
:105EB0009FEDBF6A65EEA65A06EE902AF8EEE66AF6
:105EC00066EEA56AF4EEC66AF1EE10FA40F3638658
:105ED0009FEDB86A27EE067A0C289FEDB78ADFEDB2
:105EE000B76ADFF8F08200F03186B4EEC87AF1EEDE
:105EF00010FA98BFB0EE478AB4EEE68AF1EE10FAD7
:105F0000B8BFB0EE668A88ED008A002B00F0E6800C
:105F1000B0EE007AF4EEC77AF1EE10FA05DD37EE56
:105F2000C77ADFED9F6AE7EE267A95ED017ADFED1D
:105F30009D6A27EE267AF0EEC75A8CED017ACEEDF7
:105F4000015A99B106EE901A9FED976AF8EEE66A4B
:105F500027EE075A66EE866AB7EE006A36EE666A84
:105F600025EE255AA6EE856A27EE067ADFED8F6AC2
:105F7000B27967EEA67A67EE877AFAB107EE102A51
:105F8000B8EEC77A9FED886ADFED896A27EE257A39
:105F900027EE067AB4EEE67AF1EE10FA00F3F78512
:105FA000B5EEC07AF1EE10FA01F10281B7EE006AA7
:105FB00036EE477AC6EE076A67EEA67A0C2800F03E
:105FC000A685DFED7D6A9FED7D7AF4EEE67AF1EE4F
:105FD00010FA88BFF0EE667AF4EEC77AF1EE10FAA6
:105FE000B8BFF0EE477A012BC8ED017A76DD737801
:105FF000DFED6D6A07EE903AF8EEE77AB0EE007AE0
:1060000067EEA67A737AF4EEC77AF1EE10FA05DD40
:1060100037EEC77ADFED626AE7EE267A95ED027A0F
:10602000DFED606A27EE267AF0EEC75A8CED027A31
:10603000CEED025A9BB106EE903A9FED5B6AF8EE08
:10604000E66A27EE075A66EE866AB7EE006A36EE13
:10605000666A25EE255AA6EE856A27EE067ADFEDFA
:10606000536AF37967EEA67A67EE877AFBB107EE9B
:10607000103AB8EEC77A9FED4C6ADFED4D6A27EE15
:10608000257A27EE067AB4EEE67AF1EE10FA00F3FE
:106090007A85B5EEC07AF1EE10FA01F18580B7EE9F
:1060A000006A36EE477AC6EE076A67EEA67A0C28D3
:1060B00000F02585DFED406A9FED407AF4EEE67A48
:1060C000F1EE10FA88BFF0EE667AF4EEC77AF1EEE0
:1060D00010FAB8BFF0EE477AC8ED027A092800F04E
:1060E000048597F82150002D40F0B984344BD3F843
:1060F0000080002384F82C3018F0200F06D0079B76
:106100001B8803F03003002B40F040822D4D2E4FB2
:1061100095F82420DFF8C080DFF8C0A0531E082BBC
:1061200000F20781DFE813F02301A101A9000501B6
:106130005C000900A3010501B60198F80030002BAE
:1061400040F031852B68297A4FF4807203EB0121EE
:10615000002028F00DFC2B7A0133DBB2022B2B72CE
:1061600040F05881002028F043FC002028F040FC3B
:10617000FF2028F03DFC00F01F00052801F01B84E3
:106180001BF09AFBEE68002E00F04A8400222B6977
:1061900069680120B04795F82420BFE76D7500209D
:1061A000D7A368416F12033B0AD7233C0000484342
:1061B000A4707D3F0000C84200C0F94400C0F9C48B
:1061C00064690020A0C7002050D40020FC390020C2
:1061D000F0390020D4390020947C00207060024007
:1061E0004FF4007128681BF019FB012800F01D8591
:1061F000C0F03286022840F00D811BF085FB1BF0B9
:106200005BFBEE68002E00F00B84002210462B6929
:106210006968B04795F8242080E71021CF481BF02B
:10622000FDFA8346002840F0F38001217F2024F00E
:106230000DFB0128814640F0EB805846022124F0F6
:1062400005FB002801F05B82012840F0E180162167
:106250003A2024F0FBFA431C9B02EB631BF054FB37
:106260003068F3F76FFC00210A201BF0F5FA0028D4
:1062700040F06487032385F8243010210CA81BF01C
:10628000CDFA002840F0C6809DF83A209DF83900EC
:106290009DF83C109DF83D309DF83B60120442EAA9
:1062A00000620A431B019DF83E109DF83100DBB2ED
:1062B00043EA111342EA062203F5FA636A632B8765
:1062C0009DF832209DF8383042EA002201F00F019B
:1062D000180903F00F0385F83A106A859DF830100D
:1062E0009DF8332085F832309DF8343085F8281039
:1062F00085F82C209DF835109DF8362085F82D3036
:106300009DF8373085F8303085F8310085F82E104B
:1063100085F82F201BF0F8FAAB7E002B00F00D81E2
:106320008F4828F0B9FB002304222B6285F8242033
:106330000323DBB2022B73D9042A00F0BE80082AA3
:1063400000F0BB80874B1B7823B9874EB278002AB8
:1063500040F09685069801F00BFF844B1B78072BC5
:1063600000F0158511B0BDEC028BBDE8F08F804EBA
:106370003068F3F7E7FB002108461BF06DFA814611
:106380001BF0C2FAB9F1010F44D130684FF0000B95
:1063900085F819B0F3F7D6FB40F2AB1108201BF0DB
:1063A0005BFA052800F0A684012800F0AA861BF0FD
:1063B000ABFA6B7E002B01F0FA82022385F82430C1
:1063C0003068F3F7BFFB6B7E022B14BF4FF0000960
:1063D0004FF08049002137201BF03EFA4946292022
:1063E0001BF03AFA81461BF08FFAB9F1000F11D178
:1063F0006B7E022B00F0928685F81A903068F3F7D6
:10640000A1FB002109201BF027FA00283FF405AF6B
:106410001BF07AFA95F82420531EDBB2022B8BD89E
:10642000544B69691B685B1AC82B88D91BF044FA66
:1064300095F8242080E74FF4FA71A1EB0E0EFFF7D8
:10644000AEBBB9F5FA6FC0F22281337AC3F16403AF
:1064500007EE903A9FED487A484BF8EEE77A67EE00
:10646000877AC3ED007AFFF749BB414EA8E70826BB
:10647000FF2028F0BDFAFF2800F09484013EF7D1F8
:106480006B693A68FA339342C4D21BF015FA95F857
:10649000242043E6FF2028F0ABFAFF284FF008063F
:1064A00006D0013EECD0FF2028F0A2FAFF28F8D158
:1064B0001BF02AFA042385F82430314D1BF078FEB6
:1064C0006B78022B00F00D86032B7FF43BAF41F27B
:1064D000B813EB5C002B41F0338141F2A403EB5C79
:1064E000002B41F0288141F2E803EB5C002B41F0E6
:1064F0002C8141F22C13EB5C002B3FF423AF21489D
:106500001EF00AFC1EE7A4EB0C03B3F5FA7FBFF6FE
:106510000DAB9842FFF60CABDFED1B7AFFF70DBB1E
:10652000A4EB0C03B3F5FA7FBFF61AAB9842FFF663
:1065300019ABDFED157AFFF71ABB0D4E3068F3F794
:1065400001FB4FF4007110201BF086F906461BF08A
:10655000DBF9002E3FF4E4AE97E700BFE0C7002070
:1065600000380040084D002078D100206D750020D3
:10657000987C002050D400200AD7233CCC3900203E
:1065800018B3002044C4002000000000C54B1B7855
:10659000D8077FF5BBADC44BC44AB3F90430DFED77
:1065A000C47A82FB0312DB17C3EBA2031BB208EE13
:1065B000103AB8EEC88A28EE278AB0EE480AF4F7F7
:1065C00071FBF0EE408AB0EE480AF4F7F1FAB94BED
:1065D000D878002800F03286B749B4F98A20B1F99A
:1065E000023044F250659B1AAB4241F3CD80A3F5D3
:1065F0000C43A03B45429D4201F3C3808342A8BFA8
:106600000346B1F90010B4F9886013448A1B44F2C0
:1066100050611BB28A42A4F88A3041F3BD80A2F5D2
:106620000C42A03A954203DC9042A8BF10460546B2
:10663000721912B207EE902A07EE103AF8EEE77AD6
:10664000F8EEC76A27EEE87A60EE277AA0EE267A9F
:106650009A49A4F88820E8EEA67ADFED996A27EE39
:10666000267A67EEA67A00F005BE964B1B78012BC2
:1066700000F08283192B00F07F830E2B3FF4EAAAEF
:10668000082B3FF4E7AA7CE31A46FFF798BB307A61
:10669000A9EB020303FB00F3C2F5FA6293FBF2F3EA
:1066A000C3F16403D4E6804B8049B3F90430864CCF
:1066B000DFED7F6A22889FED857A81FB0301DB177E
:1066C000C3EBA1039B1A1BB207EE903AF8EEE77AF0
:1066D00067EEA67A77EE876ABDEEE66A16EE103AA6
:1066E0002033402B40F27183DFED796ABDEEE77A0B
:1066F00017EE103A2033402B00F264839FED757A39
:10670000F4EEC77AF1EE10FA41F33780DFED725AFA
:106710009FED726A01E0F0EE477AF4EEC67AF1EE90
:1067200010FA37EEE57AF6DCDFED6D7AB4EEE77A53
:10673000F1EE10FA41F11D80DFED675A9FED696AB5
:1067400001E0B0EE677AB4EEC67AF1EE10FA77EEB9
:10675000257AF6D49FED5D7AF4EEC77AF1EE10FA61
:1067600000F3C3829FED607AF4EEC77AF1EE10FA7F
:1067700044BF9FED5B7A77EE677A67EEA75A9FED8D
:106780005B5A9FED5B6A9FED5B7AA5EE856A27EE0B
:10679000A55AA5EE867AE5EE077A95ED016AD5ED64
:1067A000005A27EEC67A65EEA77AA5EEA67AE6EE3F
:1067B000267A85ED007AC5ED017AFFF73DBAF0EE55
:1067C000676AFFF746BB4C4D4C4BD5ED027A0793F9
:1067D000B2EE0E7AF0EEE76AF4EEC76AF1EE10FA66
:1067E000B3F800B0304B42D51BF0040F3FD0B3F9E3
:1067F00004302E4A4249DFF81CA1098882FB0302BB
:10680000DB17C3EBA2035B1A9BB21AB212F1B30FF0
:10681000BCBF03F5B4731AB2B32AC8BFA2F5B473F0
:106820002049C8BF1AB29AF804300978002B4FF6F5
:10683000FF7318BF01230C077FF553A9314909687D
:1068400012FB03F3097E304A9BB211FB03F382FB78
:1068500003121A44DB17C3EB221307EE103AB8EE0B
:10686000C77A77EEC77AC5ED027AFFF73AB9B3F97E
:1068700004300E49224ADFF89CA081FB0301DB179C
:10688000C3EBA1031380FFF72CB920488368002BCA
:106890003FF419A900F1440198471D4B1B6805936B
:1068A000FFF711B965830020948300206766666650
:1068B00035FA8E3C984A0020F44A0020EC3900203A
:1068C000CDCCCC3D78460020D0280020DB0FC93F3E
:1068D00000000000DB0F4940DB0FC940E4CB16414C
:1068E000DB0F49C0E4CB16C1DB0FC9BF92E741B94A
:1068F0009730083C15A82ABEA8760020E483002023
:10690000144B0020E8830020898888882C610020AF
:1069100058AA0020CC4500201D21C848F4F79AFA57
:1069200000283FF484A9C64BDB78002B7FF47FA9B5
:10693000DFEDC47AC44938EE678AC4F5FA62FDEE29
:10694000C87A12B2CDED097ABDF924301B0381FB60
:106950000301DB17C3EBA11302FB03F343F30F3374
:10696000234407EE903AB8EEE78A85ED038AFFF7F5
:106970005EB9B649B148D1F8EC10006844F6206E13
:106980007145A8BF7146B1F57A7FB8BF4FF47A71EF
:1069900089B2C006E18540F1B1810498002840F039
:1069A0000B84AB48D0F800A0BAF936B0DFF898E213
:1069B000206BD5ED037AAEFB01E14FEA911E642115
:1069C00091FBFEF11429BDEEE77A04EB400CA8BF61
:1069D000142101308842206317EE109AA4BF0020D2
:1069E000206304EB4000ACF83490B0F9341007EEAB
:1069F000101AB8EEC77A77EEC77AFDEEE77ACDEDDA
:106A0000047ABDF9100080EAE071A1EBE07159450C
:106A100000F3A0868F494FF07E500860FFF727B93A
:106A200095F82420FFF77ABB8B4B1B7813F01003EB
:106A300000F074812279A36895ED017A002A0CBFD9
:106A400001224FF0FF3203FB02F307EE903AF8EE1B
:106A5000E77A77EE877AC5ED017AFFF7F4B81E2161
:106A60007648F4F7F7F900283FF440AB079B1B8802
:106A70005E063FF53BAB94F88030AB4240F00687B2
:106A8000764BD4ED217AD3ED006A98ED025ADFED12
:106A9000745A9FED746A27EEC57A68EE277AA8EEDD
:106AA000267AE5EE267AB4EEE57AF1EE10FA88BFA2
:106AB000B0EE657AB4EEC67AF1EE10FAF4EEE57A4D
:106AC000B8BFB0EE467AF1EE10FA88BFF0EE657A04
:106AD000F4EEC67AF1EE10FAB8BFF0EE467A88ED21
:106AE000007AC8ED027AFFF701BBFDEEC87A5E4A74
:106AF00017EE903AA2F80490D380FFF7F2BABDEEF9
:106B0000E77A594B17EE102A9A80FFF7D3BA9FED18
:106B1000547ADFED546A5449F4EEC77AF1EE10FA74
:106B200098BFB0EE677AFDEEE77AB4EEE67AF1EE62
:106B300010FA17EE902AB8BFB0EE667A012B88EDF6
:106B4000017A4A803FF753AAFFF7CBBAB4EEC87A6E
:106B5000F1EE10FA98BFB0EE478ABDEEC77AB4EEF8
:106B6000E68ADFF804A1F1EE10FA17EE102AB8BF9A
:106B7000B0EE668A88ED008AAAF80020002B7FF428
:106B8000C7A9FFF7AEBADFED396AFFF78EBADFEDBE
:106B9000376AFFF711BAF7EE005A75EEE66A85EE2E
:106BA000A66AFFF797B9324B596889067FF5C7ABDC
:106BB0002022DA60DAF800202E4B22F00102CAF817
:106BC00000201A89D20700F19F8022F00DFF0028D3
:106BD000FBD1284A938823F002031B041B0C9380EB
:106BE00098F80030002B7FF4BDAAFFF7ABBA22491A
:106BF00002334988DBB2002A7FF450A8B4F85C90D5
:106C000009F1FF390FFA89F9B9F1000FA4F85C9086
:106C10003FF78EA8002A7FF4FDA8FFF76DBAE18D3B
:106C200001F57A7189B2FFF734B86B693A68643359
:106C30009342FFF4E2AAFFF7EDBB00BFACD1002006
:106C4000E07A002000007A44D34D6210B01D00208D
:106C5000E88300206C0000206583002030000020C5
:106C600000C0F94400C0F9C4707500200000C8429B
:106C7000006002400038004090850020894ADFED26
:106C80008A7A92ED080A0993B4EEE70AF1EE10FA57
:106C900040F2808229F0C6FED4ED0A7A20EE270A5F
:106CA00029F02AFEB0F5617F099B00F38E8207EE82
:106CB000900AF8EEE76ADFED7D7A66EEA76A07EEE6
:106CC000903AB8EEE77AFDEEE67A17EE903A203386
:106CD000402B40F2CC869FED760A29F00DFE00B2E3
:106CE00007EE900AB8EEE77A56E29FED727A77EEF9
:106CF000677A42E585F81990FFF759BB0598C000FF
:106D00003FF54BAEFEF7B3BF9A891A89D207FBD481
:106D100022F06AFE00287FF458AF5AE79AF8032061
:106D2000002A40F0B382B4F90CE09AF80210A9EB03
:106D30000E0383EAE370A0EBE370884240F33485EE
:106D400003EBD37301225B10E36184F820202275EA
:106D5000A3689E44BEF5FA6FA8BF4FF4FA6EBEF565
:106D60007A7FB8BF4FF47A7E07EE90EAF8EEE77AC2
:106D7000C5ED037AFEF767BF4F4B9B7B002B7EF47C
:106D800069AF4E4A0023AB609360FEF763BFF9F72B
:106D9000BDFB089A4A4B801A988011B0BDEC028B5B
:106DA000BDE8F08F2B6A0022012B2A7641F2898000
:106DB000EA69013B01322B620823EA6185F824303D
:106DC000FFF77BBBDFED3A7AE7E4F4EEC77AF1EE4A
:106DD00010FA40F3E485DFED3B5A9FED3B6A01E09A
:106DE000F0EE476AF4EEC66AF1EE10FA36EEE57A96
:106DF000F6DCDFED366AB4EEE67AF1EE10FA40F139
:106E0000D285DFED305A9FED326A01E0B0EE667A4E
:106E1000B4EEC67AF1EE10FA77EE256AF6D49FED5D
:106E20002D7AF4EEC76AF1EE10FA40F398819FEDE7
:106E3000217A77EE666A66EEA65A9FED275A9FED95
:106E4000276A9FED277AA5EE856A26EEA55AA5EE5C
:106E5000867AE5EE076A49E41AF056FDEE680423E7
:106E6000002085F824302876002E3FF426AB2B69CD
:106E70002A686968B04795F82420531EFFF7CDBAF9
:106E8000184F3B78013B0A2B7BD8DFE813F08D02CB
:106E90007F02480233021C02E802D202BF029C02B7
:106EA00003032D00743A00208FC2753CD06D393A2F
:106EB00000000000DB0F4940106F0020D439002093
:106EC00070750020DB0FC940E4CB1641DB0F49C0D1
:106ED000E4CB16C1DB0FC93F92E741B99730083CBC
:106EE00015A82ABE1C530020022A38D1C34BDFF854
:106EF00048831B78002B41F07E80D8F8005045B3C2
:106F00002B7833B395F82820002A40F034812B7E6B
:106F1000AA6385F83C20042285F8282013F0080392
:106F20006A6AEA622A6303D0B54A41F29413D358DD
:106F30006B634FF00009C5F82490C5F80890C5F8B8
:106F40000C90284623F034FC0523C5F8409085F8C2
:106F5000283000220423C8F8002088F81430A94BF8
:106F6000A94A5B681268C833934204D325F0A4F998
:106F7000002800F0D281B278032A01F06F8001234B
:106F80003B70022A00F0F780F378002B3FF4E2A96F
:106F90009E4B1B68D90440F1B0859D4B9B8807EE42
:106FA000903AF8EEE77A9B4991ED012AD1ED022A59
:106FB00091ED033AD1ED043A91ED054AD1ED064A3F
:106FC00091ED075AD1ED085A91ED096AD1ED0A6A9F
:106FD00091ED0B7AB4EE672AF1EE10FAF4EE672A1F
:106FE00014BF01230023F1EE10FAB4EE673A18BF84
:106FF00043F00103F1EE10FAF4EE673A18BF43F0E4
:107000000103F1EE10FAB4EE674A18BF43F0010332
:10701000F1EE10FAF4EE674A18BF43F00103F1EE07
:1070200010FAB4EE675A18BF43F00103F1EE10FAFC
:10703000F4EE675A18BF43F00103F1EE10FAB4EE14
:10704000676A18BF43F00103F1EE10FAF4EE676AC5
:1070500018BF43F00103F1EE10FAB4EE677A18BFDF
:1070600043F00103F1EE10FA18BF43F00103002BC7
:1070700040F07B8491ED007AB4EE677AF1EE10FA7D
:1070800040F07384604DD4F890102B68994200F260
:1070900073843B78012B3FF45DA994F88C20002A7F
:1070A0003FF458A90B2B0DD801229A4040F603015A
